:020000040000FA
:1000000021EF01F01200FFFF10EF04F01200FFFFDC
:100010000000909400000000909000000000908686
:10002000016A1E0E015C32E20150EA6A000FE96EBD
:10003000060EEA22EF50046E909204B090829084F3
:100040009094909204B2908290849094909204B490
:10005000908290849094909204B690829084909430
:10006000909204B8908290849094909204BA908276
:1000700090849094909204BC9082908490949092FA
:1000800004BE908290849094012ACBD79092000075
:100090000000000090961200000090800000000018
:1000A0009086010E016E100E015C0DE000500114EF
:1000B00002E0908201D09092000090840000909421
:1000C000019E0146F0D7909200000000909600003B
:1000D0000000909012000000016A1E0E015C09E20F
:1000E0000150EA6A000FE96E060EEA22EF68012A63
:1000F000F4D712000000016A1E0E015C09E20150F3
:10010000EA6A000FE96E060EEA22EF6A012AF4D7C6
:10011000120000000068C0DF0168010606E00A0E58
:10012000026E020601E0FDD7F8D7550E006EB4DF6F
:10013000E1DF12000000EDDF06010F6B0601106B1E
:100140000601390E116F0601080E126F0601136BBE
:100150000601A80E146F0601156B0601166B060149
:10016000900E176F0601800E186F06010A0E196FA8
:100170000601810E1A6F0601BA0E1B6F0601200ED2
:100180001C6F06010A0E1D6F43DF12000000810E76
:10019000C96E37D8FC0EC96E34D88E8E00000000B0
:1001A000000000008E9E120009014E6B09014A07F3
:1001B000000E4B5B09014D5109014C5D01E0C96A1C
:1001C0004E2FFED709014D5109014C5D02E04CC98B
:1001D000C9FF4E2FFED78E8E8E8E8E9E4CC94DF946
:1001E000120000000900F5CF49F90900F5CF48F9E0
:1001F00009014851090146270901495109014723CD
:10020000120000000901486B496B0901540E485D5A
:100210003D0E495905E20901482B000E4923F5D747
:1002200012000000210EC26EC09EC2820000C2B247
:10023000FED7C4504D0802E2010E02D0000E00D0DD
:100240001200C16A210EC26E896A300E8A6E030ED8
:100250008B6E700E8C6E320E8D6E040E8E6E8F6AEB
:10026000800E906E916A92680F0E936E900E946E4F
:10027000956A9D0E966E7B0E976E070E986E300EE9
:10028000996E9A688D8CC79EC698C78CF00EC6165C
:10029000C680C68A240EAC6E190EAF6E900EAB6E81
:1002A00075DF0901516BBDDF000904E10A0E090188
:1002B000515D09E2640E0901515D05E2A2DFA1DF93
:1002C0000901512BF0D709015151630802E289EF6E
:1002D00001F00901466B476BF66A080EF76EF86A83
:1002E00080DF000009014851491102E102EF04F0EA
:1002F00078DF800EF61805E1FD0EF71802E1010E19
:10030000F81801E0F5D709014651471102E102EF63
:1003100004F001D8120000000DDF09014C6B090147
:100320004BA703D00901010E4C6F3EDF9EAA29D0D6
:10033000ABA209D0AB980000000000000000000054
:100340000000AB881ED0AECF4FF9ACA2FED7490E4D
:1003500009014F5D0BE14B0EAD6EACA2FED7330E23
:10036000AD6EACA2FED7410EAD6E06D0FF0E0901F8
:100370004F5D02E04FC9ADFF440E09014F5D01E141
:1003800001D0CBD709014A6B4B6B0901020E4C6FB0
:1003900009014AA902D009014C6B06DF2FD8020ED1
:1003A000F85C05E1420EAD6EF86A0ED8FF000CD87D
:1003B000410EAD6EEAD712000000550EA76EAA0ED0
:1003C000A76EA68200001200940EA66EF5DF000E46
:1003D000E96E090EEA6E0A000901080E446F090170
:1003E000080E456FEE50F56E0F00452FFBD7840EBB
:1003F000A66EE2DF442FF3D7A69412000000090195
:10040000506B0901446B440E0901445D1FE29EAA32
:10041000FED7ABA209D0AB9800000000000000009E
:1004200000000000AB8802D0AECF4FF90901445163
:10043000EA6A000FE96E090EEA224FC9EFFF0901CF
:100440004F51090150270901442BDDD709015051B3
:100450000BE1030E0901425D07E240C9F6FF41C905
:10046000F7FF42C9F8FF03D04E0EAD6EC8D7120099
:10047000FFFFFFFFFFFFFFFFFFFFFFFFFFFFFFFF8C
:10048000FFFFFFFFFFFFFFFFFFFFFFFFFFFFFFFF7C
:10049000FFFFFFFFFFFFFFFFFFFFFFFFFFFFFFFF6C
:1004A000FFFFFFFFFFFFFFFFFFFFFFFFFFFFFFFF5C
:1008000000001200280EE66EEEECFDF0E552A2EFBD
:10081000FDF01200FFFFFFFFFFFFFFFFFFFFFFFFE5
:10082000FCEF2AF01200FFFFFFFFFFFFFFFFFFFFBB
:100830000000AEECE5F01D0E4A6EF00E4B6E010EA0
:100840003CEFF0F0AEECE5F0900E4A6EF00E4B6E21
:10085000010E3CEFF0F0AEECE5F06B0E4C6EF10EDD
:100860004D6E010E4E6EFE0EDBCF4FF0506A516A98
:10087000D8904F36503651364C504F24F36E4D5071
:100880005020F46E4E505120A4ECF0F00900F5CF4A
:100890004AF00800F5CF4BF097ECF3F0B3EFE5F03A
:1008A0000FECF0F0010EE66EFD0EDB500301A72504
:1008B0004A6EFE0EDB50A821000199ECF4F0C6EC64
:1008C000EEF094ECEDF0DF50E552B3EFE5F030ECF4
:1008D000F0F04B6A020F4A6E010E61ECF0F0B3EFDC
:1008E000E5F0AEECE5F0C00E4A6EEF0E4B6E010E79
:1008F0003CEFF0F030ECF0F08DECF2F0FD0EDB5060
:100900008BECE6F0EF50B3EFE5F031C1E6FFA3DF8B
:10091000E5521200440E01243BEFEBF0AEECE5F0A3
:10092000D50E4A6EEB0E4B6E010E3CEFF0F0075009
:10093000B1ECF4F081ECF0F0006E12007EEFEAF022
:100940000A0E4A6E4B6A21EFF5F09DECEFF021EFB5
:10095000F5F0E80E4A6E030E4B6E21EFF5F09DECBC
:10096000EFF04AC23EF04BC23FF059ECE6F03E5089
:10097000006E120001012D51010B1CE07A51200B79
:1009800019E0E751010B16E0CE51080B13E0100EF1
:100990002E5D10E22E5107080DE23E51100B0BE0C8
:1009A0009FECE9F008E0100E0101635D03E2635182
:1009B000070801E3000C010CABECEBF00EE00201C8
:1009C000BC51100B0AE03450400B08E00101DC512F
:1009D000010B03E09FECE9F001E1000C010CE66A79
:1009E00075EC2EF0E5521200FC0EE66EED0EE66E92
:1009F000010E37ECEAF0E5521200010EDBEFE5F0F4
:100A0000020EDBEFE5F0B3C2E6FFE50EC3EFE5F063
:100A1000E66AE50EC3EFE5F080EC14F0000918E09B
:100A200080EC14F0000914E0960E3EECE6F06DEC5C
:100A30000FF02BB00DD080EC14F0000909E080EC31
:100A400014F0000905E0DB0E48ECE6F084EC0FF052
:100A500012000101E651010B03E05951080B02E1BC
:100A6000000E01D0010E000903E00201BA5112008C
:100A70000201B6511200AEECE5F00101E651010BA6
:100A800007E05951080B04E0FE0EDBCFBAF203D0A9
:100A9000FE0EDBCFB6F2B3EFE5F00301D251020157
:100AA000F05D0301D3510201F15913E3F051030149
:100AB000D45D0201F1510301D5590BE3D25102017A
:100AC000EE5D0301D3510201EF5903E318ECEDF0A1
:100AD00008E2D2C3F0F2D3C3F1F2D2C3EEF2D3C331
:100AE000EFF212002CECF0F0FF0805E1CBECE5F0A2
:100AF000090E5AECE9F09CECF3F04A6E0A0E4A5CDF
:100B00000BE3CBECE5F00F0EEF14000938ECF4F03A
:100B1000090ECAECF0F0EF8E1200B5ECE8F003E13C
:100B2000040E4B5D12004B5112002EECECF01394AE
:100B30001396198C0490A5EC55F001019151400BCE
:100B400009E14C51320806E2320E4C6FEEEC80F0B7
:100B5000020117870C500EE1010191AD09D033EC71
:100B6000ECF00A01D76BE66AEBEC91F0E55212006B
:100B7000B9EC4BF01200800E081406E02150010B76
:100B800003E10201315101E0000C010C800E081458
:100B900003E02150010B01E0000C010C0C500AE1B4
:100BA00001019151400B06E03550400B03E121500B
:100BB000800B01E0000C010C0201010E4D6FE20EF2
:100BC00048ECE6F01E0E096E12009BEFEDF030ECE3
:100BD000F0F004080FE011ECE7F00EE0FE0EDB5041
:100BE0000A0808E0FE0EDB500D0804E0FE0EDB50A4
:100BF000090802E1010E01D0000EB3EFE5F0070194
:100C0000C707C551C52BEA6A000FE96E0C0EEA2230
:100C1000EF5012000101E551100B03E00401FA51FD
:100C20000AE1420EE66E460EE66E8FECCDF0E5521E
:100C3000E5520101E5891200D9CFE6FFE1CFD9FFE6
:100C4000FE0EDB50D80805E1300EF36EFE0EF3CF3A
:100C5000DBFF060EAB1406E0AB98000000000000BE
:100C6000AB888FD1FE0EDB50100805E0FE0EDB5086
:100C7000110801E02BD10201050E296FFE0EDB5099
:100C8000110837E1020134510DE12150800B0AE1D6
:100C9000050105013B51010B0AE1050105013B512D
:100CA000400B05E1100EE66E86D9E55222D0050113
:100CB00005013B51400B02E00F0E01D0060EE66E1F
:100CC0007AD9E552C3C1E6FF76D9E552C4C1E6FF41
:100CD00072D9E552C5C1E6FF6ED9E5520A0E01018F
:100CE000C603F3500101C725E66E65D9E55205013B
:100CF0003B910401F0514A6E4B6AD8904B5004E688
:100D0000D30E4A5C000E4B5801E3DFD005013B5186
:100D100001E1DBD00201345101E0D7D02150800B3A
:100D200001E0D3D0049005013BA11AD001010101DB
:100D3000E551080B03E00401FA510DE1410EE66EA6
:100D4000460EE66E8FECCDF0E552E5520101E587E7
:100D500005013BB35FDF05013B9305013B91B5D036
:100D600005013BA304D056DF05013B93AED005013E
:100D70003BA725D0440EE66E4D0EE66E8FECCDF00F
:100D8000E552E5520480440EE66E4D0EE66E8FECA1
:100D9000CDF0E552E552030E0C5C04E0030E0101B8
:100DA000D35D08E1540EE66E440EE66E8FECCDF096
:100DB000E552E55205013B9705013B8586D00501CB
:100DC0003BA524D0570EE66E420EE66E8FECCDF0BA
:100DD000E552E5520480570EE66E420EE66E8FEC49
:100DE000CDF0E552E552530EE66E490EE66E8FECFD
:100DF000CDF0E552E552490EE66E460EE66E8FECFA
:100E0000CDF0E552E55205013B955FD005013BA9C8
:100E10000BD0410EE66E500EE66E8FECCDF0E55233
:100E2000E55205013B9951D005013BAB0BD0410E7A
:100E3000E66E520EE66E8FECCDF0E552E5520501FE
:100E40003B9B43D005013BAD13D04F0EE66E520ED7
:100E5000E66E8FECCDF0E552E552540EE66E520E82
:100E6000E66E8FECCDF0E552E55205013B9D2DD0AD
:100E700005013BAF2AD04E0EE66E4C0EE66E8FECAF
:100E8000CDF0E552E552560EE66E440EE66E8FEC5E
:100E9000CDF0E552E552420EE66E530EE66E8FEC53
:100EA000CDF0E552E552570EE66E430EE66E8FEC3E
:100EB000CDF0E552E5524E0EE66E420EE66E8FEC38
:100EC000CDF0E552E55205013B9F5BD0200EF36E5D
:100ED000FE0EDBCFF4FFF350F45C04E3FE0EDB50B8
:100EE0007E0807E2FE0EDBCFE6FF71DEE552000969
:100EF00048E0FE0EDB503B0804E0FE0EDB507C08B1
:100F000002E10401F92B01010101E851800B0BE022
:100F1000FE0EDB503B0807E180C1E6FFBBEC0EF0A4
:100F2000E5520101E89FFE0EDB50210804E0FE0EB1
:100F3000DB5040080AE13B0E0401FE5D04E07C0E3C
:100F40000401FE5D02E10401F92BFE0EDBCFFEF48D
:100F50000401F151EA6A000FE96E0B0EEA22FE0E5F
:100F6000DBCFEFFF0401F12B0401F02B0401F05162
:100F700008E10401FE6BFEC4F9F4FEC4F1F4FEC402
:100F8000F2F4E552E7CFD9FF1200ACA2120004013F
:100F9000F851B8ECF0F0006E0050E66E5DECFDF03C
:100FA000E5523B0E005C03E07C0E005C01E12A9000
:100FB0000401F82B1200AEECE5F0ACA2FED74FEC2A
:100FC000E6F05DECFDF0E552B3EFE5F08BEC13F0ED
:100FD00097EC13F0F29EF66A080EF76EF86A940E1C
:100FE000A66E550EA76EAA0EA76EA682000000EC94
:100FF00000F012000401F007F2513AECE9F0EF5072
:10100000006EF22B1200050E0C5C0AE12050020B60
:1010100007E10201B551020B04E1B551010B01E1F9
:10102000000C010C040E0C5C04E10101D151080B11
:1010300001E1000C010CC70EB1ECE6F000503208E3
:1010400003E33050400B09E0309C8BEC13F097EC3D
:1010500013F08BECB6F0DCEC13F0120013ECF0F0B4
:101060009C0EDE6E030EDD6E0301A551A61127E076
:10107000090EE66EFD0EDB50090DF350A5254A6EF4
:10108000F450A62199ECF4F09C0EE66E030EE66E89
:1010900094ECEDF0DFCFE9FFDF2A010EDBCFEAFFB2
:1010A00001E3DB2AEFCF00F0EF5024E0FE0EDB502F
:1010B00003E1E6EC97F0EED711EC98F0EBD7FE0EDB
:1010C000DB500BE171EC94F0160EE66EF40EE66E5A
:1010D000010EE66EFDEC97F00AD07DEC94F00E0E5A
:1010E000E66EF40EE66E010EE66E24EC98F0E55224
:1010F000E552E552020EE15C02E2E16AE552E16E80
:10110000B3EFE5F00490DCECF4F038E0048001018A
:10111000E3AB34D0CBECE5F00492EF50010B01E0EF
:101120000482A0ECF3F0016E050EEB50026EEF505E
:10113000080B01E0010EFDECF2F0FE0EEF14F310CF
:1011400038ECF4F0070EEB50E66E040EEBECF4F026
:10115000080EEB50E66E050EEBECF4F00450020BBB
:1011600002E0EF8601D0EF96CBECE5F0070E01C070
:10117000EBFFCBECE5F0080E02C0EBFF120005011F
:10118000005102012A113D1107E11C50010B03E13E
:101190004A514B1101E1000C010CAEECE5F00101EC
:1011A000E39D070110855BEC5EF04FECE6F036EC5A
:1011B00029F0E552070110955BEC5EF0080E3EEC5D
:1011C000E6F0B3EFE5F000000000000000008C98AE
:1011D00000000000000000001200000000000000FD
:1011E00000008C880000000000000000120053EC9A
:1011F00029F002016A6B6AC22AF23D6B4A514B1117
:1012000002E021949FD955EF81F00701EF51010BC6
:1012100007E0030E0C5C04E0050E0C5C01E0000C22
:10122000010C0101299D010E0E6E29BF0E681200EE
:10123000030EDBECE5F0268E12004D0EC6EFE5F056
:101240004E0EC6EFE5F001019151010B08E0C9EC2B
:1012500011F0000904E001013E51800B01E0000C97
:10126000010C040EDBECE5F03C0E096E1200268E3C
:10127000050EDBEFE5F08AECF2F08AECF2F000010B
:101280000F6E8AECF2F0106E1200E0ECF4F08AC1FE
:10129000E6FFDD0EC3ECE5F096C100F0A1ECEFF047
:1012A00005E1090E01019803F350006E0050E66E4F
:1012B000DE0EC3ECE5F022EFF0F0AEECE5F0490E07
:1012C00047ECF2F00F5010100BE0FE0EDB50EA6A14
:1012D000920FE96E010EEA220FC0EEFF10C0EDFF83
:1012E000B3EFE5F025A806D0010E076E020EE66EFC
:1012F000E4DFE552076AE66AE0DFE5521200AEEC91
:10130000E5F0FE0EDB5085ECE6F0EF5010E1FE0E4E
:10131000DBCF4AF0FD0EDB50D8804A5408E3FE0EC6
:10132000CBECEEF085ECE6F0100EEF6EEAD7B3EF03
:10133000E5F0830E0A6EFA0E29ECE7F000500F6E0E
:101340000FC010F00F6AFB0E35ECF5F000504BEFBC
:10135000F2F00101CF51800B01E0010E39ECECF00D
:101360003DC1EFFF12000101CF51800B01E0010EE2
:1013700039ECECF0EFCF3DF13D51140804E2010EE1
:101380003D6F2CA63D6B2CEFC6F0AEECE5F06DEC9E
:10139000EDF002E1EBC7EAF7FE0EDB0402E1EAC77B
:1013A000EBF7B3EFE5F0075003E03450400B02E0F9
:1013B0000C5012000101D35112000C50A5ECE6F0C4
:1013C00020EFEDF045C1E2F245C1E1F20C50D8EC5E
:1013D000F2F0400B03E00201040EE16F0101D35172
:1013E000D8ECF2F0400B03E00201040EE26F1200B1
:1013F0000FECF0F02950010B2AE12A0E165C06E1F1
:10140000085040ECEBF001E14B5021E00C0E165C73
:101410000BE108504C6E4D6A810E4C1805E14D50A1
:1014200003E102017E5113E0A2ECB6F0000909E0ED
:101430001A50400B06E1A9ECEFF003E12150100B2C
:1014400006E0190E165C05E1EEECE8F002E1000E94
:1014500001D0010EDF6E2D50800B03E12D50400BAB
:1014600002E0010EDF6E2990DF50E552B3EFE5F0A8
:101470001B9C248A1200010139AF05D004A002D0C0
:101480001B8812001B8A1200E0ECF4F0580EC6EC28
:10149000E5F01DBE02D09AECECF022EFF0F0010175
:1014A00039AF07D0060ECCECF1F0280E3EECE6F09A
:1014B000EBDF12000601980ED880B4553A0EB555F0
:1014C00009E20F50B45D0101D76F10500601B55904
:1014D000010108D0B4510F240101D76F0601B551A5
:1014E00010200101D86F12000101E4BF11D0160EC7
:1014F000AEECE9F0050E436E446A4AC23EF04BC2C0
:101500003FF0B8ECFDF03EC04AF23FC04BF2120093
:10151000110EAEECE9F0020E0F0B020105E0D890BF
:101520004B334A33E806FBE112001AB404D0370EFD
:101530003BECF4F0000C010C970EA5ECF3F0980EC8
:10154000DFEFE5F00101E5931C921C901A9A1492CA
:1015500022EC1EF002014A6B4B6B57DB9CEF0AF04A
:1015600013ECF0F0580EDE6E050EDD6E560E0F6EAB
:10157000010E106E0101E4AF07D0A80EDE6E030E5F
:10158000DD6EEA0E0F6E106A0D044A6E4B6A82EC35
:10159000F4F06FECF0F067ECF9F03CC0D7F13DC02F
:1015A000D8F101018DA706D076ECE8F0EE50D727F0
:1015B000EE50D823020EE15C02E2E16AE552E16EF0
:1015C000B3EFE5F0320E3EECE6F09F0E95EFF2F051
:1015D000AEECE5F0F7DF2250800B08E0350E165C2C
:1015E00005E10F681068410EDBECE5F004900101A5
:1015F0008DB704809DEC8FF000C70AF0FC0E016EE1
:1016000010C000F005EC4DF0012A0FC000F005EC11
:101610004DF00A6AB3EFE5F00FECF0F0010EDF6E6B
:1016200021AC06D0030EDF6E0101E58322EC1EF033
:10163000800EE4ECF4F0980EDFECE5F0D6C30FF08A
:10164000D7C310F0950E29ECF1F0E552B3EFE5F0B9
:10165000550EC6ECE5F01A801200540EC6ECE5F00B
:101660001A9012000FECF0F0FFEC26F0DF6EAFECFA
:10167000EBF007E01AA00ED0F0DFDF500BE1006ABC
:1016800007D01AB007D0E4DFDF5004E1010E006E8E
:1016900019EC92F0E552B3EFE5F0010162B702D028
:1016A0002EC163F17BECE8F0D0EFEEF0B3ECEBF0A1
:1016B00005E02050020B02E133ECE7F0120085EC6C
:1016C000E9F009E02150800B06E13E51100B03E0E8
:1016D0002050080B01E1000C010CB3ECEBF00EE024
:1016E0002150800B0BE12050080B08E03E51200BED
:1016F00005E12E50400B02E1095001E0000C010C05
:1017000068ECE6F003E03550400B04E001015A516B
:10171000040B01E1000C010C0FECF0F001018DA1B4
:101720000AD0FFEC26F0DF6EDF0403E0020EDF5C80
:1017300002E1010E01D0000EE552B3EFE5F0ADEC91
:10174000EFF005E1FFEC26F0040801E0000C010CCD
:10175000F6DF000904E1B1ECEFF001E0000C010C50
:101760008150080B0DE08150010B0AE068ECE6F0B7
:1017700003E071ECEDF004E11A50020B01E1000C02
:10178000010C8150080B19E08150020B16E08150CA
:10179000040B13E08150010B10E0050100510DE135
:1017A0002150040B0AE12150010B07E168ECE6F03F
:1017B00003E071ECEDF001E1000C010C810EA3ECF3
:1017C000E9F0010139BF268E120010C2E6FF0FC2F8
:1017D000E6FFC80EDFEFE5F01E9C9FECECF030DD7D
:1017E000EA0EA3ECE9F0268E120030ECF0F00A0DC0
:1017F000F3CF5AF3F4CF5BF3000E03015A27030E25
:101800005B23B3EFE5F00F0E07010E130E990E9F49
:10181000040E0101465D02E107010E8F100E010169
:101820002E5D14E2020E835D25E22E5102E10701D6
:101830000E9101012E0502E107010E9301012E51C7
:10184000020818E22E1D07010E1714D0835112E072
:10185000100E2E5DD5ECE8F08CC200F00A0E005C94
:1018600001E1006A001C07010E1739ECF5F0020BCC
:1018700001E10E89049007010EB704800E970EB3A4
:101880000E870E9304B00E8312008BECF1F004E689
:101890008A0E4A5C000E4B5802E2DEEF0BF08BEC36
:1018A000F1F004E6A90E4A5C000E4B5805E2020175
:1018B000E1510101275F12008BECF1F002E6D4EC5C
:1018C000EEF004E20201E151010127271200140E9B
:1018D0005EECE9F07EECF0F000501C0806E31450DA
:1018E000100B04E000500C0801E2010C000C85EC28
:1018F000E9F003E1DE51100B07E18D51400B03E0ED
:10190000DE51040B01E1000C010C9FECE9F002E058
:10191000060E01D0070EDBEFE5F007C0C8F2076A3C
:101920007BC101F07CC102F0B7ECEBF004E20701EF
:101930000551026E016E01900142029002424D0E6D
:10194000012404ECF3F0010E076E4D0E022404ECAA
:10195000F3F0C8C207F0120007010E9B0101D0ABE3
:1019600002D007010E8B12A007D007010E9B0101C8
:10197000D0AD02D007010E8B1200075006E03450A4
:10198000400B03E10201B25112000101E7A903D0AB
:101990000201B15112000A01D55112000201650E77
:1019A000C46F010EC56F075004E05F0EC46F010ED7
:1019B000C56F1200AAECF3F00FC1DFFF010E10C1DA
:1019C000DBFF34AC05D0DB50DF6E010E0FC1DBFF57
:1019D0001FECE7F085ECE9F037E107011051200B2F
:1019E00033E01051010B07E0DF500A0804E2010E5A
:1019F000DB500A0829E3010EDB50DF5C25E00A0E0C
:101A0000DF5C22E0DF50070804E20A0EE4ECE5F0B8
:101A10001BE3DF50050804E2080EE4ECE5F014E3F4
:101A2000DF50030804E2060EE4ECE5F00DE3DF50BE
:101A3000010804E2040EE4ECE5F006E3DF0406E14D
:101A4000020EE4ECE5F002E2020EDB6A020EDB506D
:101A500007E0080EDBECE5F0FA0E096E19861C882B
:101A6000030EE15C02E2E16AE552E16EB3EFE5F0FC
:101A7000070107979FECE9F006E0A6ECE9F003E028
:101A80000701078797DFBBEFEBF0AEECE5F02BA487
:101A900009D07CECEBF06BEC2EF065ECF4F0500E22
:101AA000096E2B94B3EFE5F0159E0A01DA51800B15
:101AB00006E1050E0C5C03E052ECE7F001E0158E48
:101AC00012000C50080DF2ECE7F0010EB5ECEFF04F
:101AD000E806FCE10250080D4C50F3244A6E4D50CC
:101AE000F4204A50016E12000A01DA8FDDDF020194
:101AF0009751A1ECE6F01AE24A509608000E4B54BA
:101B000015E20268960501E1026A030E965D02E1A4
:101B1000010E026EFF0E025C10E0A1ECEDF04FEC46
:101B2000F2F00150CEECF0F00A6A07D03FECECF096
:101B3000F9ECECF0178B05013B850201966B010176
:101B4000B28F500E096E2596328C12000201C769C1
:101B5000C7C2C6F2C7C2BCF7C7C2BBF7C7C2BAF793
:101B6000C7C2B9F7C7C2B8F7C7C2B7F70701C36999
:101B7000C469C169C269C1C7BFF7C2C7C0F7C1C7DD
:101B8000BDF7C2C7BEF712000101490503E1845049
:101B9000100B07E0020E495D03E18450100B01E1D8
:101BA000000C010C96880101495101E19698120040
:101BB0000FECF0F00101A65103E19C51200821E255
:101BC000DF6A090EDF5C10E2DF50D7ECE6F0EF5081
:101BD000040B08E0100EDF24E66E12EC35F0E5523F
:101BE000000902E1DF2AEDD7090EDF5C0AE2100EE0
:101BF000DF262A86DFCFE6FFD1EC34F0E552DF5056
:101C000001D0000EE552B3EFE5F020869FECECF03A
:101C1000B299B29B2682248A120001013ABB02D0FB
:101C20008C9A01D08C9C000000000050E66E04EC01
:101C30007AF0E5520000C950006E00008C8C8C8A4E
:101C4000030EE66E0AECFEF0E55212002C88070146
:101C50001081108D10990101E5A502D007011089AE
:101C60000701129712002C9807011091109D1099EE
:101C70001287120011EC7AF0F00EC616C680C68AE2
:101C80001200800EE66EE66A010EE66EAFECFBF027
:101C900065ECF4F03AEF0EF0138213800601109118
:101CA00002011E0E406F1200139020A213801392A7
:101CB00020B213821200C0ECF4F0D8ECF2F0B9ECD0
:101CC000EFF0DF6E000EDF94DF96DF98DF9ADF9C87
:101CD000DF9E0A0E006EFE0EDB5009E1030EDF5C94
:101CE00002E2050E006EDF5043E1010E40D0FE0E11
:101CF000DB50030804E1DF5002E1010E006EFE0E2E
:101D0000DB5004080EE1DF0402E1320E006E020E29
:101D1000DF5C02E15A0E006E030EDF5C02E1640E2E
:101D2000006EFE0EDB50050810E1320E006EDF047F
:101D300002E1640E006E020EDF5C02E17D0E006EB9
:101D4000030EDF5C02E1FA0E006EFE0EDB0403E020
:101D50006DECEDF00DE1DF5002E1010E006EDF04ED
:101D600002E1050E006E030EDF5C02E1190E006E4B
:101D7000E552B3EFE5F0AEECE5F0F00E07010F171A
:101D8000FE0EDB50320F63ECE6F007010F1384EC1C
:101D90005EF0B3EFE5F007509CECF2F081ECF0F070
:101DA000050DF350006E21ECE9F0EF50200B02E03E
:101DB000050E00260701BB51005C07E000C0BBF721
:101DC0000050E66EAE0EC3ECE5F01200139A20B29E
:101DD000138A6ADFB9EC4BF0E6EC1CF02050020BE2
:101DE00006E00101D3510C5C02E01B8C12001BAC1D
:101DF00002D038EC0AF01200AEECE5F02050020BF5
:101E000006E03FECBAF0000902E120922ED020500B
:101E1000020B08E052ECE7F005E0CFECB9F0D7ECAC
:101E2000B9F020822050020B06E085ECE9F003E0D7
:101E3000139E3E93CE99FE0EDB5004E120B2048047
:101E40003BEC0AF0C3DF050E0C5C08E12050020BEE
:101E500005E00201B593B59175EC38F0E0ECB9F00E
:101E6000FE0EDB5002E102011783B3EFE5F00FEC49
:101E7000F0F0D4C1DFFFB5ECE8F002E1040EDF269C
:101E80002FECE7F003E00D0EDF5C11E32FECE7F041
:101E90000CE1B5ECE8F003E0140ED45D08E30A0EA3
:101EA0002E5D03E10A0ED45D02E3000E01D0010EA7
:101EB000E552B3EFE5F0700EE66E2B0EE66E010E06
:101EC000E66EE66AE8EFE5F07E0E0A6E0C0EE66E50
:101ED000EE0EE66E020E07EFF2F0F00E8C16A0EC9E
:101EE000F4F011E22FECE7F00EE02B50010B0BE1C8
:101EF000320E3EECE6F0A0ECF4F005E22B807B0E17
:101F00007BECE6F001D812000101320E4B6F63EC5E
:101F1000E9F083EF28F00701875106E14C0EF7EC5A
:101F2000E7F00501141501E1000C010C2D9E2D9C1C
:101F300075EC38F00AEFB7F007011D891D972FECFB
:101F4000E7F009E001012E0506E16251400B03E1D3
:101F500007011D991D871200AEECE5F0D7ECEEF0FD
:101F600007E12C50010B04E101018D51200B09E127
:101F700055C258F254C257F253C256F2A8ECEDF0D3
:101F800009D0FE0EDB5006E058C255F257C254F29B
:101F900056C253F2198C04802CA002D004902C90CD
:101FA000A5EC55F0320E096EB3EFE5F0006A0101C1
:101FB0003C51060802E2DDC700F000AE02D0070186
:101FC0001CD02BA002D007013ED00701DF5106E153
:101FD0000050240825E3E05140E022D0DF050FE166
:101FE0000050290803E3E051010802E2020EDF6F0E
:101FF000230E005C32E2E05130E1DF6B2ED0020EA6
:10200000DF5D10E10050310803E3E051020802E215
:10201000030EDF6F280E005C20E2020EE05D1DE281
:10202000010E1AD0030EDF5D10E10050360803E305
:10203000E051030802E2040EDF6F300E005C0DE297
:10204000030EE05D0AE2020E07D0350E005C05E2E9
:10205000040EE05D02E2030EDF6F070E1315006E43
:10206000F80E1317DF0501E11385020EDF5D01E1B4
:102070001383030EDF5D02E113851383040EDF5D1E
:1020800001E11381070E1315005C08E0050EA4ECB6
:10209000ECF02D9069EC5EF0F00E8C161200AEECB8
:1020A000E5F021B814D0FE0EDB50CFECF1F0016E5C
:1020B000FE0EDB50040FCFECF1F0026EFF0E015C60
:1020C00008E1FF0E025C05E1199A18B8198A000EA2
:1020D00009D00150006E18A802D00250006EC0EC6A
:1020E0009BF0010EB3EFE5F00301916B926B936BE4
:1020F000946B91C38DF392C38EF393C38FF394C308
:1021000090F3030E016EFF0E015C32E0056A030ED0
:10211000026EFF0E025C22E00250EA6A890FE96E4D
:10212000030EEA22EF504C6E4D6A0150EA6A850FA9
:10213000E96E030EEA22EF50C3ECE6F0D9ECEBF0C7
:10214000EF504BECF2F005504BECF2F0D9ECEBF029
:102150000FC0EFFF10C005F00206DBD70150EA6A9E
:102160008D0FE96E030EEA2205C0EFFF0106CBD703
:10217000120000AE04D0006C01010E0E146F3DEC95
:10218000EAF0010115510AE114C115F1100E146FA6
:10219000165104E115C116F1100E156F130E186FCC
:1021A0001200AAECF3F0075045ECECF0EFCFDFFFA4
:1021B000010EC3C1DBFF020EC4C1DBFF01017AB710
:1021C00038D0075006E0010EC8C1DBFF020EC9C1BE
:1021D000DBFFDFCFE6FF19EC04F0E552E66EF8EC2A
:1021E000EAF0BFECE6F00B0EDF2463ECE6F0E66EFF
:1021F0000750EA6AE70FE96E020EEA22BFECE6F04A
:10220000DF5011E1FFECEAF0010EEF6EDB0404E1B8
:10221000500E28ECE9F007E2F8ECEAF0020EEF6E5F
:10222000FFECEAF0EF6AF8ECEAF0EF50E66E41EC12
:10223000EAF0030EE15C02E2E16AE552E16EB3EF1F
:10224000E5F013ECF0F0C3C1DFFF010EC4C1DBFF0A
:1022500001017AB71ED0075005E0C8C1DFFF010EAB
:10226000C9C1DBFF075045ECECF0EF5012E1FFEC89
:10227000EAF0EF5007E0DF040BE1500EE4ECE5F08C
:1022800008E206D0DF0405E1010EDB504F0801E251
:1022900088DF020EE15C02E2E16AE552E16EB3EF33
:1022A000E5F0030E0C5C03E1FDECECF001E0000C4A
:1022B000010C030E0C5C05E110ECEAF003E0B6053E
:1022C00001E0000C010C030E0C5C03E110ECEAF0E1
:1022D00001E0000C010C030E0C5C08E10101B65199
:1022E00005E1CE51040B01E0020C010C000C030EC1
:1022F0000C5C0BE110ECEAF003E13F51010B06E14D
:10230000B60503E13F51020B01E1000C010C06018F
:10231000F25107E0030E0C5C04E10101B651000824
:1023200001E3000C010C030E0C5C05E10101B60594
:1023300003E0B65101E0000C010C030E0C5C06E159
:1023400010ECEAF004E0030EB65D01E0000C010CB5
:1023500001013F51080B03E0030E0C5C09E03F5103
:10236000040B05E00C0404E0020E0C5C01E0000C20
:10237000010CCEEC0CF0BAECE6F0EF9CBFECEBF00D
:1023800007E0BAECE6F0EF8C0701E26B58C1D5FA32
:10239000120068ECE6F003E0C3ECEBF001E1000CA6
:1023A000010C0C5004E10A01DA51040B01E1000CAC
:1023B000010C0C5003E1BDECEFF001E1000C010C4D
:1023C00075ECEDF00CE089ECE9F009E00301D8517F
:1023D0003DECF5F0F9ECE9F0E80EDFECE5F0120089
:1023E00040ECF5F00C5005E1BDECEFF002E0020E20
:1023F000DF6E01017AB9DF84DFCFE6FFEB0EC3ECBD
:10240000E5F00C5004E10A01DAB7DA95D9DFE552BC
:10241000B3EFE5F0030E0C5C11E10101CF51040BA9
:1024200005E0B6050CE0020EB65D09E0CE51040BE6
:1024300005E0B65104E0030EB65D01E0000C010CAE
:102440000C5003E1C7ECEBF004E1C1ECEFF001E16B
:10245000000C010C72ECEAF001E0040C14ECEAF060
:1024600001E0080C040E0C5C01E11B0C0C500AE0AE
:10247000030E0C5C06E10101B65104E0030EB65DEB
:1024800001E0030C010C72ECEAF001E00A0C14EC20
:10249000EAF001E0380C040E0C5C01E1640C0C5015
:1024A00001E0500C380CEFDFE66ED4DFE66ED60E9E
:1024B000E66E0A0ED5EFE5F04BEC56F0190E01244E
:1024C0000A01D880D75503E2190E0124D76F79ECA1
:1024D000EDF0D75D03E279ECEDF0D76FD46B348883
:1024E000AAEFF0F052ECE7F00DE172ECEAF00AE14D
:1024F00014ECEAF007E1BFECEBF004E1F2ECE8F0F9
:1025000001E1000C010C896A700E8A6E030E8B6E5D
:10251000700E8C6E320E8D6E040E8E6E8F6A800E73
:10252000906E916A92688F0E936E900E946E956A7B
:102530009D0E966E7B0E976E070E986E300E996EFE
:102540009A6812002098268A0101B29B02012B5141
:1025500014E00701EF9BEF9B33BCEF8BDDEC09F040
:1025600002012B6BF1C600F00C5002E0F3C600F044
:102570000050E66EE20EC3ECE5F026821200F1ECAC
:10258000F4F0DCECEEF025ECF5F025ECF5F025ECC4
:10259000F5F0C09EF00E8C16020E0F0B05E0D890E1
:1025A00010320F32E806FBE180ECE8F0030EDCECC1
:1025B000F2F0FDE14A500F5E4B50105A2BAA0DD09D
:1025C0000A0E3E6E3F6ADBC743F0DCC744F067EC9F
:1025D000F9F03C500F263D5010227DEC94F0A9EC10
:1025E00004F0300F0101196FD0ECE9F001011A6F0E
:1025F0003A500F6E106AA0EC04F0300F01011B6F0F
:10260000300E3A241C6F300E195D02E1200E196F56
:102610001B8F410E1E6F1200AEECE5F0050101515B
:10262000EA6A000FE96E080EAFECF3F0012B0151DE
:1026300039ECE6F002E6E1ECEEF001E3016B002B91
:10264000B3EFE5F0020E68EFE9F0B4EFF3F0949227
:102650008B90949040EFE9F08B92B4ECF3F082B061
:10266000FF0C000CEFDFEEDF82A2FE0C000C070176
:10267000080EC96F8B92B4ECF3F082B207D0F2DF90
:10268000000904E0FE0EF36EF46812000701C89F13
:10269000C847C89182B0C881C907EDE1C851D8EFD9
:1026A000E9F0D9CFE6FFE1CFD9FF0701080EC96FE6
:1026B000FE0EDBCFC8F78B9282B206D0D3DF0009C3
:1026C00002E0FF0E17D011D0C837D8A006D09492E0
:1026D0009480B8DF9482B6DF06D094928B90949069
:1026E000B1DF9482AFDF0701C9070701C951E4E1F7
:1026F000000E00D0E552E7CFD9FF12008B929492E2
:102700008B90949040ECE9F0948022EF13F08B9042
:10271000949022EF13F048ECE7F05BEC0FF00EEC36
:102720005FF064EC0FF019EC5FF04BEF9CF0E3EC22
:1027300018F0909C908E38EC2CF00101796B2DEC08
:102740000BF072EC09F0020EE66EF50E4BECECF0BD
:1027500044EC0AF00701010E066F076B086B096B6A
:102760000A6B0B6B0C6B0D6BF00E0E170F6B106B77
:10277000116B126B600E136F146B156B166B186B6D
:1027800018C717F71B6B1C6B206B1D6B1E6B1F6B29
:1027900084EC5EF00601526B52C650F6547125EC83
:1027A00051F08A9831EC99F071EC98F00601556B74
:1027B00055C654F60B6A1200F29E9D0E966E8D9CC5
:1027C000FCD7EAEC26F00701F10504E14C0E005CB1
:1027D00006E203D05A0E005C02E2A9DFEDDF000C36
:1027E00044EC0AF0EAEC18F03488B9EF4BF08B8A2D
:1027F000010162B18B9AC69A8B96F00E8C14070970
:102800008C6E81EC5EF08A9AE3EC08F08B86000017
:10281000000000008B960000EDEC08F000008A8AB2
:10282000C68A12001A50800B01E0010E45ECECF054
:10283000EF50090801E2000C010CF00E8C16050E99
:102840008C12C08E7EECF0F0C3CF4AF0C4CF4BF0B8
:10285000BDECE8F0BDECE8F0C3CF4CF0C4CF4DF0D8
:10286000060ED8904D324C32E804FBE14A504C241D
:102870000701DB6F4B504D20DC6FC09EF00E8C16B5
:1028800012008F0EB1ECE6F0030E0002F3CF0CF253
:102890000050200801E3000C010C0101E251040B7F
:1028A0002EE0EEECE8F02BE02150200B28E0345035
:1028B000400B25E1E6DF000922E00A0E3EECE6F0DF
:1028C000E0DF00091CE0FA0E3EECE6F0DADF00097A
:1028D00016E0090EDBECE5F012AE04D0129EE6EC39
:1028E000EEF008D012BC06D0128CEBECEEF0020138
:1028F000020EBD6F40EC27F053EC27F0258A120042
:10290000F00E8C16070E8C12C08E7EECF0F0C3CF4A
:102910004CF0C4CF4DF0B5ECEFF0B5ECEFF04C500F
:10292000C3244A6E4D50C4204B6E4A50C3240F6ED0
:102930004B50C420106E110E54ECF2F0C09EF00EFD
:102940008C16010161514C6E4D6A3B0E4C26010EF6
:102950004D220F504C5C4A6E10504D584B6E4AC081
:10296000DDF70701DD5154080BE2DD5139ECE6F0EB
:1029700002E6FCECE7F004E22FECE7F001E0010CEA
:10298000000CC08E870EB1ECE6F0DCECEEF0D890D7
:102990000F361036D8900F361036A9ECECF0C09EEA
:1029A000D9C74AF0DAC74BF0030EDCECF2F0FDE1D8
:1029B0004A500701D95F4B50DA5B0F50D9271050AE
:1029C000DA231200860E010166254C6E4D6A000E58
:1029D0004D22D9C74EF0DAC74FF0600E436E446AFD
:1029E0004EC03EF04FC03FF0B8ECFDF03EC04EF0A0
:1029F0003FC04FF04E504C5C4A6E4F504D584B6E9E
:102A00004A50006E120030ECF0F00EE1F00E0201C0
:102A1000131507010D6F0F0E02011315006E00381C
:102A2000F00B07010C6F0DD0F00E02011415070119
:102A3000096F0F0E02011415006E0038F00B07012C
:102A4000086FB3EFE5F0C00E016E2FECE7F002E087
:102A5000B00E016E2CA802D0D00E016E01010F51F4
:102A6000012644EF4DF0AEECE5F06DECEDF002E147
:102A7000FE0EDB060750060D12ECE6F0140E4A2699
:102A80000A0E4B22FE0EDB50B8ECF3F0B3EFE5F08C
:102A90000FECF0F0A6EC0DF0050E0C5C06E1070162
:102AA000E26B0A01D56BDA931CD04FECE8F0EFCF64
:102AB000E2F70C50DF6ED5CA00F07DECEDF0DF5090
:102AC000D1ECF0F04FECF2F048ECE8F076ECEAF004
:102AD0000CE19A0E0B5C09E30B509E0806E300C064
:102AE000D5FAE66A88EC91F003D0DFCFE6FFBBDFD2
:102AF000E552075003E0D5CAB2F20BD052ECE7F032
:102B000008E00A01D76B060150850A01DA81C0ECA2
:102B10001EF0159C0701E25101E0158CC30E060161
:102B200050170A01DAA102D0140E01D0280E0601B6
:102B300050130A01DAA304D0D8CAE7F7D9CAE8F7D4
:102B400086EC1EF00C50A5ECE6F0EFCFEFF7B0EC02
:102B500025F0010EE66EE66A43ECE7F04FEC96F0E6
:102B60003EEC2CF0E2EC09F0E552B3EFE5F07DEC41
:102B7000EDF04FECF2F00C50D1ECF0F048EFE8F053
:102B80000C50A5ECE6F020ECEDF0050E0C5C0CE032
:102B90000A01DAA306D0E7C7D8FAE8C7D9FA86EC63
:102BA0001EF0E5DFBDECF3F012000FECF0F0DF6A91
:102BB000080EDF5C05E2EFECE6F0EF68DF2AF8D7FD
:102BC000E552B3EFE5F00FECF0F0DF6A080EDF5CE2
:102BD0000CE2EFECE6F0EFCF4AF0FE0EDB504A5C81
:102BE00002E1010E03D0DF2AF1D7000EE552B3EF68
:102BF000E5F00FECF0F00301D95104E0DB2B030EFC
:102C0000D95D17E34FECE6F0DEDFE552000911E194
:102C1000DF6A080EDF5C0DE2EFECE6F0EF50FF0834
:102C200006E1EFECE6F0FE0EDBCFEFFF02D0DF2A8D
:102C3000F0D7E552B3EFE5F00FECF0F0DF6A080EE5
:102C4000DF5C0BE2EFECE6F0EF50FF0804E0EFECA6
:102C5000E6F0EF5003D0DF2AF2D7FF0EE552B3EFD4
:102C6000E5F013ECF0F0DF6A080EDF5C10E2EFEC49
:102C7000E6F0010EEFCFDBFFDB50FF0806E0EFECE4
:102C8000E6F0EF68010EDB5003D0DF2AEDD7000E2F
:102C900070ECEBF002E2E16AE552E16E4A50B3EF0C
:102CA000E5F00FECF0F0318A69ECF4F08AECF2F028
:102CB0008AECF2F0DF6E319ADF50E552B3EFE5F0C7
:102CC0000FECF0F007018B6B8C6B2EA802D0010E7D
:102CD0002AD00C0EF7ECE7F0DF6E07018B2B000E0D
:102CE0008C23DF5008E0FF0EDF5C05E0580E8B5DA3
:102CF000020E8C59EEE38B518D5D8C518E5904E29E
:102D00008BC78DF78CC78EF7580E8B5D020E8C59D2
:102D100009E301018E5103E15A0E7BECE6F02E88A7
:102D2000000E01D0010EE552B3EFE5F0AEECE5F098
:102D3000AFECF0F0B3EFE5F00DECF2F003E2C5EC30
:102D4000EFF004D0FE0EDB50F60F410FB3EFE5F0CD
:102D5000C9ECEFF004E001013851E82402D0010190
:102D60003851E66EC40EC3EFE5F00FECF0F0FFEC67
:102D700026F0DF6E0F0EE66EDF5007E0030EDF5C1D
:102D800004E001018D51020B02E1000E01D0010EA1
:102D9000000905E00A0E01017D03F35001D0000E89
:102DA000E66ED90EDFECE5F0E552B3EFE5F067C172
:102DB0008FF2C3ECEBF002E168C18FF2006A02010E
:102DC0008FA302D0008807D08F51010B04E08F51F0
:102DD000800B01E0008C51ECECF002018FA502D0D9
:102DE0005F0E05D08FA702D04F0E01D05E0E006E91
:102DF0000050C6ECE5F002018FB508D08F51400BB2
:102E000002E04B0E01D04A0EC6ECE5F007010F9D23
:102E100002018F51020B05E08F51200B02E00701E8
:102E20000F8D06015295C9ECEFF005E08F51100BA4
:102E300002E006015285258A1200C3ECEBF003E1A3
:102E40008FC268F102D08FC267F1D7EF16F0AEECF7
:102E5000E5F03250080B35E10101E251100B31E190
:102E60000601BA6B020EBB6F328601018E5129E159
:102E7000450E28ECE6F02A0E28ECE6F0440E28EC8D
:102E8000E6F0530E28ECE6F0450E28ECE6F0300EA6
:102E9000072428ECE6F03B0E28ECE6F05D0E7BEC18
:102EA000E6F0FE0EDBCF2CF789C72DF788C72EF78B
:102EB00001013BA906D02A0EF5ECEEF02A0EF5EC46
:102EC000EEF0B3EFE5F00FECF0F02E50100B06E152
:102ED0003250100B03E00701F10502E1000E17D09C
:102EE00001013B51100B0AE03150200B07E1075064
:102EF00002E0400E01D0210EF5ECEEF007018A6BE6
:102F0000FE0EDBCF88F74FECE6F019D8E552E5521C
:102F1000B3EFE5F0AEECE5F00601B82B000EB923F7
:102F2000BA51B81909E1BB51B91906E14FECE6F005
:102F30008EDFE552010E01D0000EB3EFE5F0D9CFE0
:102F4000E6FFE1CFD9FF020EE1262E50100B03E180
:102F50000701F10502E1000E9AD0FE0EDBCF89F7E2
:102F6000010101013B51100B19E03150200B16E11A
:102F7000FE0EDB380F0BE66EDFDEE552E66ED6DEC8
:102F8000E552FE0EDB500F0BE66ED6DEE552E66E26
:102F9000CDDEE5522E0EE66EC9DEE552075027E182
:102FA0000601B86BB96B84B007D0E66AB3DFE552AF
:102FB000000901E001D0F7D78C9A0000FE0EDBCFAC
:102FC000E6FF04EC7AF0E5520000C950DF6E000025
:102FD0008C8A0601B86BB96B84A008D0010EE66E2E
:102FE00099DFE552000901E001D0F6D731D00101A7
:102FF00001013A51080B05E101010101E251100BF9
:1030000027E00601B86BB96B86B008D0020EE66EF9
:1030100081DFE552000901E001D0F6D78C9C000069
:10302000FE0EDBCFE6FF04EC7AF0E5520000C9505B
:10303000DF6E00008C8C0601B86BB96B86A008D0DF
:10304000030EE66E67DFE552000901E001D0F6D716
:1030500007018A5103E107018A2B14D007018A0571
:1030600011E10701881DDF5C0AE0075003E02550ED
:10307000100B05E0040E0724E66EE9DEE5520701B9
:10308000020E8A6F010EDFCFDBFFDF5000D04A6EE9
:10309000020EE15C02E2E16AE552E16E4A50E5525D
:1030A000E7CFD9FF120034ECF0F0B3EFE5F034ECE9
:1030B000F0F0FC0E58ECF2F0B3EFE5F034ECF0F089
:1030C000FC0E58ECF2F0FB0E58ECF2F0B3EFE5F02A
:1030D0001AECF0F001013EA904D0010E076E69EC74
:1030E000F4F0076A69ECF4F022EFF0F01AECF0F07B
:1030F00001013EA906D0010E076E4BECF0F0C2ECC8
:10310000F3F0076A4BECF0F0C2ECF3F022EFF0F0D2
:103110001AECF0F001013EA90BD0010E076EC5ECD0
:10312000F4F03EECE7F0FA0EDBCFE6FF08DFE55205
:10313000076AC5ECF4F03EECE7F0FA0E58ECF2F05A
:1031400022EFF0F0AEECE5F069ECF4F0D7C1E6FF69
:1031500015ECE7F0D8C1E6FF15ECE7F00FC0E6FF8D
:1031600015ECE7F010C0E6FF15ECE7F0B3EFE5F083
:10317000E0ECF4F001013EA902D0010E076EF00E62
:1031800047ECF2F022EFF0F0E0ECF4F001013EA9A0
:1031900002D0010E076EF10E47ECF2F022EFF0F0D4
:1031A000D9CFE6FFE1CFD9FFFE0EDBCFE6FF04EC7F
:1031B0007AF0E55200008C8E000000008C9EE552F3
:1031C000E7CFD9FF12002BB203D0740EFFECE7F06B
:1031D0002B8212002BA203D0760EFFECE7F02B928D
:1031E00012002BB203D0750EFFECE7F02B82120019
:1031F0002BA203D0770EFFECE7F02B921200AEEC7F
:10320000E5F032B206D0790EC6ECE5F0FE0EDBCF6B
:103210002CF2B3EFE5F0AEECE5F002015ABF07D0B7
:1032200032ECE6F05951EE265A51ED2208D0FF0E4D
:1032300059154A6E7F0E5A154B6E0AECF3F0FC0ED0
:10324000DBCFE6FF06ECEBF04A6E4B6A4ABE4B68FA
:103250000A0E07ECE9F00AECF3F0FB0EDB5069E034
:1032600001010B6B0C6B07502DE1FF0E0A01DF5DB6
:1032700029E0030EDE5D03E10101CE0E21D0050E33
:10328000DE5D02E1320E14D0020EDE5D03E10101CB
:103290009C0E16D0060EDE5D02E1640E09D0DE053E
:1032A00003E101016A0E0CD0070EDE5D05E1960E0A
:1032B00001010B6F0C6B06D0DE5104E10101380EE9
:1032C0000B6F0C69FB0EDB0416E174ECEBF006E30C
:1032D0005CECF2F0EE26E451ED2205D05CECF2F06D
:1032E000EE5EE451ED5A32ECE6F001010B51EE26B0
:1032F0000C51ED2215D074ECEBF006E35CECF2F02F
:10330000EE5EE451ED5A05D05CECF2F0EE26E451AD
:10331000ED2232ECE6F001010B51EE5E0C51ED5A5C
:10332000F7ECF4F0FD0EDBCFEEFFFE0EDBCFEDFF92
:1033300006D0FD0EDBCFB4F6FE0EDBCFB5F64FECBC
:10334000E6F0F9ECE8F044ECF5F0B3EFE5F00FEC63
:10335000F0F0140EDF6E01017AA302D0230EDF6EAF
:103360007AA102D00A0EDF6EDF50E552B3EFE5F02E
:103370000A0E036E0C5002E1EADF036E0050320DBC
:1033800012ECE6F0010E0F0B03E0E0ECF2F0FDE1D1
:1033900003500A0D56ECE8F001010F50D75D1050B4
:1033A000D8590BE2D7510F5C02015B6F0101D85174
:1033B000105802015C6FAEECECF0120004B007D0C4
:1033C00047ECEAF0010199ECF1F0110E03D0FDECAD
:1033D000F4F0100EC6EFE5F0B0C6B4F6B1C6B5F61F
:1033E00012ECF2F0CFBD06D00F500601B45F1050C2
:1033F000B55B05D00F500601B4271050B523B5C6F4
:10340000E6FFB4C6E6FF44ECF5F0056A0101CFAD76
:1034100002D0060E05266A0E052469EFF1F0FFECD6
:1034200026F0056E055003E1C7ECEBF003E1C1ECBB
:10343000EFF002E0060E05266BEC11F0006E005076
:1034400002E00050056E8EECF1F003E151C101F095
:103450000ED09FEC0BF0000903E087C101F007D00C
:10346000050E005C02E1016A02D058C101F0040EB1
:1034700005243BECEBF06DECF1F0030E005C11E188
:103480000101B6050EE1C8ECE7F0CFB505D0980E06
:10349000D7273A0ED82305D0980ED880D7573A0EA2
:1034A000D857ADECEFF00CE0000405E10101B40EDB
:1034B000D76F460E04D001017C0ED76F2E0ED86F49
:1034C000E66A0150E66ED7C1E6FFD8C1E6FFF6EC2A
:1034D000E6F06A0E052469EFF1F002015B6B5C6BAC
:1034E00021AC02D00101E78997EC04F00101E799D2
:1034F0000C5011E12C514DECEAF03ADF0101CFBD47
:1035000006D047ECEAF099ECF1F0130E69D0FDEC2F
:10351000F4F0120E65D078ECEBF00CE00101F20E45
:10352000D76F030ED86F24DF04900101CEA50CD015
:1035300004800AD009ECE8F009E0C8ECE7F018DFF5
:1035400004900101CFB5048039DF4DD0DC0E0F6E41
:10355000050E106ED6ECF1F0780E4A1806E14B50CD
:1035600004E1400E0F26060E1022050E0C5C0BE146
:10357000010EE66EE66A980EE66E3A0EE66E4BDED9
:1035800065ECF4F02FD0040E0C5C11E147ECEAF08E
:10359000E66E3A0EE66EF6ECE6F00101D1A723D016
:1035A000D151020B02E0180E1BD0190E19D00C04D9
:1035B00004E06BEC11F001080CE147ECEAF00F2499
:1035C0004A6E3A0E102099ECF4F0F6ECE6F0110E8B
:1035D00007D0FAECEEF080ECE8F066ECF0F0100EBC
:1035E000E66E71DCE552075004E05BC263F25CC238
:1035F00064F2120072DF075006E152ECE7F002E0DD
:10360000ECEF19F00CDF1200AEECE5F00701B4515D
:10361000320D6DECF1F074ECEBF011E1FE0EDB50CD
:103620000EE10C5004E101012C514DECEAF078EC74
:10363000EBF005E00101F20ED76F030ED86FB3EF88
:10364000E5F00FECF0F0075004E02550100B01E11D
:10365000BAD1CEEC0CF0D6CAB3F707011E0EB46F88
:103660000C5005E110ECE9F03FC0B4F711D0030EA7
:103670000C5C0EE1FDECECF003E10701140E07D049
:1036800009ECE8F005E0260E61ECF2F00701B46FFA
:10369000D7CA00F00701EFAF10D0190E006E0A0173
:1036A000D75D06E281ECEDF017ECF2F0005E05D09C
:1036B000190ED75D17ECF2F00026190E005C05E339
:1036C000190E005C0701B42705D0190ED8800054EC
:1036D0000701B45F040E006E0C5005E138DE17ECF4
:1036E000F2F0006E09D00C0406E0020E0C5C03E060
:1036F000040E0C5C01E1006A0701B351FE0BE842C5
:103700000024056EDF6A0550B45D13E2DF2AB35171
:10371000FE0BE842B425016E01500024FE0BE84286
:10372000B46F0050015C02E20050016E0050015C79
:10373000B36FB3C7B2F7040E0C5C03E1B351E824D6
:10374000B26F050E0C5C05E1320EB36F1F0EB46F45
:10375000B269F7ECF4F0EECFB5F7EDCFB6F7040EA3
:103760000C5C20E2DFCFE6FF4FDFE552020E0C5C7F
:1037700008E06BEC11F0020804E020EC12F0000904
:1037800009E00101D7510701B5270101D85107010F
:10379000B62308D00101D7510701B55F0101D85107
:1037A0000701B65B89ECE9F001E109D1BAECE6F07A
:1037B000EF960701B251A1ECE6F004E24A500A0884
:1037C000000E4B5403E3BAECE6F0EF863FECF4F066
:1037D000080B02E0B60E01D0B00E006EF2ECE8F07D
:1037E00002E0B30E006E0701B751005C09E1BD5164
:1037F000B51906E1BE51B61903E1B851B25D1AE040
:1038000000C0B7F7B5C7BDF7B6C7BEF7B2C7B8F7C0
:10381000B5C7D7F1B6C7D8F1B251320D2DECE6F0ED
:10382000050E0C5C04E1C80E0F6E320E106E0050D7
:10383000EDECE7F089ECE9F001E1C1D0BAECE6F09B
:10384000EF9ABAECE6F0EF8E14ECEAF018E107011B
:10385000B351020814E301013FAB04D0BAECE6F027
:10386000EF8A0DD00701B451A1ECE6F004E24A5012
:103870001E08000E4B5403E3BAECE6F0EF9EE1ECB9
:1038800023F00C5003E0030E0C5C2EE10701EF5116
:10389000800B03E174ECEBF027E1DF5025E1E2DB84
:1038A000AEECECF00A01D751190808E2190ED75D09
:1038B0001BECE8F00101D7274B50D82374ECEBF058
:1038C00008E281ECEDF01BECE8F00101D75F4B5012
:1038D000D85B01010A0ED803F3CFD8F1D703F3CF99
:1038E000D7F1F450D82704D0DFCFE6FF8DDEE552C4
:1038F0000701B351320D2DECE6F014ECEAF007E0CD
:1039000001012C514DECEAF0960E0F6E106AD3ECCB
:1039100009F0030802E10101D88F3FECF4F0200B1D
:1039200002E0B70E01D0B10E006E0701B951005C84
:1039300010E1BF510101D7190CE10701C05101018C
:10394000D81907E10701C1510F1802E1C25110183F
:103950000DE000C0B9F7D7C1BFF7D8C1C0F70FC09D
:10396000C1F710C0C2F70050EDECE7F014ECEAF03C
:1039700024E089ECE9F021E00701C3510101D719E6
:1039800009E10701C4510101D81904E10701BA5145
:10399000B35D13E0D7C1C3F7D8C1C4F7B3C7BAF753
:1039A0000701B351320D2DECE6F0B20EEDECE7F06D
:1039B000100EE66E9FEC17F0E552E0EC11F0CBEC48
:1039C0000EF081EC68F0E552B3EFE5F08EECF1F02B
:1039D00001E1120089ECE9F048E0040E005C05E327
:1039E000B4C6D7F1B5C6D8F118D0030E005C08E113
:1039F0000101B60505E1B5C7D7F1B6C7D8F10DD0BD
:103A0000DC0E0F6E050E106EADECEFF004E0400E14
:103A10000F6E060E106E5AEC0AF0F00E0F6E0A0EC4
:103A2000106E000403E0020E005C0EE101018DA1A6
:103A300005D08C516E0D2DECE6F006D0375104E028
:103A4000C80E0F5E000E105A040E005C04E1700EEA
:103A50000F6E170E106E050E005C04E1C80E0F6E9F
:103A6000320E106ECB0EEDECE7F089ECE9F03EE0A3
:103A70000101DC0ED76F050ED86FF00E0F6E0A0E27
:103A8000106E030E005C0CE1B60509E19051400B8D
:103A900006E0C8ECE7F0900E0F6E010E106ED88FA6
:103AA000ADECEFF014E001018C516E0D2DECE6F061
:103AB000AEECECF0010E0F0B05E0D890D833D73305
:103AC000E806FBE1640E0101D727000ED823050E9E
:103AD0000C5C09E101010E0ED76F060ED86FC40E03
:103AE0000F6E090E106ECF0EEDECE7F01200530EC4
:103AF000006EE66A0050C7ECF3F0075003E15C0E7D
:103B0000C6ECE5F05B0EC6ECE5F0A70E016E026AAE
:103B100004ECEFF0C20EDFECE5F05D0EC6ECE5F074
:103B20009AEFECF001013EA905D0570EE66E68EC65
:103B300018F004D0570EE66E63EC17F0E552120051
:103B400013ECF0F068ECE6F02BE011ECE7F028E184
:103B50000701875125E101013E51800B03E1050E6C
:103B60000C5C1EE14C0EF7ECE7F0DF6E050E0C5C12
:103B700011E10101E39FDFA8E38F3EA90BD0010E05
:103B8000076E4C0EF7ECE7F045ECEBF0076A339864
:103B9000DBA8338801013EAF03D0010EDF1401D052
:103BA000000E70ECEBF002E2E16AE552E16E4A5081
:103BB000B3EFE5F001013E51800B06E068ECE6F062
:103BC00003E011ECE7F001E0000C010CF3DF000969
:103BD00002E0510E01D0500EC6EFE5F071C1E6FFD4
:103BE000D00EC3ECE5F056C1E6FFD10EC3ECE5F014
:103BF00072C1E6FFD30EC3ECE5F0E6EF1DF0010164
:103C00003EA905D0560EE66E68EC18F004D0560EAC
:103C1000E66E63EC17F0E552120001013A51100B09
:103C200002E0140E01D0050EE66EAC0EC3EFE5F017
:103C30002150400B06E00101E451040B02E1E48550
:103C400001D812000FECF0F057C1DFFFC3ECEBF02E
:103C500003E15BC1DFFF09D00101E551020B05E083
:103C60009951040B02E09AC1DFFF040EDF02F3500A
:103C7000E66EC70EC3ECE5F001019951080B03E0B5
:103C8000E451040B02E0000E01D0010E000902E035
:103C90006F0E01D06E0EC6ECE5F0E552B3EFE5F025
:103CA000020EE66EBC0EC7ECF3F07C0EC6ECE5F03F
:103CB000070EE66E6C0EC7ECF3F07D0EC6ECE5F079
:103CC000BC0E0F6E020E33ECF1F07E0EC6ECE5F08A
:103CD0006C0E0F6E070E33ECF1F07F0EC6ECE5F0C4
:103CE0009AECECF048C1E6FFC10EC3EFE5F0620EBE
:103CF000006E07010E9D01015AAD03D0002A070195
:103D00000E8D0050C6ECE5F0258A12000701E75140
:103D10000C0803E3E8510C0805E2E76B0C0EE86FB2
:103D20000A01DA931200016A0D0E015C07E01FEC34
:103D3000EAF002E001501200012AF6D7000C0C0E46
:103D4000016E015007E01FECEAF002E001501200A2
:103D50000106F7D7000C0701E56BE66BD7DFE7C775
:103D600001F00701E851D880015409E38AEC04F01E
:103D7000F3500701E513F450E613012AF2D71200BD
:103D8000016A72ECEAF00BE0B5ECF0F006E24A50A2
:103D90000508000E4B5401E2012A510E0DD014EC1F
:103DA000EAF012E0B5ECF0F006E24A501408000E1A
:103DB0004B5401E2012A530E01243BECEBF0F3CF0C
:103DC000E5F7F4CFE6F71200B5ECF0F016E24A5052
:103DD0004608000E4B5411E2F2ECE8F00EE1070148
:103DE000F80EE56FE669050E0C5C01E1C7D0E76BE4
:103DF0000C0EE86F0A01DA83C1D0006A0A01D751BC
:103E0000A1ECE6F006E24A500D08000E4B5401E228
:103E1000002AD751A1ECE6F006E24A501308000E42
:103E20004B5401E2002AD751180801E2002AD75169
:103E3000190801E2002AD751A1ECE6F006E24A5047
:103E40001F08000E4B5401E2002AD751A1ECE6F006
:103E500006E24A502508000E4B5401E2002AF2EC1B
:103E6000E8F007E0020E006E0101D1A302D0040EBB
:103E7000006E0C5003E0030E0C5C1CE1B5ECF0F09E
:103E800006E24A500508000E4B5401E2012A47ECB5
:103E9000F5F006E24A500A08000E4B5401E2012AEE
:103EA00047ECF5F022E24A501308000E4B541DE295
:103EB000012A1BD0B5ECF0F006E24A501E08000EB5
:103EC0004B5401E2012A47ECF5F006E24A5028087B
:103ED000000E4B5401E2012A47ECF5F006E24A508D
:103EE0003208000E4B5401E2012AD50E4D6EEF0E42
:103EF0004E6E010E4F6E0050506E516A526A030EA4
:103F0000D890503651365236E806FAE14D505024DA
:103F10004A6E4E5051204B6E4F5052204C6E015005
:103F2000536E546A556AD8905336543655364A50B3
:103F30005324F36E4B505420F46E4C505520A4EC97
:103F4000F0F00900F5CFE5F70A00F5CFE6F775ECDC
:103F5000EDF005E00701E587E689E59FE69B030EA6
:103F60000A01D45D02E0D45109E1DDDE0701E76F0B
:103F7000E6DE0701E86F0A01DA83C8DE0A01D4052C
:103F800014E10701E805056E0A0EE85D01E2050689
:103F9000CADE0701E76F0550D880E75502E205C089
:103FA000E7F7D9DE0A01DA831200020ED45D12E1CE
:103FB0000701E729056EE751020801E2052ABFDE85
:103FC0000701E86F0550E85D02E205C0E8F7C3DECF
:103FD0000A01DA8312001E0E006E0C5004E110EC90
:103FE000E9F03F500BD078ECEBF002E0140E06D075
:103FF00009ECE8F004E0260E61ECF2F0006E0A0134
:10400000D651FE0BE842056E1200170E48ECE6F0A2
:10401000050E0A01D803F350006E0101012B78EC64
:1040200097F00101200E1C6F1E8F12001A0E48EC33
:10403000E6F00A01D9513DECF5F028ECEDF01E8FC9
:10404000120065ECF2F0F9EC7FF02DEC2EF0300E62
:1040500001011C5D02E1200E1C6F1E8F016B700EB2
:104060006DEFE9F00C5003E101012C510BD0030E70
:104070000C5C11E1FDECECF002E1650E03D0B651F1
:1040800004E1960E0F6E106A12002A0E312563ECC1
:10409000E6F00F6E106A12009EDF0701EFAF15D039
:1040A00072ECF1F0DFDF0A01D751190807E2190EAF
:1040B000D75D1BECE8F00F264B501022190ED75D90
:1040C00017E281ECEDF01DEFF2F00A01D75119086B
:1040D00003E2190ED75D0026190ED75D03E281ECCD
:1040E000EDF0005E72ECF1F0190ED75D01E1BADF80
:1040F0001200F2ECE8F00AE00101D1930A01D75175
:10410000190802E20101D1830A01D76B1200F2EC17
:10411000E8F009E00A0EDBECE5F00101D1A32BD0B9
:104120000B0EDBEFE5F0AB0E48ECE6F0B5DF75EC1F
:10413000EDF00BE00101410E196F500E1A6F0301F3
:10414000D851106AE8307F0B0F6E28ECEDF075EC5B
:10415000EDF009E00101460E1B6F2C51E82403012C
:10416000D85D07E103D074ECEBF003E101012A0E06
:104170001C6F01011E8F1200AEECE5F0070EE12668
:104180002AEC12F00A01D65D04E22AEC12F00A01D0
:10419000D66F43EC12F00A01D880D65504E243EC06
:1041A00012F00A01D66F72EC12F0000903E00A0166
:1041B000190ED76F10DF74ECEBF004E3190ED75D26
:1041C000002603D081ECEDF005260550005C03E3EA
:1041D0000550005E0AD0006AD40507E1DC51D75DC6
:1041E00004E2DCCAD7FADDCAD6FA00C0D8FAF3DE98
:1041F0000550002674ECEBF004E3190ED75D0026A1
:1042000009D081ECEDF0056E0550D880005402E233
:104210000550005EFAECF0F00BE24A505408000E34
:104220004B5406E2540E006EDCCAD7FADDCAD6FA49
:1042300000C0D9FA190ED75D03E3190ED75D03D07C
:10424000190ED880D7550701E36FE46BEFAF02D0AA
:104250000A0E01D0320EE403F3CFE4F7E303F3CF09
:10426000E3F7F450E427075002E0D7CA60F252ECBB
:10427000E7F004E0060150850A01DA81FE0EDB500A
:1042800014E02150800B11E10A01D45102E1D9DE82
:104290000AD0D40502E1B9DE06D0020ED45D02E1F7
:1042A000C5DE01D034DF960E096E3550040B13E1E4
:1042B0000A01DA51020B0FE052ECE7F00CE172EC6C
:1042C000EAF009E114ECEAF006E175ECEDF003E147
:1042D000F2ECE8F003E054DD359401D03CDDF9EC7C
:1042E0007FF0040E0C5C04E1010E09ECEFF0FDE13F
:1042F0000C500AE10E0ED8800F54010E105404E247
:104300000E0E0F6E010E106EFD0EDB5001E195D00A
:104310001950020B01E091D0050E0C5C01E18DD02B
:10432000BFECEBF001E089D0D5CADFFF026802C024
:10433000D5FA050EDB68060EDB68D950030FE96E6F
:10434000DACFEAFFEE68ED68016A050E015C5DE216
:10435000010E01C0E7FFE75204E0E846FE0BE70666
:10436000FCE10701E1154FE00750B1ECF4F001501A
:104370000F018BECE6F0EF50050DDE52F3CFDEFFC0
:10438000F4CFDDFFDD5289ECEAF01FE2010EDB50D5
:104390000F5C4C6E020EDB5010584D6E050EDBCFDD
:1043A0004EF0060EAFECEDF010E2010EDB500F5CAC
:1043B0004A6E020EDB5010584B6E050E4AC0DBFFF2
:1043C000060E4BC0DBFF0150026E89ECEAF01BE3E6
:1043D000E2ECEBF04C6E10503F584D6E030EDBCF0D
:1043E0004EF0040EAFECEDF00EE2E2ECEBF04A6EB4
:1043F00010503F584B6E030E4AC0DBFF040E4BC0FB
:10440000DBFF01C0D5FA012AA0D7FF0E0A01D55D56
:1044100007E1FF0E025C02E1D56B02D002C0D5FAC3
:10442000075002E0D5CAB2F2DF50D55D06E04FEC8E
:1044300096F057ECECF04AECEBF0B9EC4BF0070ED1
:10444000E15C02E2E16AE552E16EB3EFE5F0006A99
:10445000800E066E056E05500502F350015CF450A7
:104460000258D8B008D000C005F006420650051228
:1044700006BE09D0F0D705C000F00642065005126E
:1044800006BE01D0E8D700D01200AEECE5F02B84D8
:1044900023EC15F04BC102F02FECE7F004E08DECBB
:1044A00005F0940F026E00504C6E4D6A0250C3EC42
:1044B000E6F00F50016E10C002F0C9DF036AFFEC96
:1044C00026F0016E1D50040B2FE0010403E0020EE4
:1044D000015C2AE13550400B27E1FE0EDB5024E061
:1044E00010C202F0025020E0025039ECE6F002E681
:1044F000FCECE7F019E20250FE0BE842D8800054D1
:1045000013E20250E824005C0FE2FE0EDB0406E139
:10451000320E02010F27000E102305D0320E0201C9
:104520000F5F000E105B032A03500EE102010F6BB8
:10453000FAECF0F007E24A507108000E4B5402E228
:10454000710E006E00C010F22550020B06E12350E0
:10455000400B03E03250800B0AE0036A006A32AE7F
:1045600006D0000E0201116F126B0F6F106B03501B
:1045700007E10050E66EE66AC80EDFECE5F002D017
:10458000E5EC0BF0B3EFE5F0F9ECE9F0C20EDFEF8C
:10459000E5F0AEECE5F012ECF2F0F6DF1D8EFE0E6B
:1045A000DB5005E0075003E1680EC6ECE5F0B3EF21
:1045B000E5F00FECF0F037C1DFFF0101375108E003
:1045C0002150400B05E01C50020B02E0010EDF6E93
:1045D000FFEC26F0026E036ADF5006E0030E025C79
:1045E00003E0050E025C02E1010E036E8C0E006E0C
:1045F000035001E000683C0ECDECEFF0C50EDFEC9F
:10460000E5F0C60E016EDF50006E040E025C04E1A0
:10461000100E0026D80E016E035006E0006A040E4C
:10462000025C02E1100E006E0050E66E0150C3EC19
:10463000E5F0046A035001E0048E0450E66ECE0EED
:10464000C3ECE5F0E552B3EFE5F0B6ECEDF003E0D6
:104650000101375106E00201DF5105E10101375147
:1046600002E0E6EC1CF02B841200016AB5ECE8F0E5
:1046700001E1012A006A32900150DFECE6F0B3EC70
:10468000ECF0EF50800B06E00150DFECE6F0EF506D
:10469000006E3280E66A0050E66EDF0EDFEFE5F076
:1046A000AEECE5F0075014E1040E01012B03F350CA
:1046B000006EFE0EDB5002E0005001D0000EE66EF0
:1046C000C30EC3ECE5F00050E66EAD0EC3ECE5F0B2
:1046D000B3EFE5F0CBECF3F04D0E0A6E075003E0BC
:1046E000DE52800EDD6E010EDB5029ECE7F0FF0E8E
:1046F000005C14E0BC0EC6ECE5F0DF6ADF5039EC7C
:10470000E6F002E6FCECE7F009E2010EDB5026ECF5
:10471000F1F00050E4ECF2F0DF2AF0D70A6A020E62
:10472000E15C02E2E16AE552E16EB3EFE5F0AEEC86
:10473000E5F0016A080E015C10E2FE0EDB50012478
:1047400013ECEFF0026E100E025C040DF350006EDD
:104750000050E4ECF2F0012AEDD7B3EFE5F089EC7C
:10476000E9F00DE0AB0EC6ECE5F0D3EC09F0000982
:1047700002E1180E01D0080EE66ED9DFE5521200F4
:1047800089ECE9F00DE0CA0EC6ECE5F0A8EC0BF000
:10479000000902E0100E01D0000EE66EC8DFE552FF
:1047A00012001AECF0F00A0E0B5C08E125A803D009
:1047B000010E076ED4DF076AD2DF01D0E1DF22EFFE
:1047C000F0F0CEEC0CF0BAECE6F0EFCF4AF0BDEC36
:1047D000EDF0EF5000014A5C0EE03FECF4F0E66EC5
:1047E000BDECEDF0BFECE6F03FECF4F0800AE66ED5
:1047F000B40EC3ECE5F0120040ECF5F00701F10552
:104800004EE001013A51080B03E13A51200B02E05E
:10481000010EDF6E006A0701870507E1075002E11C
:10482000008203D0DF5001E0008602018FB30088D0
:1048300051ECECF0075002E1010E03D0DF5006E02E
:10484000040E0010E66ED0EC18F0E552010EDAEC22
:10485000E8F051ECECF0280EDAECE8F007018705FF
:104860001EE0020EC6ECE5F0020EC6ECE5F0006EAE
:10487000020E005C08E1075002E1510E0ED0DF503D
:104880000EE0570E0AD0FD0E005C09E0075002E171
:104890004E0E03D0DF5003E0540E7BECE6F0E55201
:1048A000B3EFE5F00701F10501E112002B92E3EC13
:1048B00018F0075006E0100EE66EA60EC3ECE5F009
:1048C0000AD0E66AA60EC3ECE5F0E66ABF0EC3ECBA
:1048D000E5F00DEC1EF0E668A70EC3ECE5F007501E
:1048E00013E1610EC6ECE5F0620EC6ECE5F077EC84
:1048F0001EF0650EA5ECF3F0660EDFECE5F0E66A5F
:10490000E66A660EDFECE5F0220EC6ECE5F0075035
:1049100003E1420EC6ECE5F021EC1BF0FFEC1DF0CC
:104920008DEC0CF0075002E145EC09F019D9C80EE6
:10493000E66EB50EC3ECE5F0700EC6ECE5F0020EC7
:10494000E66EE66AE00EDFECE5F0800EE66EE20E63
:10495000C3ECE5F0010165855F95B9EC11F031DF3D
:10496000280EE66E110EE66EE668A90E43ECF4F032
:10497000360EA5ECF3F0C00EE66EA40E43ECF4F098
:10498000075002E178D86CD881EC68F0A3DE0750BC
:1049900023E1D7EC16F0A8EC16F07EC1E6FFCC0EB2
:1049A000C3ECE5F050EC1EF03450040B02E0530E63
:1049B00001D0520EC6ECE5F022EC1EF0E1DE63EC15
:1049C000E9F0F7DD7FC1E6FFD60EC3ECE5F0B5EC0C
:1049D00016F0EEEC1DF049DE77EC1DF0010EE66EF0
:1049E000D8DDE55250ECEAF00601B66B090EB76F60
:1049F000B6DE01016251200B02E0640E01D0320EDE
:104A0000E66EF20EC3EFE5F001010A0E8E6F8BEC3D
:104A100013F0248A2A0E46ECF4F02E880701010ECA
:104A2000876F076A01013ABB076EA6EC0DF0E4DE62
:104A3000076A1200046A010162AF04D012BC04804C
:104A400012BE04823FB90484F2ECE8F001E004886D
:104A50000101E5B504860450E66EBA0E4BEFECF0AA
:104A6000075008E101018251E824E66EA10EC3EC73
:104A7000E5F0E0DF1200075018E101013429080DCC
:104A8000F350E66E050E345D02E2020E01D0010E17
:104A9000E66EAA0EDFECE5F001013E51400B02E0AC
:104AA000390E01D0380EC6ECE5F01200016A07019C
:104AB000EFB302D04EC101F04FC102F0EF51020B33
:104AC00008E00C5004E10601F051010802E350C176
:104AD00002F00150E66E64C1E6FF4AC1E6FFA80E8F
:104AE00043ECF4F00250E4ECF2F044C100F08BEC43
:104AF000F1F004E6F20E4A5C000E4B5802E2F20EB0
:104B0000006E0050E4ECF2F03C0E006E0701EFA1E5
:104B100002D03D0E006E0050C6ECE5F076C1E6FF17
:104B200075C1E6FF74C1E6FFA00E43ECF4F073C15B
:104B3000E6FFF30EC3ECE5F00701EFB110D0C9ECCE
:104B4000F4F004E060EC68F081EC68F01550100BB4
:104B500006E01550200B03E11598A4EC6AF0120052
:104B6000E0ECF4F0A3DF01013EA904D0010E076ED2
:104B70009DDF076A22EFF0F00FECF0F00C5003E13C
:104B8000010EE66E84D011ECE7F001E182D010EC6A
:104B9000EAF067E185EC04F02DECE6F0AA0E0101E5
:104BA0000F24D76F000E1020D86F3BBD0BD085ECC3
:104BB00004F06DECF1F0AA0E0101106AD7250F6E1A
:104BC000D8511022E1DC7D0EC6ECE5F0680EC6EC93
:104BD000E5F018ECEFF0D8DC7C0EC6ECE5F0690EE1
:104BE00011ECF3F001013B51400B400A01E0010ED2
:104BF0004A6ECF51040B040A01E0010E4A1805E089
:104C0000550E0F26000E102204D0550E0F5E000E1A
:104C1000105ADAECF1F001013B51400B400A01E07F
:104C2000010E4A6ECF51040B040A01E0010E4A182E
:104C300005E0AA0E0F5E000E105A04D0AA0E0F2631
:104C4000000E1022F9ECE9F044ECF5F07F0EC6EC12
:104C5000E5F0030EDF6E010199A113D0070EDF6EA0
:104C600010D01DECEFF090DC7C0EC6ECE5F0680E89
:104C700011ECF3F0DAECF1F0010EDF6E01017ABD18
:104C8000DF2A23ECF2F00501040E146FE66A81DCE2
:104C9000E552E552B3EFE5F00FECF0F0CEEC0CF09E
:104CA00002013F6B0601C26BC2C6C0F6339E0C50B8
:104CB00022E1F051010803E31450010B17E0010E4B
:104CC000016EF051020802E2030E016E040EF05D67
:104CD00002E1020E016E0150E7ECF2F0E00EDFECB3
:104CE000E5F0F1C6E6FFA4ECF2F003D0700EC6ECDE
:104CF000E5F036DF6AD0030E0C5C64E1BAECE6F056
:104D0000EF981450010B06E172ECEAF003E1D1ECEC
:104D1000EFF053E009ECE8F015E02E0E61ECF2F054
:104D2000016E020E026E2D0EDF6E010199A104D0FC
:104D3000040E026E4B0EDF6E14A016D00201010E9F
:104D40003F6F12D078ECEBF00FE0030E016E010E16
:104D5000026E1F0EDF6E01017AAD06D0040E016EE9
:104D6000030E026E3F0EDF6E04ECEFF0E00EDFECA0
:104D7000E5F0F3C6E6FFA4ECF2F072ECEAF003E033
:104D8000BAECE6F0EF880701200E7E6F3F0EDF5C85
:104D900002E1100E7E6F640EDF5C02E10A0E7E6F90
:104DA0004B0EDF5C02E10D0E7E6F2D0EDF5C02E12B
:104DB000160E7E6F7B6B7F6B03D0700EC6ECE5F03A
:104DC00000DD03D0700EC6ECE5F046EC4BF0E5528A
:104DD000B3EFE5F01C849F0EB1ECE6F01C9400509C
:104DE000B9ECEFF0005C02011E6F0050E00BE838F8
:104DF000E8401E27050E1E271EC200F0120020B23A
:104E000002D00C5012000101D35112000A0E47EFDC
:104E1000F2F014A205D0E3C20FF0E4C210F01200C9
:104E20009A0E95ECF2F00FC0E3F210C0E4F212001B
:104E30004C6B4D6B4E6B4F6B400E506FD89047379D
:104E400046374537443743374237413740374F3786
:104E50004E374D374C374B514F5D4A514E594951A2
:104E60004D5948514C5909E34B514F5F4A514E5BE4
:104E700049514D5B48514C5B472B502FE0D71200F6
:104E800012A409D00101CF9912BECF89D09712ACDC
:104E900009D0D08712000101CF9712BECF87D099D9
:104EA00012BCD08912001250040B04E00101CF5152
:104EB000100B09E11250040B04E10101CF51080B62
:104EC00002E1000E01D0010E0490E8B004801250FF
:104ED000040B04E00101D051080B09E11250040B4E
:104EE00004E10101D051100B02E1000E01D0010ECE
:104EF0000492E8B00482ABECEBF004E00201BC5198
:104F0000100B02E1000E01D0010E0494E8B00484FD
:104F100034AC09D0129E0101DCB1128E129CDCA3CC
:104F200008D0128C06D0129E04B0128E129C04B2CD
:104F3000128C0450040B040A01E0010E4A6E045066
:104F4000010B4A140496E8B0048607011D9904B6C3
:104F50001D891D9704A61D870101E8B906D0070128
:104F60000B9904A218D00B8916D007010B99045095
:104F7000020B06E0020E0201BD1502E007010B89DB
:104F800007010B910450020B06E0010E0201BD1552
:104F900002E007010B810450040B05E09FECE9F0EF
:104FA00002E0000E01D0010E4A6E0101DC51010B3E
:104FB0004A140498E8B0048807011B9904B81B89B7
:104FC0001B9704A81B8707990101DCA302D00701E6
:104FD00007890701109304B410830101E89104B616
:104FE000E881E89304B8E8831AEF25F00701109BE5
:104FF00012A4108BBBECEBF0A6ECE9F005E09FEC03
:10500000E9F002E0DAEC0CF0E6ECEEF0EBEFEEF0BB
:105010000FECF0F018ECF3F0200E26ECF1F000505D
:10502000026E0F0E26ECF1F001012E51005C19E129
:10503000250E025C16E1050EE0ECF1F00101CEA9AF
:1050400003D033ECE7F0286B050E0C5C07E1030E90
:10505000E66E100EDF24E66EACECF2F00A6A010E8A
:1050600002D00A6A000EE552B3EFE5F0AEECE5F0CF
:1050700085ECEDF03B812C8C2D8A5DECE8F032EC78
:10508000E6F0EE50ED1011E00101472B640E475D94
:1050900003E2BEDF00091BE10101470703E0B8DFBF
:1050A0000009FAE10101472B12D001014707FF0E69
:1050B000475D03E0ADDF00090AE10101472B640E03
:1050C000475D03E2A5DF0009F8E101014707B3EFFF
:1050D000E5F02A50800B0DE001013A51400B09E048
:1050E0002C50100B06E12B50010B03E1100E2E5D2E
:1050F00001E3000C010CD5ECEFF004E0D9ECEFF08B
:1051000001E2010C000C0701E06B070E1315006EA5
:10511000400E136F0050131301013A9D2BAA38D093
:10512000020E3C5D02E10701138701013C510208B8
:1051300007E2070E3C5D04E2020E3C5D0701E06FF2
:105140002AAE26D0070E01013C5D0BE12C50100B5E
:1051500008E14B51780803E26C0E4B5D4B6F95EC08
:1051600056F0080E01013C5D13E33A8D4B5178086F
:1051700004E207011387139B139D01013C510808AA
:1051800007E20D0E3C5D04E2080E3C5D0701E06F96
:1051900007011291129312892FECE7F00EE007013C
:1051A000128112831299B5ECE8F005E02E0505E1B5
:1051B0006251400B02E10701128921AC02D09CEC44
:1051C0000FF0BBEC2CF0258A120030ECF0F04B6AAB
:1051D000DA0F4A6E060E61ECF0F0006E009EFE0ED5
:1051E000DB50040806E1FD0EDB504F0802E2020E20
:1051F000006EB3EFE5F00101E851200B03E04651EA
:10520000040803E34651040801E2466B040E465DC0
:1052100002E1190E04D0160E462563ECE6F0006E8E
:105220000050E66EE66A3C0EE66EFEECFAF065ECC7
:10523000F4F003EC0CF0258A12000201320E346FF8
:10524000395102E0140E346FC80E496F640E506F6E
:105250001EAC2A981E50400B03E02B50800B02E13D
:10526000E3EC18F00201916BFD6B1200AEECE5F07F
:10527000FE0EDB500EE02AA006D0FE0EDB50030B24
:1052800002E1C5EC07F0280E5EECE9F0FE0EDB064D
:10529000EFD7B3EFE5F001C502F50501006B289CDF
:1052A0000101E391120056ECEAF0F5DF11ECE7F0B2
:1052B00002E0080E086E12000850220A01E167D1D0
:1052C000030A01E146D1010A01E1C7D03F0A17E014
:1052D000010A01E075D1288CD1ECEFF007E0200E37
:1052E00006014A5D03E0200E0CECE7F01E901F0E55
:1052F000086E02013D5101E164D1086A17D0050131
:10530000005101E181D011ECE7F014E005011151E9
:1053100007E1020E145D0EE18BEC0FF000090AE1CB
:1053200002013D5101E13D2B080E086E01011F0EE7
:10533000A96F1200050100070251EA6A000FE96E29
:10534000080EEA22EFCF02F7022B025139ECE6F009
:1053500002E6E1ECEEF001E3026B11ECE7F006E0AF
:1053600002C7E6FF08EC50F0E5524BD03C0E0701B7
:10537000025D04E12582248C239C12003E0E025D16
:1053800004E12592249C238C1200740E025D64E0DB
:105390000601F05107E02A8A02C7E6FF1FEC8BF0F6
:1053A000E5522A9A800E0701025D10E2C00E022526
:1053B0004A6E4B6A000E4B22200E4A5E000E4B5A7C
:1053C0000DECE6F0E8ECE7F00701026F800E025DFD
:1053D00003E10201040E676F07010251800805E234
:1053E000800E025DFD0F0201676F800E0701025DF6
:1053F00006E3220E086E05011F0E056F1200025112
:105400002BE0200E086E1200B6ECECF007E007016E
:105410000251800803E3200E0CECE7F044DF11ECAE
:10542000E7F006E0289C080E086E0101100EA96F37
:105430002850200B01E1C5D002016A5101E1C1D021
:10544000199A6ABF198A2A6B010EE66E7F0E6A15D9
:10545000D8ECE7F002016A6B12001850800B09E1EA
:105460001E50040B06E01E50080B03E08150080B91
:105470004CE12850200B09E01850800B06E001ECAD
:10548000EDF003E0250E165C1FE155EC81F00BDF1B
:10549000219411ECE7F003E00201010E3D6F28AA10
:1054A00090D002016A6B6AC22AF20601F05101E152
:1054B00088D007010251800801E283D03088200E95
:1054C000E66E1FEC8BF01DD0350E165C09E1010E67
:1054D000E66EACEC0FF0E552BBECECF0189E12005F
:1054E000A2ECB6F000090FE00D50006E020ECFECFA
:1054F000F3F00D50026E00500D6E0250E66EEEECB1
:105500008FF0E5521200F6EFB9F011ECE7F006E08B
:10551000080E086E01011F0EA96F1200FE0E070192
:1055200002150EE0238E010E016F02A102D0030EC0
:10553000016F02910243210E086E0501200E07D073
:105540000201020E676F220E086E05011F0E056F25
:1055500012000701015114E00107248008EC81F0DA
:10556000086A1EA007D0020E086EAFECEBF002E155
:10557000FEECE9F00101210EA96F1E80239E1200AE
:105580000201010E676F238E220E086E12000201C7
:10559000675113E02490670708EC81F0030E086E52
:1055A0001EB005D0070E086E006A19EC92F00101DA
:1055B000220EA96F239E1E90120005C508F012004E
:1055C00072DE120087C206F1AAECE9F00AE2100EC0
:1055D0002E5DD7ECE6F0060ECAECF0F0EFCF06F148
:1055E00004D02CA802D0960E066F0651D8804B55D9
:1055F00002E206C14BF11200DACFE4FFE2CFDAFF9C
:10560000E9CFE4FFEACFE4FFE652FC0EB36EF30EFF
:10561000B26E020125070201255105E10201320E99
:10562000256F010124811E961E9401015AA105D007
:1056300081B41E8481B21E8604D081B21E8481B4DE
:105640001E86020126070201265137E10201050EDE
:10565000266F0101AD5116E00101AD070201020103
:105660006651020B05E01E50040B02E10201668147
:10567000020102016651080B05E01E50080B02E111
:10568000020166850101AE5106E0FF0E0101AE5D2B
:1056900002E00101AE2B20AE04D00601E42B000E87
:1056A000E52307017D5109E007017D0707017D51D1
:1056B00004E17EC77DF7010124830101AC5102E0C2
:1056C0000101AC0702010D2B010129970101299568
:1056D000010129A102D001012985010129A302D0DC
:1056E00001012987010129930101299188A202D092
:1056F0000101298188A002D0010129830F0E010137
:1057000029150101266F01012651EA6AC90FE96EC8
:10571000060EEA22EFCF25F1010125A12FD020505E
:10572000080B08E0010101013E51010B03E0285084
:10573000010B24E02E50400B03E03050200B1EE004
:105740002150200B1BE0010125AF03D001012707E9
:1057500002D00101272B01010101CE51100B0EE0F7
:105760002050080B0BE02C50200B08E1010125AF65
:1057700003D00101280702D00101282B01012A973B
:1057800001012A9501012AA102D001012A85010106
:105790002AA302D001012A8701012A9301012A913B
:1057A00088A802D001012A8188AA02D001012A8397
:1057B0000F0E01012A150101266F01012651EA6A27
:1057C000C90FE96E060EEA22EFCF25F1010125A1EE
:1057D00026D0010101013E51200B16E12050080B9B
:1057E00013E02E50400B08E1010101013E51020B74
:1057F0000BE02850010B08E12E50400B10E0010196
:1058000001013E51010B0BE12150200B08E0010189
:1058100025AF03D00101280702D00101282B9EAA41
:105820001CD0ABA209D0AB98000000000000000023
:1058300000000000AB8811D00701C72B0701C6513B
:10584000C62BEA6A000FE96E0C0EEA22AECFEFFF1C
:105850000701C75102E1C6C7C5F7A1920701520768
:10586000E552E5CFEAFFE5CFE9FFE5CFDAFF11002A
:1058700001013EAB02D03E9B248A12000701EFB12A
:1058800003D0129A129812001298EFA31288129A5B
:10589000EFB3128A12000701EF81DDEC09F0C0EFCF
:1058A000ECF019A602D0199612002CA806D001011E
:1058B000E5A523D0560EDBEFE5F04B0E0A6E200E69
:1058C000016E12A002D0600E016E015035ECF5F0B1
:1058D000005013E0FF0E005C10E026840101B36B62
:1058E00047C11FF2FC0E476F12B0472B8EECE8F059
:1058F00071ECE9F026941FC247F11200220E3BEF33
:10590000F4F001018DAD09D0DE752E51635D0CE11F
:10591000D195DEA509D0D18507D0DE792E51635D02
:1059200003E1D199DEB9D18985EC0CF038EF0DF0A7
:1059300034AC02D081EF2CF02CA61BD01270129246
:1059400012A012820101CF9F12B0CF8F0701169FC4
:1059500012B0168FB3EC09F0E66A0EECC8F0E5520F
:10596000D1ECC6F00201916B258A17859ADFACEF66
:105970000CF07EEF2CF068ECE6F003E011ECE7F0C1
:1059800006E01494010159A306D0148404D01494A1
:1059900001013EB51484149614A41486149814506E
:1059A000040B04E12FECE7F001E0148812001AEC7C
:1059B000F0F0006A0301C95111E0CCC359F2CDC324
:1059C0005AF2800ECD151DE0CCC359F2CDC35AF268
:1059D0000201596D5A1F000E5A2311D0C4ECEDF08C
:1059E000595F7A0E5A5B0101A00E525D7A0E53592F
:1059F00008E2C4ECEDF0D88059577A0E5A57800E61
:105A0000006E060E436E446A59C23EF05AC23FF021
:105A1000B8ECFDF03EC059F23FC05AF2005002010E
:105A20005A1301017AA717D0C4EC3EF098EC97F016
:105A300002C101F003C102F004C103F005C107F186
:105A4000076A560E4FECEBF0010E076E560E4FEC48
:105A5000EBF0DF50076EE552B3EFE5F0AEECE5F0AA
:105A6000FB0EDBCFE9FFFC0EDBCFEAFFEECF4AF007
:105A7000EECF4BF0EECF4CF0EECF4DF0EFCF4EF03F
:105A80002CECE9F04AC0EEFF4BC0EEFF4CC0EEFF3D
:105A90004DC0EEFF4EC0EEFFB3EFE5F087ECF4F043
:105AA00096ECE7F0A10EE66E010EDCECE9F0D3EC2B
:105AB0003AF0D8A002D0010E01D0000EB3EFE5F00D
:105AC00013ECF0F00050B3ECF2F01AECFEF015EC31
:105AD000FEF00009FCE1C450006E1C50040B32E0E3
:105AE0008BECF1F004E6F90E4A5C000E4B582AE20A
:105AF0000201F3514B6AE8307F0B4A6EC80EE1ECAD
:105B0000F0F0D6ECF1F076ECE8F06FECF0F0EECFE0
:105B10003EF0EDCF3FF067ECF9F03CC0EEFF3DC04A
:105B2000EDFF76ECE8F0FA0E436E446AEECF3EF0FD
:105B3000EDCF3FF0B8ECFDF03EC0EEFF3FC0EDFF13
:105B4000EF50006E020EE15C02E2E16AE552E16EA6
:105B5000B3EFE5F00FECF0F00050DF6ED70E4A6EB9
:105B6000EA0E4B6E010EE6ECF1F00150006E009E65
:105B7000E6EC97F001AEF2D7E552B3EFE5F00FECAB
:105B8000F0F00050DF6E2450100B12E10050E66E72
:105B90008EEC04F0E552800B0BE00101450E196F0D
:105BA000520E1B6F1BC11AF1200E1C6F040E016FE9
:105BB0002B8824A808D0D30E4A6EEC0E4B6E010E33
:105BC000E6ECF1F007D0DFCFE6FF8EEC04F0E55213
:105BD000016EDF2A2BA802D0019E2B980150006E87
:105BE000009E11EC98F001AEE4D72498E552B3EF93
:105BF000E5F00DECF2F003E2C5ECEFF004D0FE0EA0
:105C0000DB50410FF60F006EE6EC97F0B3EFE5F0D6
:105C10009CECF4F0DB380F0BE66EEBDFE552FE0E8A
:105C2000DB500F0BE66EE5DFE552B3EFE5F0AEECCF
:105C3000E5F0CBECEDF0020E010100275BEC97F0F4
:105C4000DF50006E050E0101005F5BEC97F0030E64
:105C50000101005FE552B3EFE5F0AEECE5F0CBEC0F
:105C6000EDF05CECEAF0DF50006E0101020E016F16
:105C700078EC97F0E552B3EFE5F000C06FF271EC0D
:105C800094F0FF0E005C01E065DF0101B2891200B3
:105C900000C070F27DEC94F0FF0E005C01E06FDF5D
:105CA0000101B28B120071EC94F0FF0E005C01E078
:105CB00051DF0101B28D640E096E259612007DEC54
:105CC00094F0FF0E005C01E05ADF0101B28F640E18
:105CD000096E25961200AEECE5F08EECE8F07CEC57
:105CE000EBF0DEECE7F0B3EFE5F0AEECE5F08EECD8
:105CF000E8F0A0EFF1F0AEECE5F0D3EC8AF00101B2
:105D0000190EAB6FFC0EDBCFAFF1FD0EDBCFB0F1A8
:105D1000FE0EDBCFB1F1B3EFE5F0830E0A6EE00EBD
:105D200035ECF5F0800E005C08E2D3EC8AF001015E
:105D3000190EAB6F0201E00EE06F12009CECF4F064
:105D4000DBCF4BF0800E4B1407E0D2ECEDF04A6C49
:105D50004B1E000E4B2202D0D2ECEDF097ECF3F08C
:105D6000B3EFE5F0016A040E015C0DE201281BECC3
:105D7000F1F0EA2254ECEBF001501BECF1F05DEC99
:105D8000ECF0012AF0D7EA0EF7ECE7F00301C46F5C
:105D9000318A8AECF2F00301C56F319A0101E38781
:105DA0000480016A040E015C22E201501BECF1F058
:105DB000EA22EECF4CF0EFCF4DF001281BECF1F0D2
:105DC000EA22EE504C5C4A6EEE504D5899ECF4F0DD
:105DD0001DECF3F0010E24ECE7F007E20490050E51
:105DE00024ECE7F002E20101E397012ADBD704503B
:105DF000010B49E001019151080B03E102015151EE
:105E000042E00101B251020B3EE1020150513BE17F
:105E1000BCC3E6FFBDC3E6FF1DECF3F00F5010104E
:105E200032E0F40E0F5C010E10582DE20401440E16
:105E3000FB6F0301800EBD1503E00401550EFB6FDF
:105E4000CBECEBF0040E24ECE7F002E2310E026F33
:105E5000140E24ECE7F002E2330E026F3C0E24EC49
:105E6000E7F002E2390E026FDC0E24ECE7F002E20A
:105E7000340E026F020EDDECEFF003E20201320E8F
:105E8000506F4CECD0F012009CECF4F0DBAE08D07C
:105E9000DB50FF0DFE0EF3CFDBFFEBECEBF007D09A
:105EA000EBECEBF0DB50FF0DFE0EF3CFDBFFDB5036
:105EB000B3EFE5F00FECF0F00701875101E047D1B7
:105EC000F10501E144D13350040B01E13FD10C5005
:105ED00004E18650020B01E139D1E30EF7ECE7F063
:105EE0000601C16F09ECE8F001E096D0140E06013E
:105EF000E76EC119E8AE02D0C13503D0E750D880B3
:105F0000C15502E2140EC16FEC0EE76EC119E8AE86
:105F100002D0E73402D0E750C15D02E2EC0EC16F5F
:105F2000C051E76EC119E8AE02D0C13503D0E750C9
:105F3000D880C15502E2C02B0BD0C051E76EC11909
:105F4000E8AE02D0E73402D0E750C15D03E2C007FB
:105F5000C0C6C1F6080E4A6E4B6AC5C63EF0C6C63C
:105F60003FF0D9ECEDF03EC0C4F6C4C64AF04B6A2F
:105F70004ABE4B684A500601C55F4B50C65BC1C65E
:105F80004AF04B6A4ABE4B684A50C5274B50C6235D
:105F9000C4C6E6FF79DFE552016E010EE66E0E0E15
:105FA0000124E2ECE7F002012B5101E1CFD01A9E6F
:105FB0008DECE9F002E0000E01D0010E4A6E0C50AB
:105FC00003E1C7ECEBF008E00C5004E00101CE5116
:105FD000040B02E0000E01D0010E4A1805E0060194
:105FE000C1510101272704D00601C1510101275FDA
:105FF000CE51100B05E02050020B02E127C128F121
:106000000601C15101E0A2D002012B51320801E387
:106010009DD0320E2B6F9AD0E40EF7ECE7F006011C
:10602000C36F026A016AC151E76EC319E8AE02D0BC
:10603000C33503D0E750D880C35505E2C151C35DD5
:1060400094ECEAF0026E0601C351E76EC119E8AEA6
:1060500002D0C13503D0E750D880C15505E2C35105
:10606000C15D94ECEAF0016E0601C251D880025481
:1060700002E202C0C2F6C051D880015402E201C05F
:10608000C0F6000EE76EC219E8AE02D0C23503D0EA
:10609000E750D880C25505E2010EE66E0D0EE2EC27
:1060A000E7F0010E0601E76EC219E8AE02D0C23574
:1060B00003D0E750D880C25505E2010EE66E0C0E03
:1060C000E2ECE7F0020E0601E76EC219E8AE02D07C
:1060D000C23503D0E750D880C25505E2010EE66E06
:1060E0000B0EE2ECE7F0000E0601E76EC019E8AE19
:1060F00002D0C03503D0E750D880C05505E2010E6C
:10610000E66E0F0EE2ECE7F0010E0601E76EC01935
:10611000E8AE02D0C03503D0E750D880C05505E2C4
:10612000010EE66E100EE2ECE7F0020E0601E76EDD
:10613000C019E8AE02D0C03503D0E750D880C055B2
:1061400005E2010EE66E110EE2ECE7F03394E55243
:10615000B3EFE5F00FECF0F00701F10504E1FD0EFF
:10616000DB6AFE0EDB6AFC0EDB504DE102013A51A8
:106170004AE10490FE0EDB50140804E2140E85EC94
:10618000E8F00480FE0EDBCF4AF06B51D8804A5411
:1061900003E2FE0EDBCF6BF201012D51100B03E089
:1061A000050E0C5C05E10450010B02E0FE0EDB2A3B
:1061B000DF6A150EDF5C1AE2006AFE0EDB5004E0B7
:1061C000FE0EDB50DF5C0BE301012D51100B09E0EB
:1061D000050E0C5C06E002016B51DF5C02E1010E72
:1061E000006E0050E2ECE9F0DF2AE3D71450010B17
:1061F0006AE00201315167E10C5003E0030E0C5CD0
:1062000062E1338460D0FC0EDB0431E102013A51DB
:1062100006E0FD0EDB5003E12350400B57E1FE0E7C
:10622000DB50080803E2080E85ECE8F0FD0EDB50B9
:106230000C0805E20C0EF36EFD0EF3CFDBFF91ECC4
:10624000E9F0150EDF5C3FE2FE0EDB5004E0FE0ECF
:10625000DB50DF5C07E3090EDF5C07E3FD0EDB507C
:10626000DF5C03E2010EE2ECE9F0DF2AEAD7FC0E84
:10627000DB50020828E1FE0EDB50080803E2080E9E
:1062800085ECE8F0FD0EDB500C0805E20B0EF36E1A
:10629000FD0EF3CFDBFF91ECE9F0150EDF5C13E2AE
:1062A000FE0EDB5004E0FE0EDB50DF5C07E3090E60
:1062B000DF5C07E3FD0EDB50DF5C03E2010EE2EC86
:1062C000E9F0DF2AEAD7FE0EDBCF1DF2E552B3EF8D
:1062D000E5F00101D351E9ECE9F003ECF5F00150F0
:1062E000080D4A50F3240A01E26F4B50F420E36F8B
:1062F00012000101C851C35D0CE1C951C45D09E13F
:10630000CA51C55D06E1CB51C65D03E1CC51C75D05
:1063100001E0000C010C0101D3510C5C01E0000C08
:106320000C500BE1CF51400B01E0010E4A6EDC51E5
:10633000400B01E0010E4A5C2CE0030E0C5C23E1F3
:10634000DB51FBECE6F0B65D1EE109ECE8F00CE099
:106350000101CF51040B01E0010E4B6EDC51040B27
:1063600001E0010E4B5C15E009ECE8F00CE10101E5
:10637000CE51040B01E0010E4C6EDB51040B01E029
:10638000010E4C5C06E00C5003E0030E0C5C01E1D6
:10639000000C010CAEDF000903E0BDDF000901E1E4
:1063A000000C010CF7DF000930E0050E0C5C01E188
:1063B000010C0101D351E9ECE9F07DECEDF0D35192
:1063C00028ECF2F00150B6ECF4F00C50100DF3CFC5
:1063D00050F0F4CF51F02A0E50260A0E5122070138
:1063E000E251080D5050F3244E6E5150F4204F6E80
:1063F0004EC0E6FF4FC0E6FF41ECFAF0526E060ECB
:10640000E15E5250000901E1010C000C2EC163F164
:106410000FC110F11BB202D033ECE7F00CC0D3F186
:106420002E50400B03E13550200B17E001013BA338
:1064300006D0DD93D0B3DD83DD95D0B5DD85DC9D61
:10644000CFBDDC8DDC95CFB5DC85DB95CEB5DB85AE
:1064500049ECF4F0E9ECF0F01AD00101D35103E17A
:10646000DC9DCFBDDC8D030ED35D11E149ECF4F072
:10647000E9ECF0F009ECE8F006E00101DC95CFA5CD
:1064800006D0DC8504D00101DB95CEB5DB852E502E
:10649000400B03E13550200B0DE0500EE66EE66A2E
:1064A0002A0EE66E0A0EE66E7A0EE66E0A0E82EC92
:1064B000E7F00DD0050E0C5C0AE0100EE66EE66A01
:1064C0003CECF1F0D35128ECF2F023ECF3F0E1ECEA
:1064D000EFF008E0D351EA6ACF0FE96E0A0EEA2224
:1064E000E2C7EFFF120063C12EF110C10FF19FEC64
:1064F000EAF0D3C10CF02E50400B03E13550200BD5
:1065000008E030ECEDF02A0EE66E0A0E82ECE7F0C1
:106510000DD0050E0C5C0AE0D9ECF0F00C50100D1B
:10652000F2ECE7F0F0ECEEF023ECF3F0050E0C5C8F
:1065300002E0BDECF3F01200AEECE5F033DF000951
:106540000FE1C0EC15F0FE0EDB5002E15FDF01D081
:10655000CADFC4ECECF0258A85ECEDF03B833B818F
:10656000B3EFE5F02D50100B13E0A6ECE9F010E0CE
:10657000C0EC15F04BDF010E076E1982A6EC0DF092
:1065800048EC15F0076AA6EC0DF048EC15F01992EE
:1065900012002E8C35ECEFF04FEC0AF01B9431EC2E
:1065A000EFF0076A01013EA90DD0348C010EE66EB2
:1065B0001BD9E552A6EC0DF046EC4BF0BBECEBF032
:1065C00085EC0CF048EF15F0AEECE5F031ECEFF0B7
:1065D0007AECEAF012E1CF91DCB1CF81CF93DCB35A
:1065E000CF83D195DEB5D185D199DEB9D189D1914D
:1065F000DEB1D181D19FDEBFD18F2E9CB2993EA951
:1066000006D0349CE66AF0D8E552A6EC0DF048ECD2
:1066100015F0FE0EDB5002E046EC4BF0E6EC1CF011
:10662000BBECEBF0B3EFE5F0C0EC15F07AECEAF080
:1066300011E048ECE7F0358A17D8359A48EC15F0A8
:106640001D8A48ECE7F01D9A19847BECE8F0199458
:1066500063EFECF03EA903D038ECEFF0076A04D802
:1066600048EC15F0D1EF10F063C102F010C103F057
:10667000C8C1D0F2C9C1D1F2CAC1D2F2CBC1D3F2E2
:10668000CCC1D4F2D3C100F03CECEFF0DDC1E1F1BC
:106690002E50400B03E13550200B08E030ECEDF0BC
:1066A000580EE66E060E82ECE7F00BD0050E005C8D
:1066B00008E0D9ECF0F0580EE66E060EE66EDCEC63
:1066C000EDF0016A050E005C03E00050E9ECE9F032
:1066D0009DDE02C02EF103C00FF1D0C2C3F1D1C2C2
:1066E000C4F1D2C2C5F1D3C2C6F1D4C2C7F10050C1
:1066F0000C6E2E50400B03E13550200B1EE00101C3
:106700003BA30ED0D093E1B3D083D095E1B5D08533
:106710001396D0B313861394D0B5138441ECC1F013
:106720000101CF9DE0BDCF8DCF95E0B5CF85CE9552
:10673000DFB5CE85BCECF0F019D00C5004E10101BE
:10674000CF9DE0BDCF8D030E0C5C10E10101BCECD0
:10675000F0F009ECE8F006E00101CF95E0A506D0E5
:10676000CF8504D00101CE95DFB5CE852E50400BEC
:1067700003E13550200B09E0500EE3ECEDF02A0E5A
:10678000E66E0A0E82ECE7F00AD0050E005C07E028
:10679000100EE3ECEDF03CECF1F0DCECEDF001C0C0
:1067A000E2F7050E0C5C04E04FECE8F001C0EFFFEF
:1067B000049001013EB104803E913EB33E813E9380
:1067C00004B03E83139C3EB1138C139E3EB3138ED4
:1067D0002EBC03D0C4ECECF0258AFCEC38F085EC40
:1067E000EDF0BF0E3B6F120030ECF0F00AE0076AEC
:1067F00001016595E1EC23F0010E076E01015F8553
:1068000009D0010E076E01015F95E1EC23F0076AE4
:1068100001016585E1EC23F0B3EFE5F013ECF0F056
:106820000E0E0101325DDF6E060E332545ECEBF0F6
:106830000601F45126E0DCECEEF0060ED8901032A2
:106840000F32E804FBE1040EDF02F3501DECF2F01E
:10685000200E41ECEFF002E20F6A106A010EDB50ED
:106860004C6E4D6A80ECE8F0070E07ECE9F001ECA5
:10687000E9F0FF0E24ECE7F002E20F68106A0FC0A7
:10688000F5F6DF50005EFAECF0F006E24A50C80878
:10689000000E4B5401E2006A010EDB504C6E4D6A53
:1068A0000050060D12ECE6F001ECE9F00F50006E1E
:1068B0000050150802E2150E006E020EE15C02E2C5
:1068C000E16AE552E16EB3EFE5F00FECF0F00201A2
:1068D000315105E12150010B02E1345102E0000E7B
:1068E0001DD0AF0EB1ECE6F099DF0050DF6E00C0B6
:1068F000D4F7090E016E01012DB901061450010BE8
:1069000006E00150D880005402E20150006EE66AB1
:10691000E66A0050E66E45ECE9F0DF50E552B3EF71
:10692000E5F0AEECE5F0016A0A0E015C19E2FE0E3C
:10693000DB50010B06E0270E012443ECE6F0165C69
:106940000AE0FE0EDB50020B09E0310E012443EC9D
:10695000E6F0165C03E101500D6E02D0012AE4D787
:10696000B3EFE5F0AEECE5F0800E0D6E18AE17D08B
:10697000189E1850010B03E11850100B10E0100E78
:106980000D6E4FECE6F0CDDFE5522A0E165C02E10B
:10699000200E0D6E2B0E165C02E1400E0D6EB3EF55
:1069A000E5F0AEECE5F0AAECEAF04FECE6F0F5EC41
:1069B0000BF0E552D4ECF3F00101A66FA651640D83
:1069C0002DECE6F0010EEB50680FEBECF2F0D9EC99
:1069D000F3F0EAECEDF000504C6E4D6A01014C50C2
:1069E0004A5CD76F4D504B58D86F2AA60BD09C519C
:1069F000EAECEDF00101D7514A5C0F6ED8514B58CB
:106A0000106E06D09C51106AD7250F6ED8511022F7
:106A10009DECEFF056ECF0F03EC0A6F13AC09CF1D0
:106A2000B3EFE5F0AEECE5F0AAECEAF0DB50D7EC22
:106A3000E6F0030ECAECF0F0EF500101A65D02E0B3
:106A4000000E11D0FE0EDB50D7ECE6F0B3ECECF00C
:106A5000EF509C5D006E00BE006C040E005C02E214
:106A6000010E01D0000EB3EFE5F04CECF4F0920E05
:106A70004A1810E14B500EE1006A3DEC2EF0BD0EBD
:106A8000006E48EC2EF0096A228602018E6B7F6B45
:106A9000299E082A4CECF4F0930E4A1845E14B501D
:106AA00043E1010EE66E5EDFE5520A0E0D5C25E263
:106AB00002018E51050826E37F51020823E38E2B45
:106AC00029BE7F2B010E016E070E015C13E2012827
:106AD00085ECE6F0EF50006E060E015C05E1800EDD
:106AE000010118150D10006EEFECF2F000C0EFFF81
:106AF000012AEAD70101189F17D0200E0D5C08E18A
:106B000029AE02D0268E10D0298E0101188F0CD00C
:106B1000400E0D5C04E1980E086E1B8805D0100E27
:106B20000D5C02E19A0E086E4CECF4F0980E4A18D7
:106B300001E07DD04B5001E07AD0010E016E070ECE
:106B4000015C0DE2EFECF2F0EF9EEFECF2F0EF50B3
:106B50000E0803E1EFECF2F0EF6A012AF0D712C160
:106B6000A6F10A0E01011303F35014259C6F0A0EBF
:106B70001503F35016259D6F0A0E1703F3CF9EF1F0
:106B8000A06BA0C19FF1040E02018E5D0DE27F514A
:106B90000BE115C1A6F10A0E01011603F3501725EA
:106BA0009C6F9E6B9EC19DF102017F0508E114C19F
:106BB000A6F19DC19CF19EC19DF101019E6B020E4B
:106BC00002017F5D0EE113C1A6F10A0E010114035B
:106BD000F35015259C6F0A0E1603F35017259D6F71
:106BE0009E6B9A0E086ED8EC0DF0006E005013E10B
:106BF0000101A65103E19C51370802E2268E1200E2
:106C000016ECE9F00A0E005C06E10101E251010B0D
:106C100002E037EF09F000C02EF17BECE8F09EECCB
:106C200004F056EC0BF0D0ECEEF05DECE8F04CEC40
:106C3000F4F09A0E4A1808E14B5006E10101B29BAC
:106C4000B29953DA0C0E086E12008C9804902EB094
:106C50000480075003E004902FBC04803F0E07011E
:106C60003715006E04A002D0008C01D0008E010107
:106C700090A102D0300EC66E0050E66E04EC7AF0A1
:106C8000E55236C7E6FF04EC7AF0E55239C700F06A
:106C9000040E0002F3CF00F0070138BF00820701A5
:106CA00038BD008038C701F0040E0102F3CF01F0B7
:106CB000070137BF0182070137BD018004A002D060
:106CC000008C01D0008E0050E66E04EC7AF0E552A4
:106CD0000150E66E04EC7AF0E5520470200E006E6E
:106CE00004A002D0280E006E0050E66E04EC7AF08C
:106CF000E552080EE66E04EC7AF0E5528C8800004E
:106D0000310EC66E075004E12E9004B02E8003D0E1
:106D10002F9C04B02F8C120001017AB71FD015EC04
:106D20007AF0080E07244A6EF00E8C144A108C6E0E
:106D300081EC5EF08A9A0000E3EC08F0210EE66E2A
:106D400004EC7AF0E552080EE66E04EC7AF0E552B7
:106D50007CDF8A8AF00E8C1611EC7AF012000101A9
:106D60007AB71BD002010D6B15EC7AF0080E0724E0
:106D70004A6EF00E8C144A108C6E81EC5EF08A9A8A
:106D8000000063DF37C73AF738C73BF78A8AF00E4F
:106D90008C1611EC7AF00DC20EF212000750020DA3
:106DA000F3CF5BF7F4CF5CF7530E07015B27070EB9
:106DB0005C230750020DF3CF65F7F4CF66F75D0E45
:106DC0006527070E662301019C51C80D12ECE6F001
:106DD0009D51020D4A50F3240F6E4B50F420106E5B
:106DE0009E51310803E20F2A000E1022CC0E0F5ED6
:106DF000060E105AD3EC09F0006E005012E000505D
:106E0000D8ECF2F0400B03E12850040B0AE00050EC
:106E1000E66E5BEC0EF0E5520050310802E25DECEC
:106E2000E8F0010EE66E64EC99F0E552320E4B6E1E
:106E30004BC044F09EC13FF0FCECFDF03BC04AF07B
:106E40000A0E4C6E4CC044F04AC03FF092ECF1F098
:106E5000056EDFECE8F0EE50ED103CE00150055C13
:106E600044E30F2A000E10220201C9510F1812E14B
:106E7000CA5110180FE1DFECE8F0CBC2EEFFCCC234
:106E8000EDFF04ECE8F0CDC2EEFFCEC2EDFFCFC2C5
:106E900001F01AD0E66A64EC99F0E5520201A1070C
:106EA000000EA25BDFECE8F0EECFCBF2EDCFCCF240
:106EB00004ECE8F0EECFCDF2EDCFCEF201C0CFF290
:106EC0000FC0C9F210C0CAF2DFECE8F0EE50ED10CE
:106ED0000CE109D005504A6E4B6A04ECE8F04A50C8
:106EE000EE264B50ED22D3EC99F02E9AD3ECF1F034
:106EF000570EE926070EEA2254ECEBF0DFECE8F03F
:106F0000EECF4CF0EFCF4DF04C504A1819E14D50F8
:106F10004B1816E1D3ECF1F0610EE926070EEA22D8
:106F2000EECF4EF0EFCF4FF004ECE8F0EECF50F0A4
:106F3000EFCF51F050504E1802E151504F181AE067
:106F40002E8ADFECE8F054ECEBF0D3ECF1F0570EC6
:106F5000E926070E5DECECF004ECE8F054ECEBF005
:106F6000D3ECF1F0610EE926070E5DECECF0040EB7
:106F7000A4ECECF012000C0E07244A6EF00E8C14F8
:106F80004A108C6E81EC5EF08A9A00000750E96E20
:106F9000EA6AD890E936EA36530EE926070EEA2265
:106FA000EECF0FF0EDCF10F0E3EC08F0E66A04EC62
:106FB0007AF0E55200011050040DF350006E060EF9
:106FC0000FC0E7FF070B04E0E742E79EE806FCE19D
:106FD000E7500010E66E04EC7AF0E55200010F5025
:106FE000040DF350E66E04EC7AF0E552EDEC08F097
:106FF0000750E96EEA6AD890E936EA365D0EE9266E
:10700000070EEA22EECF0FF0EDCF10F0E3EC08F020
:1070100010C0E6FF04EC7AF0E5520FC0E6FF04EC86
:107020007AF0E552010EE66E04EC7AF0E552EDECF2
:1070300008F08A8A00000000F00E8C161200D9CFEA
:10704000E6FFE1CFD9FF01017AB74BD0FE0EDB504E
:1070500001E0A4DEFD0EDBCF90F20C0E07244A6E99
:10706000F00E8C144A108C6E81EC5EF08A9A00004F
:10707000E3EC08F0FD0EDB407F0B4A6EFD0EDB50AB
:10708000040DF3504A10E66E04EC7AF0E552FD0E62
:10709000DB40E8403F0B800DF350006E0050E66E81
:1070A00004EC7AF0E55207015139F00B006EFE0E48
:1070B000DB5003E0030E001201D000820050E66EA8
:1070C00004EC7AF0E552EDEC08F0FE0EDB5002E045
:1070D00052DF07D0000000008A8A00000000F00E96
:1070E0008C16E552E7CFD9FF120086D8D8EC3EF0D7
:1070F0002682248A120053C2A5F154C2A4F155C2BB
:10710000A3F10101A26BA16B20A402D0AFEF3AF072
:10711000D3EF3AF013C201F014C202F015C203F02B
:1071200078EC44F002011351015C06E11451025C59
:1071300003E11551035C04E0C5EC45F084EC5EF01E
:10714000120040ECF5F0010190A715D0FE0EDB50C7
:1071500008E0FD0EDB5005E1DF68CEA102D0010E94
:10716000DF6EFE0EDB5007E1FD0EDB5004E0010E8A
:10717000DF6ECEB1DF68DF501FE070ECE6F0A56B8C
:10718000A5C1A2F1A5C1A1F129ECF3F08DECE9F0C4
:1071900002E0000E01D0010E4A6EDF0402E0000E94
:1071A00001D0010E4A1802E0DAD901D0FCD99EECD8
:1071B00004F085ECEDF03B81E552B3EFE5F0010121
:1071C000A56BA46BA36B0201B451E8244A6E640E54
:1071D0007BECE7F03BC0A2F1320EFDECF0F0B4C264
:1071E0003FF0FCECFDF03FC0A1F10201B5A102D0DF
:1071F000AFEF3AF0D3EF3AF008AE6ED02C50400B20
:1072000003E02D50200B31E0800E0101C31507E192
:10721000C3510EE10301E3510101C45D09E2C36BF7
:10722000E3C3C4F1C76BC7C1C6F1C7C1C5F11DD067
:10723000100E2E5D1AE2360EC35D03E3360EC36FE9
:107240000DD01E0EC35D11E32C0EC35D0EE2250EA4
:10725000C35D02E21E0E01D02C0EC36FC76BC7C107
:10726000C6F1C7C1C5F1C7C1C4F12C50400B03E042
:107270002D50200B31E1800E0101C81507E1C851E6
:107280000EE10301E3510101C95D09E2C86BE3C3EB
:10729000C9F1CC6BCCC1CBF1CCC1CAF11DD0100E61
:1072A000635D1AE2360EC85D03E3360EC86F0DD07B
:1072B0001E0EC85D11E32C0EC85D0EE2250EC85DE2
:1072C00002E21E0E01D02C0EC86FCC6BCCC1CBF1EC
:1072D000CCC1CAF1CCC1C9F1AAECE9F023E2E55175
:1072E000040B20E0C3511D0809E2E351200B03E029
:1072F000E351400B0FE0E38B230E08D0E351200B4A
:1073000003E1E351400B06E0E39B110EE66ECDEC8A
:1073100008F0E552A6ECE9F005E02E51635D02E1CC
:10732000C3C1C8F12C50400B03E02D50200B23E0CB
:107330002150400B09E11350080B06E02E50400B82
:1073400012E0CE51100B0FE12150400B12E0205003
:10735000020B03E11350040B06E12050020B09E07D
:107360001350080B06E070ECE6F0C5DEB5ECEAF071
:1073700002D0C0ECEAF02C50400B03E02D50200B63
:1073800025E12150400B03E01950400B09E0135058
:10739000080B06E02E50400B09E1B3ECEBF006E1E0
:1073A0002050020B11E01350040B0EE027ECE8F024
:1073B000A2DE9CC1BEF19DC1BFF19EC1C0F19FC1C3
:1073C000C1F1A0C1C2F102D0CBECEAF001017A51C7
:1073D000040B09E0800E081406E0100E2E5D03E297
:1073E0000201280EFA6F2050020B19E10201B5517B
:1073F000010B03E1B551020B12E0050E0C5C07E036
:107400002150800B0CE0050E01019B5D08E121502D
:10741000400B05E032ECE8F0D2DEB5ECEAF02E509D
:10742000400B01E09BD02C50400B04E185ECE9F0CF
:1074300001E194D02EC100F02C50400B05E02D50FE
:10744000200B02E163C100F0800E081401E186D038
:10745000100E005C01E382D021EC11F02DBA0DD0AA
:10746000D6ECEAF0C8C1A1F1C9C1A2F1CAC1A3F129
:10747000CBC1A4F1CCC1A5F10CD032ECE8F0C3C172
:10748000A1F1C4C1A2F1C5C1A3F1C6C1A4F1C7C194
:10749000A5F116ECE9F02D50200B04E0005001019D
:1074A0002E5D07E12D50200B49E100500101635D85
:1074B00045E02DAA0BD000C00FF100C02EF162B73D
:1074C0000FD000C010F100C063F10AD000C010F16D
:1074D00000C063F162B704D000C00FF100C02EF10C
:1074E0002EC1D2F1BBECE9F02EC1E6FFE6680BEC51
:1074F00047F0E552E552056E010162B70FD02DAAA3
:1075000006D0050EE66E052401ECEAF005D0050E66
:10751000E66E055059ECEBF017ECE6F00E0E052484
:1075200029ECE7F00101D19B00BAD18B0A6AC2ECC9
:1075300046F021820201010E346F12002050010B2F
:1075400003E02D50200B09E13150020B07E02D50D4
:10755000200B04E1A6ECE9F001E0DCDD1200010102
:10756000A551A027A051090803E20A0EA05F9F2B96
:10757000A4519F279F51090803E20A0E9F5F9E2B8B
:10758000A3519E279E51630803E2640E9E5F9D2BCC
:10759000A2519D279D51630803E2640E9D5F9C2BC1
:1075A000A1519C2712000101A551A05FA0510A081A
:1075B00003E20A0EA0279F07A4519F5F9F510A086C
:1075C00003E20A0E9F279E07A3519E5F9E51640807
:1075D00003E2640E9E279D07A2519D5F9D516408A2
:1075E00003E2640E9D279C07A1519C5F1200F00EE0
:1075F0008C140F098C6E81EC5EF08A9A000018C71B
:10760000E6FF04EC7AF0E552E3EC08F0EDEC08F06C
:107610008A8A12002D9007500701196F1A6B170EF6
:1076200007011927070E07011A23470E4A6E19C7CB
:10763000E9FF1AC7EAFF4A50EF120750EA6A2F0F14
:10764000E96E070EEA22EFCF33F7070133A105D029
:1076500019C7E9FF1AC7EAFFEF94070133A305D062
:1076600019C7E9FF1AC7EAFFEF92070133A505D052
:1076700019C7E9FF1AC7EAFFEF90070133AD05D03C
:1076800019C7E9FF1AC7EAFFEF9C0E0E07244A6EDE
:10769000F00E8C144A108C6E81EC5EF08A9A000019
:1076A0000750EA6A170FE96E070EEA22EF50E66EFE
:1076B00004EC7AF0E552E3EC08F0EDEC08F082A877
:1076C0002D808A8A1200A6DF050E3EEFE6F0AEECB2
:1076D000E5F001017AB73ED064ECE8F0EFCF33F784
:1076E000FE0EDB5006E1470EE1ECEAF0470B4A5C88
:1076F00001E090DFFE0EDB5006E1380EE1ECEAF02F
:10770000380B4A5C21E007500701196F1A6B170EFE
:107710001927070E1A23570E4A6EC8ECECF04A5090
:10772000EF1633A703D0C8ECECF0EF8633A903D0F3
:10773000C8ECECF0EF8E33BB03D0C8ECECF0EF8A72
:10774000C2DF010EDAECE8F02FECF3F033C7EFFF05
:10775000F00E8C16B3EFE5F00701040E506FD890D1
:107760004033413342334333443345334633473365
:10777000502FF6D7120001017AB71200D3ECF1F0C6
:10778000530EE926070EEA22EECF67F7EDCF68F732
:10779000D3ECF1F05D0EE926070EEA22EECF69F791
:1077A000EDCF6AF7030E07013C156B6F6C6B020E91
:1077B000D8903F333E333D333C33E806F9E167C7A9
:1077C0004AF068C74BF066ECE7F040ECFBF03BC0DA
:1077D000EDFF3AC0EDFF39C0EDFF38C0EFFF69C7DC
:1077E0004AF06AC74BF066ECE7F063ECFCF03FC090
:1077F000EDFF3EC0EDFF3DC0EDFF3CC0EFFF38C0E8
:107800006DF739C06EF7020E0701D8903C373D374F
:107810003E373F37E806F9E1020E0F0B070105E09E
:10782000D89068336733E806FBE1020E0F0B0701BF
:1078300005E0D8906A336933E806FBE16BC73EF098
:107840006CC73FF067C743F068C744F067ECF9F0D6
:107850003C5007016D254A6E3D506E214B6E060E61
:1078600007ECE9F075ECF1F069C743F06AC744F042
:1078700097ECF0F00701020E486FF10E496F03011B
:10788000C95107E0C1ECE8F0DAC14AF7D9C14BF7BA
:1078900004D053C14AF752C14BF73FC740F73EC728
:1078A00041F73DC742F73CC743F70701476B47C75E
:1078B00046F747C745F747C744F74EDF18EC27F0B0
:1078C00044C739F745C738F746C737F747C736F7CC
:1078D00000010F5007013627000110500701372320
:1078E000000E3823392312007EECF0F00050016EB8
:1078F000020E3EECE6F07EECF0F00050026E010E5F
:107900003EECE6F07EECF0F0040EE66E04ECEFF0F8
:107910009DECE7F009E0040ECDECEFF00250E66ECE
:107920009DECE7F001E0010C000C40ECF5F0F00EEE
:107930008C1607288C121C847EECF0F00701355160
:10794000005C15E23451005C12E322A20CD02292BA
:10795000CBDF000902E0DF2A0AD03C0E3EECE6F065
:10796000C3DF000903E0010EDF6E01D0DF6A1C9463
:10797000F00E8C16DF50E552B3EFE5F00750E82427
:107980007F0F10240A6E0F50016E1200AEECE5F06E
:10799000090EE1260F6A106A770E0F5C010E10586F
:1079A00008E2ECDF006805EC4DF00F2A000E102213
:1079B000F3D7E66A41ECEAF00701336B335139EC57
:1079C000E6F002E6FCECE7F001E33BD164ECE8F022
:1079D00033C7EFFF010EE66E7ADEE5520C0EDAECED
:1079E000E8F01F0EE5ECEFF023ECE8F033C700F011
:1079F0005BEC97F01AA802D000EC05F03BEC96F097
:107A000033C700F0620EDE6EDD6A560E1FECE7F043
:107A1000030EDB6A400E005C63E2DC0EF1ECEDF07D
:107A200000502F0803E2AA0EF1ECEDF0200E005CEE
:107A300009E2CC0E86ECEBF00050070803E27C0E66
:107A400086ECEBF0080E00C0DBFF800E00244A6ECF
:107A50004B6A000E61ECF0F00A0D020EF3CFDBFF73
:107A6000030EF4CFDBFF080EDB50006E3C0E19EC6A
:107A7000E7F0090E005C03E2500E19ECE7F000504D
:107A8000180808E2210E005C05E2020EDBCFDEFFE3
:107A9000DBCFDDFF0050240803E2280E19ECE7F0ED
:107AA00076ECE8F0CC0ED880EE54010EED5404E2F2
:107AB000CC0EDE6E010EDD6E040EDBCF4AF0050E3D
:107AC000DBCF4BF0DECF4CF0DDCF4DF04C504A5CBD
:107AD0004D504B5805E2040EDBCFDEFFDBCFDDFF60
:107AE00076ECE8F0060EEECFDBFF070EEDCFDBFF06
:107AF00011ECEBF0020EDBCF4CF0030EDBCF4DF0C0
:107B00004A504C5C4B504D5801E398D0180E070179
:107B1000335D12E1D950060FE96EDACFEAFFDE0ECF
:107B2000D880EE54000EED5407E211ECEBF0E30EBA
:107B300050ECF4F001E27BD00A0E4A6E4B6A060E5E
:107B4000DBCF3EF0070EDBCF3FF059ECE6F03EC056
:107B50009CF13AC09DF10A0E01019D03F3CF9DF106
:107B6000A06BA0C19FF1A0C19EF1CEEC36F0BBECA2
:107B700037F0060EDBCF3CF7070EDBCF3DF70701F2
:107B80003E6B3F6BA00E416E860E426E010E436E41
:107B9000446A3CC73CF03DC73DF03EC73EF03FC79E
:107BA0003FF040ECFBF038C03CF739C03DF73AC03D
:107BB0003EF73BC03FF7DFDDAFEC36F0040EDAEC0A
:107BC000E8F00701C80E356F250E346F11ECEBF0AD
:107BD000620E50ECF4F002E21C0E346F1AA803D0CF
:107BE000060E355F34272282A0DE00091BE0060E58
:107BF000DBCF0FF0070EDBCF10F0F8ECEDF033C762
:107C000000F005EC4DF0D950060FE96EDACFEAFF2F
:107C1000CC0EEE180CE1010EED1809E1012A05EC7D
:107C20004DF005D007013451D880005407E2060E0C
:107C3000DB06070E01E35CD7DB065AD70701332BBF
:107C4000BDD60C0E346FDD0E356F760E0F6E010E45
:107C5000106E040E24ECE7F023E290DE44EC4DF0CD
:107C600057EC99F0FF0E005C07E1420E7BECE6F06A
:107C70000FC029F710C02AF7450E0F180DE110505C
:107C80000BE1280E005C03E300502A0805E2450ED4
:107C90007BECE6F000C02BF70F06000E105AD9D788
:107CA000D1EC10F00201800E8B6F75EC38F0090EEC
:107CB000E15C02E2E16AE552E16EB3EFE5F0BAC1E0
:107CC00001F0BBC102F00101000E0D6F0D0E0E6F31
:107CD0000A01D751040DF3500C10036EBDEC0CF0EB
:107CE000066E0C5004E1C7ECEBF001E00686030ED3
:107CF0000C5C05E10101B651080DF35006121200AB
:107D00000A01040EDE6FDF69075005E10C5003081D
:107D100002E3E05101E1000CD2DF0A01DF6BE05128
:107D2000DF5D30E2F1ECF0F0EF50015C23E10101A6
:107D30008AECE7F0EF50025C1AE18AECE7F0EF50D2
:107D4000035C12E18AECE7F0EF50006E1F0E0014A6
:107D5000065C07E10050E00BE838E8400A01DE6FFE
:107D6000010C0D07000E0E5B0D07000E0E5B0D07DC
:107D7000000E0E5B040E01010D27000E0E230A01FA
:107D8000DF2BCDD7DF69000C0301C95107E0C1EC3F
:107D9000E8F0D9C120F1DAC121F104D052C120F1BB
:107DA00053C121F10101F10E226F020E236F120067
:107DB0001AECF0F034BC39D02CBC1AD0076A38D891
:107DC0002550100B04E10101E851400B0CE0800E3E
:107DD000081403E03050800B03E01950400B03E01F
:107DE000010E076E25D8309E21BC20D0199C1ED0D4
:107DF0002DAA08D02150400B03E02050020B16E1C1
:107E0000076A13D02150400B09E1A6ECE9F003E129
:107E1000E851400B03E0010E076E0AD82150400BD9
:107E200005E02050020B02E0076A02D822EFF0F0D2
:107E30001AECF0F00101080E9C6F150E9D6FF40E08
:107E40000F6E010E106E2150400B06E052ECE7F071
:107E500003E0B1C201F003D0BDEC0CF0016E0150A3
:107E6000E66E06ECEBF04A6E4B6A4ABE4B684A502F
:107E70000001A5ECEFF0A0EC04F001019E6F3AC008
:107E80009FF1A06BA56BA5C1A4F1A5C1A3F1A5C1EC
:107E9000A2F1A5C1A1F12150400B04E052ECE7F0A2
:107EA00001E1FBD0075017E03450400B14E10CC047
:107EB0005DF2CFC15EF2D7CA5FF25BC261F25CC213
:107EC00062F2D3C10CF0DCC1CFF160C2D7FA63C259
:107ED0005BF264C25CF20C5006E0030E0C5C31E114
:107EE0000101B6512EE09DECEFF05BC23EF05CC2AA
:107EF0003FF059ECE6F03EC0A3F14CECE6F03AC09E
:107F00003FF0FCECFDF03FC0A4F15BC24AF05CC264
:107F10004BF00A0E36ECF3F04AC0A5F120EC12F05B
:107F2000000903E1D3EC3AF002D0AFEC3AF009ECEF
:107F3000E8F023E0FEECEDF020EC12F0000918E090
:107F40001AD0040E0C5C19E297EC04F001010F0E3C
:107F5000A36FD6ECF1F0780E4A1804E14B5002E121
:107F6000100EA3270C0404E06BEC11F0010803E1F0
:107F7000D3EC3AF002D0AFEC3AF007500EE1C0DE9D
:107F8000000902E01C8A03D01CAA07D01C9A6DECE1
:107F90001AF0E66A66EC4BF0E55274ECEBF005E1A2
:107FA0001C50200B3FE007503DE1D751DE25FC0F70
:107FB000E16F190EE15D056E190EE15D04E2190E27
:107FC000D880E155056E0701EFAF07D04CECE6F025
:107FD00005C03FF00AECEBF00AD00550FE0BE8427A
:107FE0000101A36FA46B05A002D0050EA46F0C04C1
:107FF0000BE00C5003E1C7ECEBF006E0030E0C5C69
:1080000008E1C1ECEFF005E10A01E151190808E3CC
:1080100004D00A01E151190803E2AFEC3AF002D0B2
:10802000D3EC3AF0075023E034BC0AD05DC20CF028
:108030005EC2CFF15FC2D7FA61C25BF262C25CF28C
:108040000101E8970201D65101019D5D0FE1020196
:10805000D75101019E5D0AE10201D85101019F5DE6
:1080600005E10201D9510101A05D01E0E887075057
:1080700045E10201295106E0D75101019E5D02E070
:1080800005013B859CC1D5F29DC1D6F29EC1D7F2B8
:108090009FC1D8F2A0C1D9F231D0FFEC26F0016E19
:1080A0006BEC11F0026E010405E0020E015C02E0CF
:1080B000025014E0025002E00250016E01010F0E66
:1080C000A36FADECEFF003E0100E0101A32735AC78
:1080D00002D029ECF3F001040CE00ED0030E015C99
:1080E0000DE109ECE8F002E0FEECEDF0C1ECEFF0A0
:1080F00003E1D3EC3AF002D0AFEC3AF02EC100F03D
:10810000075005E03450400B02E163C100F000501D
:108110000A0801E3A8D0100E005CD5ECE8F0DCEC16
:10812000F4F001E185D04AECF5F001E181D02CDEDC
:10813000A00E0101205D7A0E2159F10E2259020E86
:10814000235918E2A00E4E6E7A0E4F6EF10E506E4D
:10815000020E516E20514E5C4A6E21514F584B6EAB
:1081600022515058235151584AC0D7F14BC0D8F131
:10817000006A15D020C14AF021C14BF022C14CF059
:1081800023C14DF0A00E4A5E7A0E4B5AF10E4C5AA6
:10819000020E4D5A4AC0D7F14BC0D8F10068590EB3
:1081A0000F6E020E106EE3AB04D0640E0F6E020E63
:1081B000106E0FC04EF010C04FF0506A516AFFECC5
:1081C000EEF04C6A4D6AEDECF1F04EC041F04FC05C
:1081D00042F050C043F051C044F040ECFBF038C0D6
:1081E00020F139C021F13AC022F13BC023F1010155
:1081F00021C120F122C121F123C122F1236B98EC8E
:1082000097F00101A26BA2C1A1F104C13CF504C128
:10821000A3F105390F0B05013D6F0101A46F0F0E8E
:10822000051505013E6F0101A56F00C03FF514D093
:1082300082EC08F00101A26BA2C1A1F1A0ECF3F065
:10824000A36F050EEB50A46FA56B006AEF50010BF6
:1082500001E0006882EC08F0005003E0D3EC3AF053
:1082600002D0AFEC3AF09CC1A1F19DC1A2F19EC138
:10827000A3F19FC1A4F1A0C1A5F1075007E12050CF
:10828000020B0AE02150400B0AE106D03450400BAB
:1082900003E185ECE9F003E032ECE8F002D0D6EC43
:1082A000EAF00101E351200B07E0075003E02E51F3
:1082B000635D02E1020E9C5FE8BD27D01A9E075065
:1082C00004E02E50400B01E11A8E8DECE9F003E042
:1082D000AFEC3AF002D0D3EC3AF0075016E00101CF
:1082E0003A51080B12E03E51100B0FE10A0E9C6F41
:1082F000330E9D6F1E0E9E6FA06BA0C19FF17AA7DB
:1083000004D0050E9C6F370E9D6F01017A51080B4A
:108310002CE02150400B29E1016A3A51080B0BE097
:108320003E51100B08E08D51400B05E0E851080B61
:1083300002E1020E016E076A430E4FECEBF0010EF4
:10834000016EA6ECE9F003E1E851400B07E08D5126
:10835000400B03E0E851080B01E0016A010E076ED3
:10836000430E4FECEBF0DF50076E01017AA71DD0F2
:108370009CC1E6FFFDECE8F0016E9DC1E6FFFDEC5F
:10838000E8F0026E9EC1E6FFFDECE8F0036E0A0E17
:1083900001019F03F350A025E66EFDECE8F001011A
:1083A000076F460EE66ED9D8D4D09D514A6E4B6AFF
:1083B0000A0EDEECF3F001019C510A0D56ECE8F0D8
:1083C000010E0F26000E1022F8ECEDF044EC4DF0FB
:1083D0000A6A270E005C06E1460E0F1803E11050F2
:1083E00001E1002A64ECE8F0EF50005C0AE02A505A
:1083F000040B07E1040EA4ECECF064ECE8F000C020
:10840000EFFF2A94CEEC36F02EAA0DD008AE03D0A2
:10841000BBEC37F008D0E7C2E6FF010EE66E1FECBA
:1084200038F0E552E5529CC14AF04B6A4C6A4D6AFD
:10843000400E416E420E426E0F0E436E0DECE8F0A0
:108440009DC14EF04F6A506A516A100E416E270E60
:10845000426E436A446A4EC03CF04FC03DF050C08B
:108460003EF051C03FF040ECFBF038C04EF039C058
:108470004FF03AC050F03BC051F0F4ECEBF09EC12D
:1084800052F0536A546A556A640E416E426A436AF6
:10849000446A52C03CF053C03DF054C03EF055C059
:1084A0003FF040ECFBF038C052F039C053F03AC016
:1084B00054F03BC055F052504A2653504B22545072
:1084C0004C2255504D229FC156F0576A586A596A3E
:1084D0000A0E416E426A436A446A56C03CF057C075
:1084E0003DF058C03EF059C03FF040ECFBF038C0C2
:1084F00056F039C057F03AC058F03BC059F05650CA
:108500004A2657504B2258504C2259504D22A0C158
:108510005AF05B6A5C6A5D6A4A505A2407013C6FF4
:108520004B505B203D6F4C505C203E6F4D505D20AA
:108530003F6FBBEC3BF0AFEC36F002018B51CDEC62
:10854000ECF008E14B5006E125BC04D0E66A67EC8C
:108550003BF0E552E552B3EFE5F0D9CFE6FFE1CFCE
:10856000D9FF02010D6B15EC7AF001010101905168
:10857000010B07E001010101E851040B02E1300E9B
:10858000C66E0C0E07244A6EF00E8C144A108C6EC8
:1085900081EC5EF08A9AE3EC08F0FE0EDBCFE6FF9A
:1085A00004EC7AF0E552FE0EDB50006EFE0EDB505E
:1085B000530807E00150E66E04EC7AF0E5520150F2
:1085C0000026FE0EDB50460804E0FE0EDB50560887
:1085D00015E10250E66E04EC7AF0E5520350E66EC7
:1085E00004EC7AF0E55207C1E6FF04EC7AF0E552BC
:1085F00000500224032401010725006EFF0E000233
:10860000F350E66E04EC7AF0E552FE0EDB505308B0
:1086100006E1C950006EE66A04EC7AF0E5528C88F7
:108620000000000000000000310EC66E8A8AF00EC5
:108630008C1611EC7AF0E552E7CFD9FF1200D9CFB2
:10864000E6FFE1CFD9FFB9C19CF1BAC19DF1BBC131
:108650009EF1BCC19FF1BDC1A0F10101A66BFE0E50
:10866000DB500A0807E22A96FE0EDBCFE6FFD1ECCC
:1086700034F0E5520101006B800E01011615036E06
:10868000800E01011315026E010EEA6E9C5105D891
:108690009D5103D89E5101D814D0076B066F0A0E66
:1086A000065DD8A003D0066F072BF9D70051110F34
:1086B000E96E0751EF6EE92A0651EF6E002B002B91
:1086C000000C04D8E552E7CFD9FF12009FC117F183
:1086D000A0C118F10101A65105E10A0E9C5D02E25C
:1086E000100E116F0701EFBB03D00101100E186FC0
:1086F0000701EFAD05D00101100E176F17C118F17A
:108700001EBC03D00101138F03D0025001011313CB
:108710005FEC0BF0000903E10101168F03D0035059
:1087200001011613A65109081AE20201495117E086
:1087300071EC94F00101020E006F9CC100F05BEC43
:1087400097F0A6C100F00101006B5BEC97F0010E01
:10875000E66EE66A7FEC09F0E552E552120001018F
:10876000A65118E00701EF51200B14E1298C17C125
:1087700018F116C117F115C116F114C115F113C185
:1087800014F112C113F111C112F13DECF3F03BC031
:1087900011F11200299C1200D9CFE6FFE1CFD9FFD9
:1087A000020EE126010EA6C1DBFF2EAC0FD02EC1BA
:1087B000DFFFEFC7F0F7B9C19CF1BAC19DF1BBC1B2
:1087C0009EF1BCC19FF1BDC1A0F115D063C1DFFF17
:1087D0000101D351EA6AE90FE96E070EEA22EFCFF1
:1087E000F0F7BEC19CF1BFC19DF1C0C19EF1C1C1F6
:1087F0009FF1C2C1A0F10101A66BDF500A0806E299
:108800002A96DFCFE6FFD1EC34F0E5520101016B8F
:10881000800E01011E15026E010EEA6E9C5105D8F4
:108820009D5103D89E5101D816D0076B066F0A0ED2
:10883000065DD8A003D0066F072BF9D70151190F99
:10884000E96E0751300FEF6EE92A0651300FEF6ED7
:10885000012B012B000C010EDBCFE6FF0BD8E552FC
:10886000020EE15C02E2E16AE552E16EE552E7CF19
:10887000D9FF1200AEECE5F0300E01019F251F6F0D
:10888000A65105E10A0E9C5D02E2200E196F070158
:10889000F0AD03D00101200E1F6F01011B8F6DECA5
:1088A0000BF0000903E101011E8F03D0025001010A
:1088B0001E13A65116E00701F051200B12E11EC154
:1088C0001FF11DC11EF11CC11DF11BC11CF11AC1FC
:1088D0001BF119C11AF13DECF3F03B50300F0101CF
:1088E000196FA6C1A7F1FE0EDBCFA6F1B3EFE5F03D
:1088F000E66A08D8E55231A204D0010EE66E02D82D
:10890000E5521200AEECE5F0050EE126FE0EDB505E
:108910000CE1C3C1DFFF010EC4C1DBFF049020B036
:108920000480040E2EC1DBFF0ED0C8C1DFFF010E94
:10893000C9C1DBFF049031B20480030E15C2DBFF16
:10894000040E63C1DBFF020EDB6A0450010B01E180
:1089500004D11C0EDF5C01E300D1100EF36E040E97
:10896000DBCFF4FFF350F45C01E3F7D00E0EDF5CD5
:1089700001E383D0070EDF5C48E2030EDF5C16E202
:10898000020EDF5C0DE2DF5005E0460EE4ECE5F0A0
:1089900001E3E3D0800E1FECE7F00201400EBCD0F3
:1089A000010EDB500A0801E3D8D00BD0050EDF5CC6
:1089B00015E2030EDF5C0BE11E0EE4ECE5F001E3D3
:1089C000CCD0C00E1FECE7F00201800EA5D0010E46
:1089D000DB50140801E3C1D0100E23D00201080EB1
:1089E000156F050EDF5C0AE1190EE4ECE5F00BE310
:1089F000010EDB50320801E3B0D005D05A0EE4EC92
:108A0000E5F001E3AAD0100EA6D0090EDF5C16E255
:108A1000070EDF5C09E1010EDB50280801E39DD061
:108A2000300E1FECE7F007D0300E1FECE7F0280EF9
:108A3000E4ECE5F032E20201080E6ED00201200EF5
:108A4000156F090EDF5C07E1550EE4ECE5F001E37C
:108A500084D0300E80D00D0EDF5C09E20A0EDF5CA0
:108A60000AE1010EDB50140801E377D004D03C0E7C
:108A7000E4ECE5F072E2080E6ED0160EDF5C37E231
:108A8000120EDF5C18E20E0EDF5C0AE1010EDB5015
:108A90003C0863E20C0E1FECE7F00201200E3CD014
:108AA000110EDF5C04E3460EE4ECE5F056E20C0E3A
:108AB0001FECE7F029D00201100E156F120EDF5CDB
:108AC00005E1010EDB50280848E20FD0130EDF5CF1
:108AD0000CE0140EDF5C05E15A0EE4ECE5F03DE23B
:108AE00004D0010EDB50320838E2010E34D0180EEB
:108AF000DF5C14E2160EDF5C0AE1010E1FECE7F00A
:108B00000A0EE4ECE5F006E20201100E05D0030EB9
:108B10001FECE7F00201040E156F1FD00201040ED6
:108B2000156F180EDF5C05E1320EE4ECE5F015E29E
:108B30000BD0190EDF5C05E1010EDB5032080DE2AF
:108B400003D01A0EDF5C02E1030E05D0460EE4EC02
:108B5000E5F003E2030E1FECE7F0FE0EDB50EA6ADD
:108B6000130FE96E020EEA22020EDBCFEFFFFE0EBC
:108B7000DB5003E0030EDBCF15F2050EE15C02E2F1
:108B8000E16AE552E16EB3EFE5F007010A6B1F0EF3
:108B90000B17116B0D6B0DC70CF7030E06171F0E8D
:108BA0000717096B09C708F72EC100F0AAECE9F016
:108BB00002E20FC100F00201135103E02050010B4B
:108BC00047E100500A0A3FE0030A39E0010A35E0B4
:108BD0000F0A2DE0010A27E0030A20E0010A1BE04A
:108BE000060A14E0010A0FE0020A08E0010A36E171
:108BF0000701118D11830A890B8B30D00701118F6A
:108C000011830A892BD007010B8D02D00701118334
:108C100011870A8B23D007010B8D11830701118364
:108C2000118B0A8D1BD007011189118304D0070114
:108C3000118311890B8F0A8F11D007010B8F070148
:108C400011850A870BD00701118311850A8506D08B
:108C5000E66A03EC15F0E55215C211F72EC100F0DB
:108C600000500A0802E20FC100F0010162A707D01C
:108C700063C100F000500A0802E210C100F00201D6
:108C8000145103E03150020B35E100500A0A2FE085
:108C9000030A2AE0010A26E00E0A21E0010A1DE08B
:108CA000020A18E0010A14E0060A0FE0010A0BE0CC
:108CB000020A06E0010A23E107010689078B1FD09B
:108CC000070106891CD00701078D0701068B17D005
:108CD0000701078D0701068D12D00701078F0701D5
:108CE000068F0DD00701078F0701068708D00701FF
:108CF000068505D0010EE66E03EC15F0E552010184
:108D00003EB905D0FC0E07010613E00E071303EF72
:108D10000CF033EC0EF02C50040B08E00050D7ECB4
:108D2000E6F0EF50020B02E126EC0EF0258A12006D
:108D30000FECF0F0830E0A6E0A0EE66E01010F03CF
:108D4000F350E66E740EE66E020E17ECE6F0DE0EE1
:108D500029ECE7F00050DF6EFE0E35ECF5F0010176
:108D6000E49D2F9EB90E005C05E1FF0E0201745DCB
:108D700001E02F8EA30EDF5C02E10101E48DE552DC
:108D8000B3EFE5F01AECF0F0075034E11950010BA5
:108D900031E1CEDF01015951080B03E12E510908E1
:108DA0000EE229EC05F0FF0805E1800EE66E3BECD3
:108DB00005F0E55229EC05F001014B6F08D0FF0EDC
:108DC0008F5D03E1320E8F6F02D08FC14BF1E2EC69
:108DD000F3F02B8483EC28F035EC23F02CA60AD09A
:108DE000E66A0EECC8F0E5520701169F12B0168F26
:108DF000D1ECC6F0C4ECECF025A808D038EC0DF0AE
:108E000025A804D0010E076ED1EC10F0076AD1EC52
:108E100010F022EFF0F00FECF0F0FD0EDB50100D33
:108E2000F350DF6E010E0A6E0201680EC36FFD0E75
:108E3000DB500A080AE2020E0A6E690EC36FFD0ECD
:108E4000DB50F00F100DF350DF6EE8ECEFF002E0B6
:108E5000AAECF1F0DF50E552B3EFE5F00201B351B7
:108E600003E0B351330802E20D0EB36FB451A1EC2D
:108E7000E6F005E2E4ECE8F002E21E0EB46FB5BFE6
:108E8000B56B120013ECF0F0E8ECEFF01BE0AAEC8D
:108E9000F1F00F0E26ECF1F00A0E005C07E1010183
:108EA000E251010B03E00A6A000E5AD200C02EF113
:108EB00001018D51100B06E00A0E1DECE6F002E2F6
:108EC000FE0EDB682EC10FF10101E5A506D0E39B84
:108ED000450EE66ECDEC08F0E55202018C6B010107
:108EE000E59533EC0EF0AAECE9F022E2100E2E5DCF
:108EF000E6ECF3F072EC05F0F6ECF0F011E07AEC51
:108F0000F1F001010F6FEF380F0B02018C6F80EC55
:108F1000E6F0800B03E00101E585E38DFADE08D081
:108F2000FE0EDB680101090E0F6F0FC12EF1268EB8
:108F30009EECF0F0100EE0ECF1F00F0E0101CD15FB
:108F40000C6ECD390F0BD36FD351060802E20CC063
:108F5000D3F10C0401E1CE91020E0C5C01E1CE8153
:108F600049ECF4F0B66F62B704D02EC163F10FC1C3
:108F700010F163C110F163510A0817E2100E635D2E
:108F8000E6ECF3F0F6ECF0F005E07AECF1F001013C
:108F9000106F08D0FE0EDB680101090E106F10C1C2
:108FA00063F1268E63C100F002D0FDECEBF00050BF
:108FB0000101635D03E12E51635D10E02DECF2F0E1
:108FC000050EE66EDF2401ECEAF017ECE6F00A0E7F
:108FD00026ECF1F000380F0B0101D36F040E4BECBF
:108FE000EFF0DB0EE66E010E17ECE6F09EECF0F013
:108FF000E8ECEFF003E1C3C20AF002D0100EDF2666
:10900000100EE4ECF4F0ACECF2F0E8ECEFF05CE025
:109010002EC1E6FFE66860ECE7F00B0E26ECF1F0FF
:10902000030E0C5C09E01F0E0101CE17E00E0014C8
:10903000CE1349ECF4F0B66F0050046E0101CE97E8
:109040000450080B01E0CE870C0E26ECF1F0440E24
:109050000101CF17BB0E0014CF13ECECEFF0070E9D
:109060000101D017F80E0014D013ECECEFF00A0E4B
:109070000101D117F50E0014D113C3C20AF00D0E71
:10908000E66E030EDF24E66EB60EE66E020E17ECF9
:10909000E6F02DECF2F00C0E26ECF1F0440E01019E
:1090A000DC17BB0E0014DC13ECECEFF0070E010133
:1090B000DD17F80E0014DD13ECECEFF00A0E0101E1
:1090C000DE17F50E0014DE130201BCBFBC6B0A6A8A
:1090D000C3C107F5C4C108F5C5C109F5C6C10AF584
:1090E000C7C10BF5C8C10CF5C9C10DF5CAC10EF554
:1090F000CBC10FF5CCC110F519B42DD01394139634
:10910000139A209201013B51020B1CE052ECE7F054
:1091100019E10101D051010B04E034ECBAF000096F
:1091200011E10101D051010B05E02E51635D02E117
:10913000138A20821396D0B313861394D0A509D036
:10914000138407D0A8ECEDF00101DD95DD93D095F7
:10915000D09341ECC1F0AAECE9F01AE2680E0F25B9
:10916000EBECF2F000500101C35D016E01AE03D0E3
:10917000C351005C016E015003080AE2050EEFECDA
:10918000EFF0C30EE66E010E9CECE6F000C0C3F1FA
:10919000010163510A081AE2680E1025EBECF2F0A7
:1091A00000500101C85D026E02AE03D0C851005CE0
:1091B000026E025003080AE2050EEFECEFF0C80E53
:1091C000E66E010E9CECE6F000C0C8F1320EFFEC3A
:1091D000E7F0300EFFECE7F0C0ECECF0BBEC2CF06D
:1091E00054EC0EF0139C01013EB1138C139E3EB360
:1091F000138E8AEC80F0139801013EB913882CA4D9
:10920000D09F1294D0BF12840701109B12A4108B20
:109210000201BD51030802E3BD5102E1020EBD6F20
:1092200053EC27F02CB602D00101CF9F1290010120
:10923000CFBF12801292CFAF1282B3EC09F00101BE
:109240005A51800B05E02C50040B02E026EC0EF086
:10925000660E0A6E080E01012E03F32829ECE7F0D2
:1092600000C042F5FF0E005C02E10501426B010601
:1092700044EC4DF0FF0E005C01E1006A7F0E00142B
:109280000501406F01015A51100B04E1E251200B1E
:1092900001E1CF9B080E6303F350050F29ECE7F0C3
:1092A00000C043F5FF0E005C02E10501436B0106BF
:1092B00044EC4DF0FF0E005C01E1006A7F0E0014EB
:1092C0000501416F01015A51100B0AE1E251200BD7
:1092D00007E16251080B03E01C50080B01E0DE912E
:1092E0000A6A010E07C0DBFF3EA905D0076EE7EC56
:1092F00068F081EC68F0076AE7EC68F081EC68F0F0
:1093000015A403D00501FA0E446F010EDB50076E61
:109310006A0E01010F250A6EF00E29ECE7F0FF0E30
:10932000005C01E1006A00C0E0FA040E0002F350A4
:10933000E66EE66A000EE66E0D0E17ECE6F00A6ABF
:1093400021DDACEC0CF0C0ECEAF0CBECEAF0010172
:10935000276B1EBC04D00701D36BBBECE9F0010EF8
:1093600070ECEBF002E2E16AE552E16E4A50B3EFD5
:10937000E5F00FECF0F00B0E01012E5D0BE2C4C125
:10938000E6FFC3C1E6FFEAECF3F0005001012E5DF9
:1093900001E0B1D00B0E635D07E2FDECEBF0005095
:1093A0000101635D01E0A7D00A0E2E5D02E24BC110
:1093B0008FF19EECF0F040EC27F00101CF9F12B04E
:1093C000CF8FD09F12B4D08F3BA30DD0F80ED01703
:1093D000D09120B2D081D09313B6D083D09513B45E
:1093E000D0859BEC55F02EC1D2F1B3ECF1F0050E17
:1093F00059ECEBF0E4ECF4F0E8ECE5F005ECEEF021
:109400000C1018ECEAF0050EE66ECE0EE66E010EBC
:109410004BECEFF0E8ECE5F07AECEAF018E02DEC3C
:10942000F2F00A0E26ECF1F00F0E001605ECEEF04D
:10943000001018ECEAF07AECEAF009E0040EE66EAF
:10944000DB0EE66E010E4BECEFF0E8ECE5F0050EFE
:1094500001ECEAF0E66E050EDF24CEECF0F01DBA6A
:1094600045D09EECF0F001015951080B03E12E515B
:10947000090805E24BC1E6FF3BEC05F0E5522CEC98
:10948000C6F00101CF51800B01E0010E39ECECF088
:109490003DC1EFFFE8ECEFF003E1C3C20AF002D0F8
:1094A000100EDF260CECEEF0DFCFE6FFE8ECE5F087
:1094B0000A6AC0EC15F0660E0A6E080E01012E0352
:1094C000F350016E40C500F0A0DA012A42C500F059
:1094D0009CDA080E01016303F350040F016E41C5CD
:1094E00000F093DA012A43C500F08FDA0A6A43ECF0
:1094F000F3F00201306BE552B3EFE5F00FECF0F062
:109500007F0EDF6EF2ECE8F007E02D50400B04E137
:109510002D50800B01E1DF060F0E06010D17DF1C39
:109520000E17E552B3EFE5F006010D910E9F0F996E
:10953000EE0E101712171399149112009CECF4F010
:10954000DBCFE6FF12EC14F0E552E71803E006016A
:109550000D8F02D006010D8D01013FA502D006013D
:109560000E8101018DA102D006010E87B3EFE5F057
:109570001A9E0050050A01E174D0010A5CE0070A56
:109580002AE0010A23E0030A1FE0010A01E01200B9
:1095900006010D8B8DECE9F002E0000E01D0010E0A
:1095A0004A6EC7ECEBF001E0010E4A1802E006013A
:1095B0000D890601F051010801E20E83010191AD10
:1095C00064D006010E871200E66A02D0010EE66E34
:1095D000B5DFE552120006010E898DECE9F002E0DC
:1095E000000E01D0010E90ECEBF002E006010D89B7
:1095F0000101B65103E0030EB65D02E106010D79EB
:10960000D1ECEFF002E006010E8333A00ED08DEC1A
:10961000E9F002E0000E01D0010E90ECEBF003E067
:1096200006010D8D02D006010D8F01013FA72DD03F
:1096300006010E81120006010E8B0101D1A725D073
:10964000D1A303D006010D8D02D006010D8F0101BB
:109650009151080B03E10201515117E006010E83FD
:10966000120006010E8D0201B551040B04E04D51AC
:1096700002E106010E830201B5A102D006010E87A8
:109680000201B5A302D006010E851200800E081457
:1096900005E02150010B02E10C5002D0FFEC26F056
:1096A000006E2CDFB8EF4AF0060150510A01DA9142
:1096B000040B01E0DA8168ECE6F007E006015251A4
:1096C00001015999800B01E059891200AEECE5F0D7
:1096D0000C50006EFFEC26F0056E6BEC11F0046E82
:1096E000045006E00450006E21BE02D00450056E06
:1096F0001B0E002443ECE6F0016E210E052443EC22
:10970000E6F0026E005005E1C7ECEBF002E0220E3D
:10971000016E055005E1C7ECEBF002E0420E026E6F
:10972000030E005C09E1045007E1C1ECEFF004E036
:10973000200E016E400E026E0150C6ECE5F007509F
:1097400006E1FE0EDB5003E00250C6ECE5F0040E2D
:10975000005C0DE10101D1A707D0D151020B02E05D
:10976000270E03D0280E01D0240EC6ECE5F0B3EF8F
:10977000E5F00FECF0F034B886D0075002E1B9EC18
:1097800011F00A01DA5106015099010B01E05089EC
:109790000A01DA5106015095010B01E050850A01DA
:1097A000DA510601010B02E0509B01D0508B0A01F7
:1097B000DA510601010B02E0509701D050878EEC80
:1097C000F1F006E10601508D528F5291509F21D049
:1097D000030E005C0EE10601508D509F93EC11F0DA
:1097E000000903E00601509D508F0601528F5291EF
:1097F00010D00601509D508F529F010159A902D0EF
:109800000601528F06015291010159B902D0060199
:1098100052812150800B14E11550100B11E01550AE
:10982000200B0EE10C5009E0030E0C5C06E0050E67
:109830000C5C03E0F2ECE8F003E01598A4EC6AF0AD
:10984000030E0C5C03E0050E0C5C02E160EC68F0BA
:1098500014900C5004E1149001018DB51480030E96
:109860000C5C04E11490010191B51480149A14A0C9
:10987000148A54EC0DF0075004E18AEC80F0E6EC19
:109880001DF0BBEC2CF03450100B18E1010191518C
:10989000400B14E02150800B11E107500FE1FFEC69
:1098A00026F0010804E0FFEC26F0020807E10C5066
:1098B000DF6E0C6A0FEC1AF0DF500C6EFAEC1AF047
:1098C0002682D8EC3EF0010EE66E00DFE55221EC78
:1098D0001BF0AFEC23F034B848D0FFEC1DF0A4EC43
:1098E0006AF0F0EC11F04CEC26F01D983590010177
:1098F000E7BB02D020EC09F0050E0C5C03E0E1ECC4
:10990000EFF002E18DEC0CF01AEC25F007502DE1A0
:10991000BCEC25F0D9EC22F022EC1EF0D7EC16F0CE
:1099200068ECE6F002E0C0EC23F0B5EC16F034A4ED
:1099300002D050EC1EF01FECE8F058C1E6FFE66ADA
:10994000EFECF3F0016E01016281005006E0030EBE
:10995000005C04E1B651010801E26291F7EC13F0FA
:10996000050E005C02E145EC09F03498E552B3EFD6
:10997000E5F08E9400000000030EE66E04EC7AF031
:10998000E552040E0A5CE66E04EC7AF0E5520150F2
:10999000E66E04EC7AF0E55274ECFDF0006E000027
:1099A0008E841200D9CFE6FFE1CFD9FF8E9400005C
:1099B0000000060EE66E04EC7AF0E5528E8400009C
:1099C000000000008E9400000000020EE66E04EC21
:1099D0007AF0E552040E0A5CE66E04EC7AF0E55289
:1099E0000150E66E04EC7AF0E552FE0EDBCFE6FFA6
:1099F00004EC7AF0E5528E84040EE66E46ECFDF03F
:109A0000E552E552E7CFD9FF120013ECF0F0005019
:109A1000DF6E010EDB6A38D8DF50005C2DE0040EEB
:109A20000A5C16E2F29EA1980A50AA6E0150A96E35
:109A3000DF50A86EA69EA69CA684550EA76EAA0E01
:109A4000A76EA682F28E040EDAECE8F0A69414D08B
:109A50008D8A010EDB2ADFCFE6FFA4DFE55289DF26
:109A6000DF50005C02E041EC0EF0DF50005C04E0EF
:109A7000050EE4ECE5F0EDE3020EE15C02E2E16AE2
:109A8000E552E16EB3EFE5F0CBECF3F0040E0A5CC7
:109A90000AE20A50AA6E0150A96EA69EA69CA68054
:109AA000A850006E13D08D8A010EDB2A62DF0050B1
:109AB000DF6E5FDF0050DF5C02E041EC0EF0005033
:109AC000DF5C04E0050EE4ECE5F0EEE3020EE15CA1
:109AD00002E2E16AE552E16EB3EFE5F0AEECE5F0EB
:109AE00013ECEEF011E0FC0ECBECEEF029ECE7F01D
:109AF000FD0EDBCFE9FFDB2AFE0EDBCFEAFF01E341
:109B0000DB2A00C0EFFFECD7B3EFE5F0AEECE5F0F9
:109B100013ECEEF011E0FE0ECBECEEF0016EFC0E5D
:109B2000DBCFE9FFDB2AFD0EDBCFEAFF01E3DB2A17
:109B3000EF5018ECEAF0ECD7B3EFE5F0D9CFE6FF41
:109B4000E1CFD9FFE6528E848D9A00000000060E08
:109B5000E66E04EC7AF0E5528D8A00000000000009
:109B60008D9A00000000D80EE66E04EC7AF0E55203
:109B7000D7C7E6FF04EC7AF0E552E66A04EC7AF027
:109B8000E552E66A04EC7AF0E5528D8ADF6A1E0E31
:109B9000DF5C07E2640EE66E36EC29F0E552DF2A60
:109BA000F6D7E552E552E7CFD9FF1200D9CFE6FF4D
:109BB000E1CFD9FF35AE33D08E848D9A00000000FE
:109BC000030EE66E04EC7AF0E552D7C7E6FF04EC2C
:109BD0007AF0E552FC0EDBCFE6FF04EC7AF0E552BA
:109BE000FB0EDBCFE6FF04EC7AF0E552FA0EDBCF9A
:109BF000F3FFDB06F35000090FE074ECFDF0006E9C
:109C0000FD0EDBCFE9FFDB2AFE0EDBCFEAFF01E32F
:109C1000DB2A00C0EFFFEAD700008D8AC69EE5521E
:109C2000E7CFD9FF120013ECF0F0DF6ADF2AFA0E5B
:109C3000DBCFE6FFC5ECF4F01AECEEF0FA0EDBCF6A
:109C4000E6FF96ECE7F0AC0EE66E030EE66E1AEC5D
:109C5000EEF0010EDB6AFA0EDB50E4ECE5F017E201
:109C6000010EDB50E76E2CECE9F0E750CAECF0F0A7
:109C7000EFCF4AF0010EDB50EA6AAC0FE96E030E3B
:109C8000EA22EF504A5C03E1010EDB2AE4D71EEC26
:109C9000EEF002E041EC0EF01EECEEF003E00A0EF6
:109CA000DF5CC4E30A0EDF5C02E3000E01D0010EAC
:109CB00070ECEBF002E2E16AE552E16E4A50B3EF7C
:109CC000E5F0D9CFE6FFE1CFD9FF35AE46D08E849F
:109CD0008D9A00000000060EE66E04EC7AF0E55264
:109CE0008D8A0000000000008D9A00000000020E26
:109CF000E66E04EC7AF0E552D7C7E6FF04EC7AF0A2
:109D0000E552FE0EDBCFE6FF04EC7AF0E552FD0EE5
:109D1000DBCFE6FF04EC7AF0E552FA0EDBCFF3FF7F
:109D2000DB06F350000911E0FB0EDBCFE9FFDB2A75
:109D3000FC0EDBCFEAFF01E3DB2AEF50006E0050A0
:109D4000E66E04EC7AF0E552E8D700008D8AC69EF4
:109D5000050EE66E36EC29F0E552E552E7CFD9FF65
:109D600012000701D76B020EE66EE66AE668D70EB0
:109D7000E66E010E91ECE8F00101D71D01E1D81D5E
:109D800002E018ECEFF0120013ECF0F0358E070152
:109D9000D76BDF6ADF2A100EE66EE66AE668000E11
:109DA000E66E090E91ECE8F045ECEBF0DB5005E0D7
:109DB0000901001D09E1011D07E1010EDB6A41EC0B
:109DC0000EF0010EDAECE8F0010EDB5003E1050EB7
:109DD000DF5CE0E3DF50040802E2010E6DD0090110
:109DE000001D04E1011D02E1020E66D002510425AE
:109DF0000F6E03510521106E000E0F5C400E1058BF
:109E000002E2030E59D006C9D7F107C9D8F1010102
:109E1000000ED75D380ED85902E2050E4DD0400E27
:109E200002010F24AD6F000E1020AE6FAD51010185
:109E3000D7250F6E0201AE510101D821106E08C95D
:109E4000D7F109C9D8F1800ED75D030ED85902E2C7
:109E5000060E32D00FC0AFF210C0B0F20201AF5107
:109E60000101D7250F6E0201B0510101D821106EFA
:109E70000AC9D7F10BC9D8F1BC0ED880D755020E4C
:109E8000D8550FE20FC0A5F310C0A6F30301A551EA
:109E90000101D7250301A76FA6510101D8210301B4
:109EA000A86F0EC9D7F10FC9D8F10101D751D81148
:109EB00002E1040E01D0000E70ECEBF002E2E16A68
:109EC000E552E16E4A50B3EFE5F0AEECE5F01F0E5F
:109ED0000501115D0DE2112B1351EA6A150FE96EB0
:109EE000050EAFECF3F0132B13511F0801E2136BB7
:109EF000B3EFE5F0AEECE5F0FDECECF062E10F6AFB
:109F0000106AFE0EDB500D0803E11F0E0F6E106A83
:109F1000FE0EDB500A0803E11D0E0F6E106AFE0EE6
:109F2000DB50090803E1EF0E0F6E106AFE0EDB50E6
:109F3000080803E10F68020E106EFE0EDB507F086A
:109F400004E1B50E0F6E030E106EFE0EDB501F08FF
:109F50002EE27F0E1DECE6F02AE2410E1DECE6F04B
:109F60000EE3FE0EDB505A080AE3200E4A6EFE0E88
:109F7000DBCFE7FF4A50E726FE0EE7CFDBFF020EFE
:109F8000E66E7A0E0301A7254C6E010EA8214D6ED8
:109F9000FE0EDB50E00FE82444ECF0F00F0EE66E0E
:109FA000000EE66E40DE4E6E050EE15E4E500F5026
:109FB00010102CE010C0E6FF88DFE5520FC0E6FF6E
:109FC00023D0FE0EDB504B6A7A0F4A6E060E61EC10
:109FD000F0F0046E2450040B09E10450800B06E0FD
:109FE0006F0EE66E72DFE55224840BD02450040B12
:109FF00008E00450800B05E17F0EE66E66DFE55257
:10A000002494049E0450E66E60DFE552B3EFE5F061
:10A010000FECF0F0800E1DECE6F003E3200E85EC73
:10A02000E8F00201050E3D6FFE0EDB50740811E1F1
:10A03000010E3D6FFDECECF008E105011151FC0B48
:10A04000E842E842020F02013D6F0501006B1E82EB
:10A050002BD0FE0EDB5028E0DF6A150EDF5C11E22C
:10A0600049ECF3F00BE1DF2A9DECE8F050ECEFF067
:10A07000DF2A9DECE8F050ECEFF003D0030EDF2672
:10A08000ECD7150EDF5C04E14FECE6F033DFE55270
:10A09000200E1DECE6F003E2200E85ECE8F04FEC1C
:10A0A000E6F01FEC8BF0E552E552B3EFE5F013EC70
:10A0B000F0F024A012D01EB009D00201685D1CE3AC
:10A0C0000701016B026B68C269F216D00201682BAE
:10A0D000685180081BE2800E18D01EA010D0070E19
:10A0E0000701015D09E2012B02910243020E020108
:10A0F000685D02E30701028F0201010E06D0020132
:10A10000682B6851800802E2800E686F1E9024B0B0
:10A110001E802450010B03E1020E685D04E01E5016
:10A12000020B01E189D01EA204D00701CC0E026F00
:10A130000FD0070102910243028F070ED88001550C
:10A14000016E01500106000903E002910243F9D7B4
:10A1500000C70AF00201695107081DE269513F0872
:10A1600002E23F0E696FB6ECECF006E0200E0CEC5C
:10A17000E7F0200E50ECEFF0A9ECEFF00CE0070157
:10A18000035109E0800E02016925006E03C701F04A
:10A19000070103073ADC780E0701025D18E22A8AFC
:10A1A00002C7E6FF67EC04F0E552DF6EDF500EE019
:10A1B000B6ECECF00BE03D5104E0DFCFE6FF28DF2A
:10A1C00004D0DFCFE6FF1FEC8BF0E5522A9A0101A5
:10A1D000B2A732D00701035105E002C700F003C760
:10A1E00001F013DC0701035106E01E50020B03E1EE
:10A1F0001C0E025D1EE103510BE01C0E025D08E126
:10A20000CC0E006E030703C701F005EC4DF01E8273
:10A210000101B29755EC81F0350E165C03E1410E59
:10A22000DBECE5F0259224BC25820201010E3D6F96
:10A2300001D003070701026B0A6A020EE15C02E229
:10A24000E16AE552E16EB3EFE5F006015051545D6D
:10A2500003E15251555D1DE050C654F652C655F605
:10A2600076ECEAF009E1050E0B5C06E1E66804EC29
:10A270007AF0E552E66807D052C6E6FF04EC7AF0C1
:10A28000E55250C6E6FF04EC7AF0E5528E8E8E8ED3
:10A290008E9E2850020B2AE02A50010B27E106016E
:10A2A0005051515D03E15251535D20E0510E28ECB5
:10A2B000E6F006015051515D09E050C651F6310EED
:10A2C00028ECE6F050C600F04BEC99F00601525134
:10A2D000535D09E052C653F6320E28ECE6F052C642
:10A2E00000F04BEC99F03B0E28ECE6F01200000079
:10A2F00012000601DE6BF00E8C140609CFECEBF0B9
:10A3000084AE02D00601DE81F00E8C140409CFEC7D
:10A31000EBF084AE02D00601DE83F00E8C14070948
:10A32000CFECEBF084AE02D00601DE85F00E8C148B
:10A330000509CFECEBF084AE02D00601DE87F00E0B
:10A340008C140209CFECEBF084AE02D00601DE895A
:10A35000F00E8C140109CFECEBF084AE02D00601B4
:10A36000DE8BF00E8C140309CFECEBF084AE02D040
:10A370000601DE8DF00E8C14CFECEBF084AE02D033
:10A380000601DE8FF00E8C161200F4ECF3F01DECDB
:10A39000E6F008E3FE0EDBCFE6FFFD0E38ECEDF055
:10A3A0000AE207D0FD0EDBCFE6FFFE0E38ECEDF043
:10A3B00002E2010E01D0000EB3EFE5F013ECF0F075
:10A3C0002FB26CD0DF6A080EDF5C36E2F00E8C1420
:10A3D000DF108C6EB70EB1ECE6F000C06FF707012E
:10A3E0006F51190827E2FE0EDB5004E1F00E8C16C7
:10A3F000010E57D0B70EB1ECE6F000C070F70701C0
:10A400007051190817E2B70EB1ECE6F000C071F711
:10A41000030EE66E70C7E6FF6FC7E6FF9DECE7F040
:10A4200009E0030EE66E71C7E6FF70C7E6FF9DEC1C
:10A43000E7F002E1DF2AC7D7F00E8C16080EDF5CCA
:10A440002AE2DE52010EDD6E080EE4ECE5F010E2C9
:10A45000070EE66E010EDB503B0F43ECE6F0E66EB6
:10A4600070C7E6FF9DECE7F003E1010EDB2AECD7B5
:10A47000080EE4ECE5F00FE26FC772F770C773F7F0
:10A4800071C774F7010EDB50080DF350DF100701A0
:10A49000756F755106D0080EDF5C02E1000E01D029
:10A4A000800E70ECEBF002E2E16AE552E16E4A5098
:10A4B000B3EFE5F0AEECE5F01F981F9EFE0EDB500B
:10A4C000005C01E01F8E1F9CFE0EDB50D880005404
:10A4D00001E21F8C020E016E2DA204D01F88FE0E19
:10A4E00000C0DBFF1FAE90D01F50200B01E0010E1B
:10A4F0004A6E1F50400B01E0010E4A5C01E081D022
:10A500001FAC0DD00150D880005414E20150005E01
:10A51000FE0EDB50D88000540DE21F880BD00128BE
:10A52000E86C005C07E201500026FE0EDB50005C88
:10A5300001E21F88010159A50FD00050036EDF0E04
:10A54000B1ECE6F08BECF1F002E6D4ECEEF002E2D6
:10A550001F985AD00350006E1FA853D0FE0E00C0A3
:10A56000DBFF049476ECEAF004E1C90E0B5C01E138
:10A5700004840450040B12E1F5EC6DF0000904E0D2
:10A5800001013E51200B3DE0FD0EDB50FF0839E09C
:10A590000201415136E12150200B33E08EECE8F00E
:10A5A0000101010E016F04A403D0FE0EDB5011D097
:10A5B000FD0EDB50006EBFEC2DF0500E096EFE0E4E
:10A5C000DB40E840E8401F0B006E00501E0802E22E
:10A5D0001E0E006E78EC97F004B413D0030E010148
:10A5E000015D016E0150012A53ECE6F0200EEF6E82
:10A5F00054ECF4F0EF50300804E154ECF4F0200E89
:10A60000EF6E1F9A1FBC1F8AFE0EDB50B3EFE5F002
:10A610001350040B08E1F5EC6DF0000904E00101B2
:10A620003E51200B2EE08EECE8F001012D0E1A6F4A
:10A6300020A402D02B0E1A6F0201555107E154518C
:10A6400005E1535103E10101200E1A6F4CECE6F0D5
:10A6500055C23FF092ECF1F0300F01011B6F300E4C
:10A660003B241C6F300E0201542501011D6F0701B0
:10A67000EFAB05D0300E0201532501011E6F010121
:10A680001C8F1200C0ECF4F0A5ECE6F0EFCFDFFF7A
:10A690000101A16BA26BA36BA46BA56B1EAE03D0D3
:10A6A000050EA36F3ED076ECE8F0EF50400B03E1CF
:10A6B0002850040B1DE04FECE6F05BEC0EF0E55289
:10A6C00000C0A3F10050630827E20101A36BA22B95
:10A6D0007D0E005C02E1190EA36FD6ECF1F0FA0ECC
:10A6E0004A181AE14B5018E1A22B320EA36F14D076
:10A6F00076ECE8F0EF50200B02E0A52B0DD076ECC5
:10A70000E8F0EF50100B07E0020EA46F5AA704D038
:10A71000050EA46F01D0A42B2BAE03D0020E3EEC8D
:10A72000E6F0E552B3EFE5F0B10E006E02018FA541
:10A7300002D0B50E006E0050A3ECE9F038C100F075
:10A7400002018FA502D07EC100F078EC97F0300EA8
:10A7500001011D5D05E155ECEFF002E1200E1E6FD9
:10A760001200AEECE5F0050E4C6E4CC044F0FE0E4F
:10A7700069ECECF04B6A3D0F4A6E070E61ECF0F0AD
:10A78000006E71EC94F0010125ECEEF00C0E1DEC66
:10A79000E6F003E20E0E126F0ED00E0E136FFE0ED9
:10A7A000DB50630802E2100E136F0F0E1DECE6F093
:10A7B00002E2090E146F140E176F120E186FB3EF2A
:10A7C000E5F0AEECE5F07DEC94F00101012BFE0E1E
:10A7D000DB50006E78EC97F02C50100B07E1640E04
:10A7E0001DECE6F003E20101200E1A6F2CA807D041
:10A7F00001014D0E1E6F570E1F6F1B8F18D0FD0EDF
:10A80000DB5003E101011C8F07D00A0E1DECE6F0BE
:10A8100003E20101200E1B6F0101570E1E6FE6516E
:10A82000010B05E05951080B02E02A0E1F6FB3EF30
:10A83000E5F0BBEC2CF08EECE8F02FECE7F007E055
:10A84000010EE66E8DEC05F0940FE66E03D0E66A1D
:10A850004BC1E6FFB6DFE552E5522CA806D005EC69
:10A86000EDF04BC1E6FF7DDFE55212000FECF0F09A
:10A87000B90EA3ECE9F037C1DFFFC3ECEBF003E066
:10A88000B1ECEFF001E1DF6ADF50006E78EC97F099
:10A89000640EDF5C03E20101200E1D6F0A0EDF5C17
:10A8A00003E20101200E1E6FE552B3EFE5F08EECDE
:10A8B000E8F04CC100F078EC97F0640E01014C5DBB
:10A8C00002E2200E196F0A0E4C5D02E2200E1A6F92
:10A8D000930E006EBFEF2DF0020E0201965D04E1B3
:10A8E0000C0EDBECE5F00AD00D0EDBECE5F0030E10
:10A8F0000201965D03E10101320E1E6F500E096EDA
:10A900001200F00E006E68ECE6F002E0F30E006E4E
:10A9100048EC2EF035C100F068ECE6F002E056C1DC
:10A9200000F05CECEAF001011E8F1200AEECE5F0E5
:10A930002BC100F0C3ECEBF003E15BC100F011D0E0
:10A9400068ECE6F00EE057C100F0FE0EDB5009E0C7
:10A9500001019951020B05E09951040B02E09AC1E3
:10A9600000F0B3EFE5F0D20E006E68ECE6F00CE01C
:10A97000C3ECEBF009E001019951020B05E099519C
:10A98000040B02E0F60E006E48EC2EF0010EE66EAF
:10A99000CDDFE55278EC97F0300E01011D5D05E149
:10A9A00055ECEFF002E1200E1E6F1200AEECE5F068
:10A9B00057ECF4F0400B03E12850040B05E00101D3
:10A9C0009151020B01E18BD057ECF4F0200B03E026
:10A9D0002850040B02E00101A06B57ECF4F0400B8F
:10A9E00003E12850040B57E00101A2510EE0A351EE
:10A9F0000CE1FE0EDB5005E19E5102E19F5101E0AA
:10AA0000A26B9E6B9EC19FF16AD05A0EA35D13E1AB
:10AA10004CECE6F09EC13FF02CECEEF007E100506C
:10AA200003E101019F5102E00101A36B01019F6B52
:10AA300000509E5F54D09E5102E19F5150E09F51C3
:10AA40004A6E4B6A9E510A0D56ECE8F0A3514DEC4C
:10AA5000EAF082ECF4F0D7C143F0D8C144F0B8EC8E
:10AA6000FDF03AC0D5F13BC0D6F10101D551D61168
:10AA700036E0D5510F5ED651105AFE0EDB5001E183
:10AA8000A36B0A0E4A6E4B6A56ECF0F03EC09EF184
:10AA90003AC09FF124D057ECF4F0100B20E057ECB3
:10AAA000F4F0200B1CE1020E016E01015AA702D046
:10AAB000050E016E01C0A4F101C044F09FC13FF03A
:10AAC0002CECEEF004E1005002E000C0A4F1FE0E18
:10AAD000DB5005E0005003E000500101A45FB3EF3C
:10AAE000E5F0AEECE5F04FECE6F0E66A5FDFE5524C
:10AAF000E5529CC1D0F29DC1D1F29EC1D2F29FC15C
:10AB0000D3F2A0C1D4F2D3EC3AF001019C510FE191
:10AB10000301E35101019D5D0AE2D0C29CF1D1C263
:10AB20009DF1D2C29EF1D3C29FF1D4C2A0F1020125
:10AB3000852BB3EFE5F07AECEAF006E1DD93D0B3D4
:10AB4000DD83DD95D0B5DD85120001013BA306D084
:10AB5000D09313B6D083D09513B4D085ECDF04B076
:10AB600057DD41ECC1F075EF38F02EBC12000A0E33
:10AB700002015403F3504C6E4D6A5551640DF3506D
:10AB80004C244A6EF4504D204B6E535101014A241F
:10AB9000D96F000E4B20DA6F0A0E006E0701EFAB83
:10ABA00002D0010E08D0EFA907D0140E006E0101EB
:10ABB0005AA702D0320E006E20B403D00101D2ECAD
:10ABC000ECF029AA1AD0D6ECF1F0100ED8804A5633
:10ABD000270E4B560101DA514B18E8AE02D04B3428
:10ABE00004D04A50D95D4B50DA591FE200501BEC9B
:10ABF000E8F0D9274B50DA2318D000504B6AF00FF9
:10AC00004A6ED80E4B2201014B50DA19E8AE02D041
:10AC1000DA3504D0D9514A5CDA514B5806E200507B
:10AC20001BECE8F0D95F4B50DA5B2084800EDA151C
:10AC300003E02094D2ECECF0D6ECF1F0D9C13EF078
:10AC4000DAC13FF0D9ECEDF04BAE04D03A6C3B1ECC
:10AC5000000E3B223A500101D95F3B50DA5B9DEC7C
:10AC6000EFF050ECF3F03EC055F23A500101D96FCD
:10AC7000DA6B0A0E4A6E4B6A50ECF3F03EC054F2A7
:10AC80003AC053F244EF56F00101CEA9308E198C30
:10AC90000480A5EF55F00A01DA9F54EC0DF0016A2B
:10ACA0000C5011E152ECE7F02BE10701EFBF11D09E
:10ACB0000A0E016E10ECE9F03F50006E0150005C8E
:10ACC0001FE200501CD0030E0C5C13E10701EFAF34
:10ACD00002D0160E14D0FDECECF002E1140E0FD0F1
:10ACE000B65102E11E0E0BD0260E312563ECE6F0C4
:10ACF00006D0F2ECE8F002E0010E01D0160E016E73
:10AD00000150160802E2160E016E12000A0E010131
:10AD10000F5D09E12C50100B06E14B51500803E286
:10AD2000790E4B5D01E3000C010CF0DF000903E03C
:10AD30000101500E4B6F1200AEECE5F000AE14D0E6
:10AD4000FF0E0002F3CF85F2850EE96E020EEA6E69
:10AD5000EFCF3FF0FE0EDBCF44F0FCECFDF03FC048
:10AD6000EFFF0201856D09D000C03FF0FE0EDBCF82
:10AD700044F0FCECFDF03FC085F2B3EFE5F00101DB
:10AD80008DAD07D02EAC02D0FDEF04F002010A0E0B
:10AD90003C6F12000101E6A503D0E6956DEFECF0E3
:10ADA0000601D951D995010B01E0D985D951D9971F
:10ADB000020B01E0D987D9918850400B01E0D9817D
:10ADC000D9938850800B01E0D9830F0ED915E7EC99
:10ADD000E6F000A005D000AE02D0DF0701D0DF2BE7
:10ADE000DA51DA95010B01E0DA85DA51DA97020BD4
:10ADF00001E0DA87DE51DA91020B01E0DA81DE51FF
:10AE0000DA93010B01E0DA830F0EDA15E7ECE6F0D6
:10AE100000A009D06DECECF000AE03D00601E00715
:10AE200002D00601E02BDB51DB95010B01E0DB8555
:10AE3000DB51DB97020B01E0DB87DE51DB91080B76
:10AE400001E0DB81DE51DB93040B01E0DB830F0EBD
:10AE5000DB15E7ECE6F000A009D06DECECF000AEFD
:10AE600003D00601E10702D00601E12BDC51DC959D
:10AE7000010B01E0DC85DC51DC97020B01E0DC8793
:10AE8000DE51DC91200B01E0DC81DE51DC93100B04
:10AE900001E0DC830F0EDC15E7ECE6F000A00AD041
:10AEA0000201320E3B6F00AE03D00601E20702D072
:10AEB0000601E22BDD51DD95010B01E0DD85DD5161
:10AEC000DD97020B01E0DD87DE51DD91800B01E0B3
:10AED000DD81DE51DD93400B01E0DD830F0EDD15DA
:10AEE000E7ECE6F000A00AD00201320E3B6F00AEA4
:10AEF00003D00601E30712000601E32B1200045001
:10AF0000010B4A6E0450020B01E0010E4A5C07E09F
:10AF1000060EE66EF40EE66E010E07EFE7F0E00EA9
:10AF20000101F215016E1F0EF215026EF3C103F05E
:10AF3000015003E0E00E015C48E1025062E0015084
:10AF4000021203501FE12050080B06E03E51010B96
:10AF500003E02850010B16E02E50400B03E0305068
:10AF6000200B10E02150200B0DE002502727CE517E
:10AF7000100B08E02050080B05E02C50200B02E1DC
:10AF80000250282703041AE13E51200B12E1205001
:10AF9000080B0FE02E50400B06E13E51020B09E07A
:10AFA0002850010B06E12E50400B08E03E51010BEA
:10AFB00005E12150200B02E002502827020E035C1D
:10AFC00020E102500601DF271200800E015C11E132
:10AFD000100E025C16E2070E0214400F166E188E59
:10AFE0001898189002A602D0188801D01880E3950E
:10AFF0001200C00E015C05E1030E025C02E202C019
:10B00000F3F1120019BE12008A8C81AE03D0010147
:10B01000EE9712008150800B31E10101EE51080BD7
:10B020002DE1F29E8A9C04900492090E016EF26B4F
:10B03000060E5EECE9F0270E026E0150010803E2F5
:10B040000101F291F24381AE09D00150010805E2FD
:10B0500002060101F28F047001D004829EAA04D07E
:10B06000020E025E2BECEAF0025068ECE9F00106F9
:10B07000E2E145DF8A8C0101EE87F28E12000FECCF
:10B08000F0F0C0DF28A004D09CECCBF07AEF5DF0AC
:10B090002450800B4CE13150400B49E120A61BD0DD
:10B0A00040ECEDF0010129990201855102E0010116
:10B0B00029890101299B020185AF02D00101298B59
:10B0C000010129A934D01EAC02D0ECEC0BF0020136
:10B0D000640E506F2CD027C100F001012999005057
:10B0E00001E02989299B00BE298B29BB006C76ECE5
:10B0F000EAF00FE1B90E0B5C03E0E30E0B5C05E137
:10B10000D8900032D890003207D00038E842070BC0
:10B1100002D000380F0B006E005007E00101298DAE
:10B12000299F29BB298F276B02D001012999010191
:10B130002951100B09E0CE51100B06E12C50200BC9
:10B1400052E01E50400B4FE12050080B1DE03E51D5
:10B15000200B09E02E50400B06E1CE51100B14E0FD
:10B160002951100B11E048ECEDF001012A99020180
:10B17000855102E001012A8901012A9B020185AF64
:10B1800032D001012A8B2FD028C100F02A9900501B
:10B1900001E02A892A9B00BE2A8B2A992ABB006CCF
:10B1A00031AC05D0D8900032D89000320FD01CA21C
:10B1B00004D00038E8461F0B08D033A004D0003874
:10B1C000E842070B02D000380F0B006E00500AE077
:10B1D0000701280ED86F01012A8D2A9F2ABB2A8FCA
:10B1E000286B01D02A992C50200B03E01E50400BF5
:10B1F0000DE001012951100B01E00AD32A51100B77
:10B2000001E006D32150200B01E102D3D7CADCFABA
:10B21000D6CADDFABFDDDFC600F00601D9990050BD
:10B2200001E0D989D99B00BED98BD9A938D0D9BB27
:10B23000006CF3ECEFF033E0DF6B0201640E506F53
:10B240001350080B0DE11350040B0AE1020E01012B
:10B25000795D0EE13E51200B0BE02E50400B08E1D2
:10B26000298A0601D9BB299A80DCBBECECF017D007
:10B270003A51010B14E03E51010B11E1E1C227F1FB
:10B280000601D9AB04D0E1C227F10101276D01010C
:10B290002989CEA903D027C128F12A892884E0C6AC
:10B2A00000F00601DA99005001E0DA89DA9B00BE6D
:10B2B000DA8BDAA97CD0DABB006CF3ECEFF001E1B9
:10B2C00076D0E06B010E0E6EDABB0E68EEECE8F0A5
:10B2D0006CE02E50400B03E085ECE9F066E1050ED2
:10B2E0000C5C03E1DEEC0BF060D0020196510EE045
:10B2F000030ED1ECF4F0960EE66E020ED5ECE5F0FE
:10B300006CEC54F0188E3A0E166E4FD032BC4DD005
:10B31000060150A725D03584BEDC0E040BE133ECCA
:10B32000EEF008E2190E0124D75D04E2020ED65FAA
:10B33000D72B11D0800E0E140EE043EC12F0FF0F4D
:10B340000A01D65D08E279ECEDF0D880D75503E22A
:10B35000020ED627D7070A01010ED46F348821D0F8
:10B3600050A523D0358475ECEDF008E0C80EE66EEC
:10B37000280EE66ED80EE66E030E0AD08CDC190E8F
:10B380000124E66E79ECEDF0E66ED70EE66E0A0E5D
:10B39000D5ECE5F00A01030ED46F348879EC20F087
:10B3A000010EE66EE66E43ECE7F04AECEBF0E1C628
:10B3B00000F00601DB99005001E0DB89DB9B00BE59
:10B3C000DB8BDBA962D0DBBB006CF3ECEFF05DE064
:10B3D000E16B010E0E6EDBBB0E68050E0C5C03E12B
:10B3E000DEEC0BF052D0EEECE8F04FE02E50400BCC
:10B3F00003E085ECE9F049E1060150AB26D0358445
:10B400004ADC800E0E140CE033ECEEF009E279EC2D
:10B41000EDF0D880D75504E2020ED65FD7070FD0E3
:10B420000E040DE143EC12F0FF0F0A01D65D07E2B6
:10B43000190E0124D75D03E2020ED627D72B0A018D
:10B44000020ED46F3488AAECF0F0060150A91BD08C
:10B45000358453EC12F0B5ECF0F007E24A501408D2
:10B46000000E4B5402E253EC12F0B5ECF0F009E29E
:10B470004A503D08000E4B5404E253EC12F053ECDA
:10B4800012F05CEC12F04AECEBF0E2C600F00601C0
:10B49000DC99005001E0DC89DC9B00BEDC8BDCA980
:10B4A00098D0DCBB006CF3ECEFF001E192D0E26BE2
:10B4B000010E0E6EDCBB0E682DA418D068ECE6F011
:10B4C00008E1C80EE66E350EE66E010ED0ECE5F032
:10B4D0000AD0C80ED1ECF4F0560EE66E010ED5EC93
:10B4E000E5F0EEEC1DF081EC54F06FD050AD19D0CA
:10B4F000320E006E010191AD02D0640E006E00505C
:10B50000E66E080EE66E4C0EE66E010ED5ECE5F02A
:10B5100057EC54F04CC103F5EEEC80F002011787B4
:10B5200054D050AF52D01FECE8F0010190A503D0E9
:10B5300031EC09F04AD03450040B25E0000403E05C
:10B54000020E005C20E10E50482748C1E6FFC10E04
:10B55000C3ECE5F00E0EDBECE5F048C100F00101B4
:10B5600048AF04D048C100F00001006C00900042D8
:10B5700078EC97F001012B0E1D6F48AF02D02D0E15
:10B580001D6F1F8F22D002018FA50FD03C0EE66EDB
:10B590007E0EE66E010ED0ECE5F07EC1E6FFCC0E2D
:10B5A000C3ECE5F094EC53F00FD018EC1EF03C0E19
:10B5B000E66E380EE66E010ED0ECE5F0A8EC16F063
:10B5C00094EC53F0020119832B842E8E02011E0E7F
:10B5D000306FE3C600F00601DD99005001E0DD891F
:10B5E000DD9B00BEDD8BDDA913D1DDBB006CF3EC70
:10B5F000EFF001E10DD1E36B010E0E6EDDBB0E68C5
:10B600002DA62FD068ECE6F00AE13C0EE66E2B0E7C
:10B61000E66E010ED0ECE5F050ECEAF01FD0C3EC82
:10B62000EBF006E13C0EE66E5B0EE66E010E12D00C
:10B6300001019951020B09E09951040B06E03C0EFF
:10B64000E66E9A0EE66E010E05D03C0EE66E570EC3
:10B65000E66E010ED0ECE5F022EC1EF0B3EC54F0F7
:10B66000D3D052AFADD0010190B5AFD034B632D007
:10B6700021BE04D08D0E006E53EC2EF0FF0E0E5C3A
:10B680000CE102013F0ED8800F55000E10551FE24D
:10B69000400E0F5F000E105B1AD087C201F02C50D5
:10B6A000100B07E102018751780803E26C0E015C80
:10B6B000016E01500101D45D0AE20201480E0F5DE6
:10B6C000710E105904E2400E0F27000E1023E5EC16
:10B6D0000BF09AD002012D6B780E016E026AD5EC48
:10B6E000EFF002E0DA0E016E2CA804D0960E016E87
:10B6F0000A0E026E0150E66E0250E66E4B0EE66ECA
:10B70000010ED5ECE5F02B84E2EC2AF086EC56F045
:10B7100000090BE00101500E4B6F0E0406E1D5EC61
:10B72000EFF003E00101790E4B6F19EC54F0780E45
:10B73000016EB5ECE8F002E1500E016E2C50100BDA
:10B7400010E10E0403E1790E4B5D06E0800E0E144D
:10B7500008E001504B5D05E1328EEEECE8F001E0CF
:10B760001D941FECE8F03250800B0EE102013151C4
:10B770000BE000500CE0050E005C09E0030E005CDD
:10B7800003E110ECEAF003E00E505AECEFF032AEB9
:10B7900014D0329E04981AA006D004882DEC0BF029
:10B7A000050E3EECE6F083EC28F0AEDA04A802D0F9
:10B7B00028EC0BF00E505AECEFF00201188B24D05D
:10B7C00052A122D0010190A503D031EC09F01CD088
:10B7D00037C1DFF218EC1EF0280EE66E370EE66E6B
:10B7E000010ED0ECE5F0B6ECEDF003E001013751CD
:10B7F00006E00201DF5105E10101375102E0E6EC0C
:10B800001CF0020119852B842E8E02011E0E306F52
:10B810001EAC64D00701EF83DDEC09F001013E911D
:10B82000139C3E51010B01E0138C65EC34F0006E6B
:10B8300000500F0802E20F0E006E100E0002F3CF50
:10B8400021F25AEC2FF01E9A050E0701D3250201B2
:10B85000D880215501E21E8A2B50800B13E1205124
:10B8600011E0050E0701D35D0201215D03E220EC2A
:10B8700009F01E881E50100B31E01E50200B2EE0E8
:10B88000020109D02B50800B0AE11E50800B07E10A
:10B890001E50200B04E0FA0E206F1E981FD02BBE06
:10B8A00002D01DEC09F02CBA17D00C0EE66E050E76
:10B8B00059ECEBF0E66E96ECE8F00AE007C5C3F150
:10B8C00008C5C4F109C5C5F10AC5C6F10BC5C7F164
:10B8D000E1C227F10101299B010129891E50800B3A
:10B8E0000BE101012951100B01E172D02050080B2E
:10B8F0006FE02150200B6CE002011E0E306F1EAC79
:10B9000002D0140E306F2CAA2FD01EBC16D001010D
:10B910004751630801E2476B800E271506E0FB0ED6
:10B92000275D03E2276B000E12D0800E27154FE132
:10B93000275103084CE2276B09D00101276B2BAE7E
:10B9400009D00501065143E1320E066F010E3AECB3
:10B95000EEF03DD0AA5103083AE3010E3AECEEF0C6
:10B960000101140EAA6F33D0178305013B812C8C83
:10B970002D8A70ECE6F00C50E66E42EC53F0E55286
:10B9800040ECEDF01E50800B06E00101275103E171
:10B99000AFEC3AF016D0020185AF0AD0EFC7E6FF50
:10B9A00071EC55F0E5520201E1510101272709D060
:10B9B000855107E0EFC7E6FFE8ECEAF0E15101014D
:10B9C000275F02018551DCE12E829EEC04F01E9E71
:10B9D00001012A51100B5DE02050080B5AE0215064
:10B9E000200B57E002011E0E306F1EAC02D0140E69
:10B9F000306F178305013B832C8CD3C1DFFF2E50A2
:10BA0000400B03E1B3ECEBF002E00C50DF6E2EAC28
:10BA100004D02D8A70ECE6F003D02D9A27ECE8F0E4
:10BA2000DFCFE6FF42EC53F0E55248ECEDF00201C7
:10BA300085AF0CD0DF50D8ECF2F0E66E71EC55F02B
:10BA4000E5520201E251010128270BD0855109E09E
:10BA5000DF50D8ECF2F0E66EE8ECEAF0E2510101DA
:10BA6000285F02018551E1E12E822EAC03D09EECCD
:10BA700004F002D03DECE8F025A605D0010E096ED9
:10BA80000701140E826F0101CEA903D00701280E11
:10BA9000D86F2CAC2BD0B3ECEBF00FE02951100B8E
:10BAA0000CE02A51100B03E12C50200B06E02E5025
:10BAB000400B03E105013B832C9C01018DAD03D0BC
:10BAC0002C9C08AE198CFCEC38F001013EA9308E9C
:10BAD000D8EC3EF02C9C26822D50200B06E02E50F8
:10BAE000400B03E1B3ECEBF001E0248A01012A9959
:10BAF00029992894E552B3EFE5F0AEECE5F0180E85
:10BB000007011B171C6BFE0EDB5001E11C81FE0EB2
:10BB1000DB0401E11C836DECEDF001E11B81FE0E05
:10BB2000DB50030801E11B83FE0EDB50040801E13A
:10BB30001B85B3EFE5F0075005E0D5CAE6FFDDDF72
:10BB4000E5521200180E07011D171E6B0A01D55190
:10BB500002E107011E810A01D50502E107011E83EA
:10BB6000020E0A01D55D02E107011D81030E0A01E3
:10BB7000D55D02E107011D83040E0A01D55D02E1D6
:10BB800007011D851200000000000000E3EC08F032
:10BB9000EDEC08F082A82D808A8A1200020E68EC73
:10BBA000E9F0C3EF5DF0050EE66EFFEC18F0E5522C
:10BBB000F00E8C148C6EA5D88A9A00001FC700F076
:10BBC0000101E8AD02D0F2C700F00101E8A915D0EB
:10BBD0000050E66E04EC7AF0E5521DC704F0049CB8
:10BBE00007011EB1048C049E07011EB3048E04508D
:10BBF000E66E04EC7AF0E5521DD0060E00C0E7FFB9
:10BC0000070B04E0E742E79EE806FCE1E750E66E3A
:10BC100004EC7AF0E5523F0E0014040DF3500701D6
:10BC20001E11E66E04EC7AF0E5521DC7E6FF04EC47
:10BC30007AF0E552A8DFF00E8C1406098C6E61D8FC
:10BC40008A9A000020C700F00101EEA315D0005031
:10BC5000E66E04EC7AF0E5521BC704F0049C070181
:10BC60001CB1048C049E07011CB3048E0450E66EC4
:10BC700004EC7AF0E5521DD0060E00C0E7FF070B7A
:10BC800004E0E742E79EE806FCE1E750E66E04ECDC
:10BC90007AF0E5523F0E0014040DF35007011C1119
:10BCA000E66E04EC7AF0E5521BC7E6FF04EC7AF08E
:10BCB000E55269DF1200F00E8C1404098C6E21D855
:10BCC0008A9A000010C7E6FF04EC7AF0E5525BDFC9
:10BCD0001200F00E8C1402098C6E13D88A9A0000A0
:10BCE00013C7E6FF04EC7AF0E55212C7E6FF04EC56
:10BCF0007AF0E55211C7E6FF04EC7AF0E5524EDF28
:10BD00001200010E68EFE9F0050EE66EFFEC18F088
:10BD1000E5522D90DEDF47DFF7EC13F0F00E8C14C8
:10BD200005098C6EEEDFEDDFECDFEBDF8A9A0DC7E5
:10BD3000E6FF04EC7AF0E5520CC7E6FF04EC7AF07B
:10BD4000E5520BC7E6FF04EC7AF0E5520AC7E6FFBE
:10BD500004EC7AF0E55222DFF00E8C1403098C6EAD
:10BD6000D0DF8A9A00000FC7E6FF04EC7AF0E552B4
:10BD70000EC7E6FF04EC7AF0E55205DFF00E8C14F6
:10BD80000A098C6EBEDF8A9A000009C7E6FF04EC40
:10BD90007AF0E55208C7E6FF04EC7AF0E55207C7EF
:10BDA000E6FF04EC7AF0E55206C7E6FF04EC7AF011
:10BDB000E552E9DE80DFF00E8C1401098C6EC6823C
:10BDC000C6909FDF8A9A000000000000000016C79E
:10BDD000E6FF04EC7AF0E55215C7E6FF04EC7AF0D2
:10BDE000E55214C7E6FF04EC7AF0E552D7DEC680D0
:10BDF000C692F00E8C161200810E48ECE6F0320E60
:10BE0000096E308836C12AF21200030E0A6E2A0E1D
:10BE1000E66E000EE66E0A0E07EFF2F0030E0A6EF3
:10BE2000AA0EE66E2A0EE66E0A0EE66E300E29EFB8
:10BE3000F5F090EFF4F0AEECE5F005013B8F6DEC22
:10BE4000EDF00DE101013EB902D08D9D08D03E9983
:10BE5000E66A23EC91F0E55201018D9D34D0FE0E8F
:10BE6000DB5024E085ECE9F021E1CE993EB909D020
:10BE70003E89010EE66E23EC91F0E55201018D8DB5
:10BE800003D08D8D09EC91F0198638EC0DF01B82F2
:10BE9000FEECB9F026ECBAF01B929FECECF0F70E3A
:10BEA000E66EF30EE66E010E07ECE7F0FE0EDB50D9
:10BEB00011E185ECE9F00EE08D9D09EC91F038EC94
:10BEC0000DF075EC38F0FE0EE66EF30EE66E010E28
:10BED00007ECE7F0B3EFE5F012001E50400B0CE06A
:10BEE0002B50800B09E12250200B06E02B8E130E05
:10BEF000A3ECE9F020EC09F0120025A808D0010E0F
:10BF0000E66E99DFE5520F0EF9ECF3F01B86120096
:10BF1000010124A16AEF67F00101249102012207C7
:10BF20000201225101E0A8D10201640E226F020138
:10BF3000ED6B0201295102E00201290701018E5136
:10BF400006E001018E0701018E5101E132960201E6
:10BF500030510EE02050080B0BE0020130070201C7
:10BF6000305106E11EAC02D01E8E02D02EBE2E9E97
:10BF7000300E0401F75D06E10201176B186B196BB7
:10BF80001A6B02D0C3ECCDF002012A5126E0050164
:10BF9000005123E12850400B20E102014A514B118E
:10BFA0001CE102012A0702012A5117E10D50006E1F
:10BFB00002016A5108E07F0E02016A15006E199AAB
:10BFC00002016ABF198A010EE66E0050E66E72EC3D
:10BFD00090F0E552E55202016A6B02016E07020120
:10BFE0006E511EE10701F1050FE102010F0E6E6FA8
:10BFF000560E02011E5D07E2870E006E24885FEC7C
:10C000002EF00968268E0CD00101545102011E5DEC
:10C0100007E2870E006E24885FEC2EF00968268EFA
:10C02000020128514EE0020128070201285147E190
:10C030002250200B44E00E0E165C3AE150ECB0F0BA
:10C0400028702892520EE66EDBEC07F0E552520E95
:10C05000E66EDBEC07F0E55228B011D0570EE66E25
:10C0600075EC2EF0E55275EC38F048EC15F04E0EFC
:10C07000E66EDBEC07F0E552EAEC18F013D0580E50
:10C08000E66E75EC2EF0E5523BEC96F0E80EE66EAF
:10C0900046ECFDF0E552E3EC18F0520EE66EDBECF8
:10C0A00007F0E5523B0EE66EDBEC07F0E55207D0F9
:10C0B00028A005D04C0EE66E6BECCBF0E5526AEF93
:10C0C00067F0FBECC5F0010101013B51100B06E1EB
:10C0D0001450020B05E01A50200B02E1060105770F
:10C0E0002950400B01E0010E020F016E2950400B58
:10C0F00001E0010E050F026E03681EAC10D0015066
:10C10000EA6A110FE96E010EEA22EF7E0150EA6A37
:10C11000110FE96E010EEA22EF50800B036E5FEC07
:10C120000BF0000923E0FF0E035C11E10250EA6A04
:10C13000110FE96E010EEA22EF7E0250EA6A110F3A
:10C14000E96E010EEA22EF50800B036E0FD0025011
:10C15000EA6A110FE96E010EEA22EF9E0250EA6AC6
:10C16000110FE96E010EEA220350EF126DEC0BF095
:10C1700000091AE0FF0E035C08E10250EA6A190F99
:10C18000E96E010EEA22EF7E0FD00250EA6A190F23
:10C19000E96E010EEA22EF9E0250EA6A190FE96E7B
:10C1A000010EEA220350EF12DCEC04F0000902E079
:10C1B00006011A792350040B05E02D50100B02E004
:10C1C0000601127912EC08F000090EE02D50400B28
:10C1D0000BE12D50800B08E10101E3B703D006010C
:10C1E0000E7102D006010E810201435105E0145088
:10C1F000080B02E00601027358ECC5F0000903E1E8
:10C200002F50200B27E02F9AE3EC18F0016A030E61
:10C21000015C15E2026A040E025C0BE2020E006E83
:10C2200019EC92F0320EE66E36EC29F0E552022A55
:10C23000F2D7E66836EC29F0E552012AE8D7EAECB5
:10C2400018F00101629926820FEC9CF043ECC5F0D6
:10C25000DFECC4F002013D5102E002013D070201A2
:10C26000915105E02350100B02E1020191070201F8
:10C27000455102E0020145072850010B28E081509A
:10C28000010B03E02150040B22E01CEC16F0FF0828
:10C290001EE12E50400B1BE12150200B18E01950DD
:10C2A000800B15E10201245102E002012407020182
:10C2B00024510DE12AA003D0C5EC07F0FBD73B0EBB
:10C2C000E66EDBEC07F0E5520201280E246F060152
:10C2D000F45102E00601F407010199AD17D1030101
:10C2E000C6070301C65101E011D1C69AF00E8C14A5
:10C2F00007098C6E06DD8A9A00000000000000002D
:10C300000000000000000000049082B804808A8AC7
:10C31000C68AF00E8C160101E5BD12D00301010E94
:10C32000C66F04A00CD00301060EC66F0101E58D97
:10C330000301CA6BCB6B0301C86B0301C76BE6D06B
:10C34000D8900301CB33CA330301C82B04A003D018
:10C350000301CB8F09D00D0E0301C85D05E2030177
:10C36000C72B070E0301C7170301040EC66F030195
:10C37000C8510F0801E3CAD00301960EC66F010130
:10C38000E59DCAC30FF0CBC310F000010F1C01E103
:10C39000101C0CE1020E02017E5D07E1B90E0B5C80
:10C3A00004E1248A26820601426BB0D00FC00FF050
:10C3B00010C010F00F1E101E10C000F0700E0016FE
:10C3C00000380F0B006E0301C751005C01E09ED0E6
:10C3D0000F0E00011016000110A603D0F00E000190
:10C3E00010120FC0D9F110C0DAF10101DA3504E3FF
:10C3F000D9511708FC0EDA5501E388D00101D89015
:10C40000DA5104E6E90ED95D030EDA5901E37ED074
:10C41000D0C3CEF3D1C3CFF3D9C1D0F3DAC1D1F3B6
:10C420000A0E0F6E106A030E0301C95D03E2640E6B
:10C430000F6E106A0101D9510301CE5D4C6ECF51D0
:10C440000101DA554D6E4CC0E6FF4DC0E6FF9EEC93
:10C450002EF0E552E552F3CF4AF0F4CF4BF00F50F7
:10C460004A5C10504B584BE2D0C3CCF3D1C3CDF350
:10C47000FF0E0301C95D02E20301C92B030E030194
:10C48000C95D22E30101D9510301CE5D4C6ECF514C
:10C490000101DA554D6E4CC0E6FF4DC0E6FF9EEC43
:10C4A0002EF0E552E552F3CF4AF0F4CF4BF0000EF8
:10C4B000D8804A54000E4B540CE20201345109E179
:10C4C000BBEC05F0000905E0D7EC2CF03488B9ECA2
:10C4D0004BF0020E02017E5D11E1B90E0B5C03E030
:10C4E000E60E0B5C0BE1248A2682B90E0B5C06E19A
:10C4F0000601080E426F06011E0E436F07D00301AE
:10C50000C951020803E20301010EC96F02014A5139
:10C510004B1167E01CA020D002014A07000E4B5BC4
:10C5200002014A514B1117E11A50200B14E01CA2D2
:10C5300010D09CEC0AF04DEC05F0F0C2D7F1F1C23E
:10C54000D8F10CEC0BF00201280E4A6F230E4B6F52
:10C5500002D0A2EC0AF045D02150400B42E01A5024
:10C56000400B3FE001010101B251080B03E11A50F9
:10C57000200B37E002014A07000E4B5B1A50200BDC
:10C580000CE0A0EC1DF000090AE18150010B05E16F
:10C5900001010101E351100B02E1000E01D0010E77
:10C5A0000490E8B0048002014A514B1103E00450AA
:10C5B000010B17E002014A6B4B6B0101E39904A0E8
:10C5C00006D002012A6B2AC26AF255EC81F0A2EC75
:10C5D0000AF00101B2A704D0259224BC2582228E44
:10C5E00021940201505102E0020150070201515111
:10C5F00002E00201510702014F5102E002014F0720
:10C600000201465102E0020146070201425102E0E6
:10C6100002014207020140510FE0020140070201FE
:10C6200040510AE108504A6E4B6A820E4A1801E1F5
:10C630004B5002E054EC0EF02B50200B56E0020160
:10C640003B5153E10701DE5102E00701DE07010122
:10C650002E5107083AE27BEC28F0000936E008AEDC
:10C660000ED00701DE510AE180EC14F0D6EC0FF099
:10C6700002010F0E456F07015F0EDE6F25D002012C
:10C68000455122E1010101013B51040B04E10A0E75
:10C6900001012E5D07E12DEC0BF0060EE66E36EC87
:10C6A00029F0E5520CEC05F0D6EC0FF00101010188
:10C6B0003B51040B04E10A0E01012E5D02E128EC5E
:10C6C0000BF002010F0E456F10D0800E081405E12B
:10C6D000010101013B51040B08E10701DE5105E1B5
:10C6E000D6EC0FF007015F0EDE6F02012307020197
:10C6F000235146E10201280E236F1BAC10D07EECC3
:10C700004AF00C50006EB8EC4AF006010F790601B1
:10C710000FA904D0D3C100F0B8EC4AF031D01CA866
:10C7200003D0060112792CD01DA203D00601147982
:10C7300027D01A50200B07E0010101013B51100BDB
:10C7400002E1060105772550020B04E1C4EC0DF06F
:10C75000000916E00201405113E108504A6E4B6A8D
:10C76000820E4A1801E14B500BE02650040B06E103
:10C770002D50800B05E12D50400B02E10601107198
:10C780000501445129E0BBEC05F0000925E02250E9
:10C79000100B22E005014407050144514A6E4B6A23
:10C7A000D8904B5004E6960E4A5C000E4B580CE3B2
:10C7B000050144514A6E4B6A960E4A1801E14B50EE
:10C7C00002E10501446B08D006011C91140E05011D
:10C7D000445D02E206011C8102013B5102E00201BC
:10C7E0003B0702013C5116E0010101018D51400B54
:10C7F00011E0BBEC05F000090DE002013C0702016D
:10C800003C5108E11B8226ECBAF01B920101286B17
:10C8100028C127F10701D85109E00701D80707010E
:10C82000D85104E10101286B28C127F102013A51D6
:10C830001EE002013A0702013A5119E1FFEC26F02D
:10C84000000903E16AEC98F012D00701D551070105
:10C85000D6110DE00701D55102E00701D507070108
:10C86000D65102E00701D6070201020E3A6F02011B
:10C8700039510CE0020139070201395107E1188EE4
:10C88000170E166E2DAC02D00F0E166E0101AB51B5
:10C8900074E00101AB070101AB516FE1AFC1F6FFDD
:10C8A000B0C1F7FFB1C1F8FF0800F550006E0201FA
:10C8B000E05107E0830E0A6EE0C201F044EC4DF057
:10C8C0000A6A0201AB51AC1120E0010EE66EABC268
:10C8D000E6FFACC2E6FF060EE66E010EE66E13EC56
:10C8E0004EF04A6E050EE15E4A50016E06C100F040
:10C8F0000201AB2B000EAC233550800B05E001503C
:10C9000003E000507F0801E2006A005015E00101D9
:10C91000190EAB6F0050E66E1FEC8BF0E552020172
:10C92000E05103E00201E02B06D00101AF2B000E25
:10C93000B023000EB12321D02950080B03E1315060
:10C94000080B02E0299619D00201E05105E002012E
:10C95000E06BFA0E096E04D0D8900932D8900932F3
:10C9600024A60BD0E80EE66EED0EE66E010EE66E26
:10C970007BEC2EF0E552E552E5520201385106E01B
:10C98000020138070201385101E1269E02013751A8
:10C9900009E0020137070201375104E1060141694C
:10C9A00041C640F60101A85102E00101A8070701B4
:10C9B000825102E00701820702013F512AE0020191
:10C9C0003F0702013F5125E1000E0601E76EC01945
:10C9D000E8AE02D0C03503D0E750D880C05503E29E
:10C9E0000601C00702D00601C02B000E0601E76E4B
:10C9F000C219E8AE02D0C23503D0E750D880C25584
:10CA000003E20601C20702D00601C22B0201050E95
:10CA10003F6F0201FA516AE00201345167E108BE3A
:10CA200003D00201FA6B62D00201FA070201FA5147
:10CA30005DE120A20BD0BEC19CF1BFC19DF1C0C180
:10CA40009EF1C1C19FF1C2C1A0F10AD0B9C19CF150
:10CA5000BAC19DF1BBC19EF1BCC19FF1BDC1A0F1A6
:10CA600001019C514C6E4D6AE80E4D02F3CF4DF022
:10CA7000030E4C02F3504D26E80E4C02F3CF4CF05F
:10CA8000F4504D2601019D510A0D4C50F3244A6E7D
:10CA90004D50F4204B6E0A0E4E6E4EC044F09EC1B7
:10CAA0003FF0FCECFDF03F5000014A240F6E000EF9
:10CAB0004B20106E030E0F0B05E0D89010320F3292
:10CAC000E806FBE10201FB510F1802E1FC511018CE
:10CAD0000DE00FC0FBF210C0FCF2400E016E000131
:10CAE000105001260FC000F08AEC92F00201315183
:10CAF0002EE00201310721BC25D00101E4A106D0BE
:10CB00000201316B0101E491F6EC27F01B50800B20
:10CB100019E0800E081416E02150010B13E1020108
:10CB2000316B1B9E0A01DA8F54EC0DF0010EE66E9C
:10CB300088EC91F0E5520201020E3C6F0201178B66
:10CB400005013B850201315102E1248A268202015E
:10CB5000205109E01E50400B06E0020120070201AF
:10CB6000205101E11E8E0501065102E00501060774
:10CB70000201485107E0020148070201485102E161
:10CB800044EC0AF009506EE0090609506BE101011E
:10CB9000B29D0101B29F30980101E3951D921C984E
:10CBA0002682248A289821BA13D0040E0101465DFA
:10CBB00008E1010101019051100B03E10101E88F2F
:10CBC00005D080C1E6FFBBEC0EF0E5528DEC2EF0F7
:10CBD000218A27EC94F06DEC5FF001010101E8512E
:10CBE000100B14E02E50400B11E12250200B0EE0F0
:10CBF000180E165C0BE11850100B08E0020E0B6EBD
:10CC0000EDEC9BF0C0EC9BF012AC188E020196513B
:10CC100003E13250400B26E022AA1DD0092A01016F
:10CC2000B28F020E0201965D15E1020197514A6E24
:10CC30004B6A4B3404E24A509608000E4B5408E20B
:10CC40007DEC94F0100EE66E2DEC98F0E55202D0DB
:10CC50000201972B07D0329C0201965103E0188EF7
:10CC60003A0E166E02012D5102E002012D0702015B
:10CC70002E5102E002012E0702012F5102E00201B3
:10CC80002F070201475102E0020147070201435109
:10CC900002E0020143070201445102E0020144079D
:10CCA0000101AA5102E00101AA070301E25102E0D9
:10CCB0000301E20702014C5102E002014C070201AC
:10CCC0004D511EE02250200B0CE1110E4A6E4AC05D
:10CCD00044F04DC23FF0FCECFDF03B5002E1060198
:10CCE0000E7302014D072250200B05E02150400B2E
:10CCF00002E0DCEC05F002014D5102E108EC05F028
:10CD0000060143510EE0060143070601435103E1CA
:10CD100006015A0E436F26860F0E0601435D01E29F
:10CD200026960201325110E00101EEA503D0020166
:10CD3000010E326F020132070201325102E153EC5F
:10CD400085F002011E0E316F02014E5113E0010108
:10CD500001012951400B0EE102014E0702014E5123
:10CD600009E147C100F019863582C8ECB6F002012E
:10CD7000010E346F0201345101E178D00201340711
:10CD80000201345101E072D078EC44F0C5EC45F07A
:10CD900084EC5EF031EC93F021A204D0219275EC8A
:10CDA00038F054D02CA602D051EC2CF0FAEC90F0D4
:10CDB00048EC15F0E6EC1CF025AC0DD025A806D00B
:10CDC000010E076EE66A67EC3BF0E552076AE66A19
:10CDD00067EC3BF0E552259C076A01018DAD07D059
:10CDE00001018D9D010EE66E1BEC5FF0E552EAEC51
:10CDF00018F0640EE66E36EC29F0E55201017AB7C0
:10CE00001ED00701F1051BE03550020B18E125A8E3
:10CE10000DD0010E076E95EC3CF0000907E1480EBD
:10CE2000006E5FEC2EF00101320E1F6F076A95EC69
:10CE30003CF0000904E1480E006E5FEC2EF0DFECE0
:10CE4000C4F01CA603D0C9EC32F01C9619B008D06F
:10CE5000E2EC2AF095EC56F0E66A45EC22F0E55259
:10CE60001990020117890501BF0E3B6F020149515C
:10CE700006E0020149070201495101E1268202014F
:10CE8000355102E0020135070201415102E0020181
:10CE900041070201335102E00201330702012C5124
:10CEA0000AE002012C0702012C5105E1780EE66E22
:10CEB00068EC18F0E55202012B5107E002012B0744
:10CEC00002012B0502E1A2EC12F002013E5102E048
:10CED00002013E07120006014F6B4FC64EF64FC6C9
:10CEE0004DF64FC64CF64FC64BF6120013ECF0F061
:10CEF000DE52010EDD6EFE0EDB5022E118ECF3F087
:10CF0000050EE66E200EDF24E66E4B0EE66E060E74
:10CF100017ECE6F026A406D0FF0E06014B5D0FE1EC
:10CF2000DADF0DD0050EE4ECF4F0B90EE66E010E7A
:10CF300017ECE6F00F0E26ECF1F00050DF6E0A6AF7
:10CF400026B44BD00101B951630807E3B9510FE191
:10CF50000301E3510101BA5D0AE23E0E46ECF4F032
:10CF6000FE0EDB5001E1B7DF010EDB6A22D0FE0EC0
:10CF7000DB501FE12D50800B07E0DF500A0804E270
:10CF80000701EF9BDDEC09F0DFCFE6FF1FEC43F07C
:10CF9000E55201018D51100B0CE00A0E475D09E2CC
:10CFA00071EC94F023ECE8F0DFCFE6FFF8ECA4F0AE
:10CFB000E5520201395111E1640E0101475D07E2BA
:10CFC0004CECE6F047C13FF003ECECF005D04D0E21
:10CFD000196F030E4715310F1A6F016A050E015CB8
:10CFE00031E20150EA6A4B0FE96E060EEA22EF5079
:10CFF0004B6A120F4A6E070E61ECF0F0026E2D0EB6
:10D00000025C05E10101B35102E1200E026E020152
:10D01000395116E1020E012453ECE6F002C0EFFF95
:10D0200026A404D00101610E196F0AD0015008E155
:10D030002C9A2A0E025C04E12D50800B01E02C8A10
:10D04000012ACCD72650040B05E10201395102E137
:10D0500001011B8F010EDB5070ECEBF002E2E16A84
:10D06000E552E16E4A50B3EFE5F022ECEFF0016ECD
:10D0700047515AECE7F0050EE66E4B0EE66E060ED3
:10D08000E66E200E012429EFF5F03450400B04E049
:10D090000101DE51800B09E13450400B04E1010134
:10D0A000D151400B02E1000E01D0010ED8EFE9F0A2
:10D0B00034AC03D00101DE8F12000101D18D1200CA
:10D0C00034AC03D00101DE9F12000101D19D12009A
:10D0D000D3EC09F00101076F020E075D01E10707BC
:10D0E00041ECEEF0EFCF06F106511F0801E2066BAE
:10D0F0000490D1BD0480075003E00490DEBF04809B
:10D100001200CEEC0CF0EBEC1FF0E2DF300E016E03
:10D110000450010B1AE00701EF51010B16E0030E5A
:10D120000C5C13E03FECF4F0080B08E08BECF1F042
:10D1300004E61F0E4A5C000E4B5807E206C1E6FFEC
:10D14000E90EC3ECE5F0310E016E0150C6ECE5F0DE
:10D150009CDFF3501596E8B0158612007DEC94F034
:10D16000110E76ECE9F0B4DF010106510F0802E27E
:10D170006D0E1B6F0651B9ECEFF0310F1D6F030EF2
:10D180000615310F1F6F81EF68F0248E209600681E
:10D1900048EC2EF0AEEF68F0249E05EC0EF034ACB7
:10D1A00002D035ECEFF012003450400B04E00101E6
:10D1B000DE51010B09E13450400B04E10101CF5174
:10D1C000200B02E1000E01D0010ED8EFE9F033ECA4
:10D1D000E9F0EF04016E5EECEBF001C03FF0FCEC17
:10D1E000FDF03B50026E5EECEBF001C03FF092ECC4
:10D1F000F1F0036E04900101CFBB0480075003E0FF
:10D200000490DEB10480110EE66E430E022443EC5E
:10D21000E6F0E66EA90EDFECE5F04A0E032443ECDF
:10D22000E6F0E4ECF2F00450010B02E0012802E128
:10D23000000E01D0010E000902E0370E01D0360EBB
:10D24000E4ECF2F0006A02B004D003280E0DF350B3
:10D25000006E0050E66EA30EC3ECE5F0100E4A6EB1
:10D2600021ECE9F04A50EF1622A832D0AB0E4B6EFB
:10D27000EF0E4C6E010E4D6E6BECE8F0EF044E6E4F
:10D280004F6A506A4B504E24F36E4C504F20F46E50
:10D290004D505020A4ECF0F00800F5CF4AF021ECFE
:10D2A000E9F04A50EF120450010B04E06BECE8F097
:10D2B000EF5002E1000E01D0010E4A6E21ECE9F0C0
:10D2C0000BECECF0DF0EEF14F310EF6ECBEC0EF086
:10D2D0006BDFF3501594E8B0158404B002D005015B
:10D2E000446B120071EC94F0170E2CECE7F033EC69
:10D2F000E9F0EF5006E1F7ECEFF00E0E2CECE7F062
:10D3000010D033ECE9F056ECF3F03F280101166F32
:10D310000E0E176F5EECEBF08AECE8F03B28010193
:10D32000186F7DEC94F0910E6DECE9F022A823D0FB
:10D330000101030E016F6BECE8F0EF5003E1010710
:10D34000A60E17D06BECE8F056ECF3F03B50310F23
:10D3500001011F6F1F5102E1630E1F6F070E005C7A
:10D3600002E23E0E06D00E0E005C02E2410E01D03B
:10D37000440E6DECE9F0D7EFECF0308AA3ECE7F067
:10D38000209672EF69F0309A05EC0EF034AC02D0C2
:10D3900035ECEFF0120071EC94F0050E0C5C12E12C
:10D3A0000101030E006F100E0201B3253BECEBF000
:10D3B0002DECE6F017EC2EF0040EFEECF3F001017C
:10D3C000188F29D0030E0C5C1AE109ECE8F009E093
:10D3D000220E61ECF2F02CECE7F0B30E2CECE7F04F
:10D3E0001AD01DECEFF00101006F17EC2EF00101D7
:10D3F000100E146F15510FE1100E156F0CD0F2ECDA
:10D40000F2F02CC100F05BEC97F00101155102E144
:10D41000100E156F186B7DEC94F0AE0E006E09ECDB
:10D42000E8F002E0B40E006E050E0C5C07E1E90EB8
:10D43000006E0201B5A502D0E20E006E00506DEF45
:10D44000E9F02580A3ECE7F02096A5DF050E0C5C43
:10D4500006E0E3EC18F0030E006E19EC92F01200F7
:10D46000050E0C5C03E145EC09F004D044EC0AF035
:10D47000EAEC18F0259005EC0EF05BEF0FF071EC84
:10D4800094F00101B6511BE0030EB65D06E11F0EDC
:10D49000006E7AAD08D03F0E05D02D0E006E99A11A
:10D4A00002D04B0E006E5BEC97F00101115102E1CE
:10D4B000100E116F002BA40E006EAAEC2DF07DEC67
:10D4C00094F0CB0E4A6EEA0E4B6E010E4C6EB6C156
:10D4D0004DF0EDECE5F0DEEFE7F03380A3ECE7F0A4
:10D4E0002096CDDF46EF4BF0339005EC0EF081EF48
:10D4F0006CF0AEECE5F089ECE9F01CE0FE0EDB50E0
:10D5000002E0350E01D0340EC6ECE5F0A6ECE9F0F1
:10D5100011E02150200B0EE0010E076E89ECE9F0BE
:10D5200008E0FE0EDB5002E0350E01D0340EC6ECF2
:10D53000E5F0076AB3EFE5F0E66AF9ECE9F0A50E6D
:10D5400043ECF4F08AEFF2F01AECF0F00701BC5172
:10D55000B15D14E11550100B01E0010E4A6E34501C
:10D56000010B4A5C0BE11550200B01E0010E4B6EE4
:10D570003450020B01E0010E4B5C2EE0076AB1C78C
:10D58000BCF7349015B83480349215BA348215A89B
:10D590001DD015AA16D089ECE9F010E00701B151B1
:10D5A000140D2DECE6F0C8DF01013EA907D0010EF5
:10D5B000076E89ECE9F001E0BFDF076A010EE66E55
:10D5C00006D0E66A96DFE552330E04D0E66A91DFB4
:10D5D000E552320EFFECE7F022EFF0F00701B15117
:10D5E000140D2DECE6F02DEC2EF01CC119F11DC12F
:10D5F0001AF11EC11BF11FC11CF10101200E1D6F8C
:10D60000480E1E6F5A0E1F6F300E195D02E1200E7C
:10D61000196FA4EF6AF0318C2096006848EC2EF068
:10D62000EEEF6AF0319C05EF0EF0095004E0255052
:10D63000080B01E130880D0E005C03E146ECF1F0CF
:10D6400009D00A0E005C03E151ECF1F003D0005068
:10D650000CECE7F0095006E03050100B03E1FA0E35
:10D66000096E25861200010E0701D8908337843792
:10D67000E806FBE122AC02D0070183810D0E070111
:10D68000855D01E2852B1200229C8650020B01E091
:10D69000228C07017B5111E122AC51D07B2B010E72
:10D6A000836F846B856F3198866F7E51FE0BE842E5
:10D6B0007E257D6F010124931200010124A33FD038
:10D6C000249307017B053BE122BC2BD031A826D057
:10D6D0000C0E855D20E2D89084338333000E835D89
:10D6E000040E845918E23A0E83254A6E020E8421F4
:10D6F00099ECF4F0E8ECE7F0006E090E005C03E151
:10D70000EAEC8AF008D0005006E0610E005C02E30B
:10D71000200E005E8ADF07017B6B1200318833EF39
:10D720006BF0A1DF31A804D00701010E866F06D08F
:10D730000701862B86510C0801E27B6B31981200A1
:10D7400008AE05D0229C8650020B01E0228C070116
:10D750007B5110E122BC76D00101249307017C6B40
:10D7600008AE70D0020E7B277E51FE0BE8427E256C
:10D770007D6F12007B050BE17B2B7EC77DF70101DE
:10D78000249322AC5FD00701080E7B6F12000101C9
:10D7900024A358D02493070E07017B5D47E17B6BE0
:10D7A00022AC41D0095004E02550080B01E130883B
:10D7B0007C514D6A3A0F4C6E060E4D227F5144EC5F
:10D7C000F0F0E8ECE7F0006E810E005C03E1070189
:10D7D0007F6B20D0800E005C04E10701200E7F6F7C
:10D7E00019D00D0E005C03E146ECF1F013D00A0EE7
:10D7F000005C03E151ECF1F00DD00B0E005C02E196
:10D800002A0E06D00A0E005C05E0005003E000502E
:10D810000CECE7F0095009E03050100B06E1FA0E6D
:10D82000096E25861200080E7B6F1200080E7B5DC4
:10D8300004E122AC07D07B6B12007C917C4322BCBC
:10D840007C897B2B120071EC94F0810E2CECE7F0BC
:10D850000C5008E10601F15105E10101002B640EB5
:10D860002CEFE7F0F2ECF2F0F1C600F0030E0C5CE6
:10D8700002E1F3C600F05BEC97F0050EE66E040ED5
:10D88000A3EFE8F0E0DF7DEC94F0030E0C5C14E114
:10D89000D1ECEFF006E0F30E4A6EF30E4B6E010E84
:10D8A00005D0EE0E4A6EF30E4B6E010E4C6E0DEC73
:10D8B000E6F04CC0E6FF0AD0BC0E4A6EEA0E4B6E94
:10D8C000010E4C6EF0C64DF0EDECE5F0DEECE7F04D
:10D8D0004CEC26F02AEC12F0006E00500A01D65DE6
:10D8E00004E200C0D6FA6AECF2F012003184A3EC34
:10D8F000E7F0209642EF6CF0319405EC0EF081EFEA
:10D900006CF048ECEEF0A00ECEECF0F0140E016ED0
:10D910003FC100F005EF4DF00FECF0F0E6C64AF025
:10D92000E7C64BF008ECEDF006015FECEFF00BE31F
:10D93000E4C64CF0E5C64DF0B5ECEFF0E6514C5CBA
:10D94000E7514D581FE2E451E6250F6EE551E721FE
:10D95000106ED89010320F3261ECEBF0030EDCEC5D
:10D96000F2F0FDE14A500601E85F4B50E95B80ECC4
:10D97000E8F0030EDCECF2F0FDE14A500601E82786
:10D980004B50E923E4C6E6F6E5C6E7F661ECEBF0BA
:10D9900008ECEDF008ECEDF05FECEFF00BE361EC80
:10D9A000EBF0BDECE8F0BDECE8F04A50E45D4B5024
:10D9B000E55902E2DF6A09D0E851E45DE951E55931
:10D9C00002E2010E01D0020EDF6E61ECEBF008EC1A
:10D9D000EDF04A50E825EA6F4B50E921EB6FDF503C
:10D9E000E552B3EFE5F0229C8650020B01E0228C59
:10D9F00022AC03D00201822B02D00201832B83517F
:10DA00007BECE9F001E14B5008E082514C6E4D6A2D
:10DA1000FF0E4C1822E14D5020E182517BECE9F0E1
:10DA20000DE14B500BE1815139ECE6F004E6FF0EBD
:10DA30004A5C000E4B5805E2812B03D0815101E076
:10DA400081070601F15105E181C2E6FFE20EC3EC58
:10DA5000E5F00201836B83C282F2209E0601EC5145
:10DA600009E122AC45D0010EEC6FE46BE56BED6B88
:10DA7000EE6B3ED0EC0515E122BC3AD0020EEC6F05
:10DA80004BDF006E00500BE0070E0601EE5D07E273
:10DA9000EE2BED91ED430050010801E2ED8F060100
:10DAA00019D0020EEC5D24E122AC17D061ECEBF052
:10DAB000030EDCECF2F0FDE106014A50E85D0F6E6A
:10DAC0004B50E959106E0F50E45D1050E5590EE2CD
:10DAD000010EEC6FE46BE56B0BD0EA51EA254A6E60
:10DAE000EB51EB214B6E5FECEFF002E2030EEC6FBB
:10DAF000030EEC5D68E1ED91ED43ED8F070ED880EC
:10DB0000EE55016E01500106000903E0ED91ED4371
:10DB1000F9D7780EED5D55E2095004E02550080B69
:10DB200001E13088EDC6E6FF67EC04F0E552006ED7
:10DB3000200E005C03E300506E0802E22A0E0BD0B8
:10DB40002A8A00500CECE7F00601E451EA5DE55149
:10DB5000EB5903E2200E0CECE7F0040E0601F05D39
:10DB600026E12AAA0CD0600E3E6E090E3F6EE8C672
:10DB700043F0E9C644F0B8ECFDF03EC0EFF6C2EC6D
:10DB80008AF0000914E00101390E1A6F1AC119F167
:10DB90006E0E1B6F640E0601EF5D07E24CECE6F0C3
:10DBA000EFC63FF003ECECF01A6F01011C8F2A9ACC
:10DBB000095007E03050100B04E12586FA0E096E7B
:10DBC00031860601EC6B208E12000101E4830C50BB
:10DBD00002E109DF07D0209E78ECEBF002E054DD93
:10DBE00001D0AEDD0101E4931200800E081419E0AB
:10DBF0002B50020B16E12150200B13E00201E051E3
:10DC000010E10C5004E10601F051010806E3030E97
:10DC10000C5C07E1D1ECEFF004E02A0E0101B21533
:10DC20000DE0800E081409E111ECE7F006E00601B2
:10DC3000F25103E002013D5101E0000C010C020130
:10DC40004C5103E1120EDBECE5F01200AEECE5F016
:10DC500006C201F007C202F02DA203D0020E85EC2D
:10DC6000E8F0A6ECE9F040E03A51800B3DE1020E0D
:10DC700085ECE8F002010A5139ECE6F002E6FCEC32
:10DC8000E7F015E20A514A6E4B6A800E32ECF2F070
:10DC9000036E03504E6E4F6A0250CBECE6F0070E57
:10DCA0000F0B03E0E0ECF2F0FDE14A50025E0201EE
:10DCB0000A51A1ECE6F018E24A508008000E4B54DD
:10DCC00013E20A5118ECEBF04A50036E03504E6E0B
:10DCD0004F6A0150CBECE6F0070E0F0B03E0E0ECCF
:10DCE000F2F0FDE14A50015E07C0C8F2076AFE0E7D
:10DCF000DB0409E00150E66EA60EC3ECE5F002017C
:10DD0000188335B09CDFFE0EDB5009E00250E66E52
:10DD1000BF0EC3ECE5F0020118851DB890DFC8C244
:10DD200007F0B3EFE5F0FAECF0F004E2E4ECE8F031
:10DD300001E2006AFAECF0F007E24A50E308000E54
:10DD40004B5402E2E30E006E005064ECEFF000244E
:10DD5000006EFAECF0F005E2E4ECE8F002E2FA0E14
:10DD6000006E1200B3ECF1F02E51635D03E1B65189
:10DD7000E9ECF0F081EF6CF0A6EC0DF0BCEC25F0D6
:10DD80006AECF2F0E6EC1CF0F9ECECF02050020B3F
:10DD900005E078ECEBF002E02EECECF0B9EC4BF0A7
:10DDA00005013B8712000FECF0F0E1EC13F088EC7A
:10DDB0005FF021AA07D00301E65102E0E60702D096
:10DDC000BEEC93F012DF000902E0FFDE01D0209EDE
:10DDD0002550200B06E00201345103E184EC5EF093
:10DDE000259AEEECE8F012E03450400B0FE101010F
:10DDF000CF51200B0DE0050140510AE08450040B87
:10DE000007E1445105E1280E446F02D00501446B3F
:10DE100002013B5102E079EC51F00101B45112E1F1
:10DE20002850010B0FE165EC34F0006E1EAC73EF6F
:10DE300078F00701D351F00BE83AD35D0024D36F9B
:10DE400073EF78F0B40515E12850010B12E163EC93
:10DE50008CF05AEC2FF0EEECE8F002E173EF78F082
:10DE6000F2ECE8F002E173EF78F0B2EC2EF073EF31
:10DE700078F0020EB45D09E12850010B06E14DEC8B
:10DE800014F0A0EC94F073EF78F0030EB45D07E1AA
:10DE90002FB473EF78F071EC98F073EF78F0040E14
:10DEA000B45D01E0B7D00201355102E073EF78F0C4
:10DEB0001850100B03E11850010B02E0000E01D0C6
:10DEC000010E2390E8B0238022AA4DD04FECEEF053
:10DED00023A036D00101A8511EE1175002E1010E26
:10DEE00001D0100E8009186E2850010B03E10E0EB0
:10DEF000165C05E10201030E286F640E226F28A054
:10DF000004D0480E67ECEFF03FD0F8EC09F00009C0
:10DF10003BE01B8439D0175003E00C0E175C34E152
:10DF2000810E186E175001E1229A0201020E356F20
:10DF300028A003D0540E67ECEFF00201286B24D028
:10DF4000175022E12350010B1FE1229A2850010BA8
:10DF500006E00C0E165C03E1520E67ECEFF00201D6
:10DF6000020E356F11D032B40FD0E66ADEEC51F0FC
:10DF7000E552000909E032840201020E356F640E99
:10DF8000416FE06B08AE356B3250040B02E173EF6A
:10DF900078F00201355102E073EF78F032944FECE3
:10DFA000EEF0175002E173EF78F00101280EA86F30
:10DFB0002A0E175C05E12150400B02E01E0EA86FEF
:10DFC0000A0E175C09E0090E175C06E0120E175CDA
:10DFD00003E0110E175C02E12D0EA86F350E175CE1
:10DFE00002E1FA0EA86F0201020E356F228A186A4A
:10DFF0001750166E28B005D0F8EC09F0000901E0C2
:10E000001B8429B602D00101AB6BA6EC0DF02B846A
:10E0100073EF78F0050EB45D0FE12951100B05E1A7
:10E020002A51100B02E179EC51F028A073EF78F03F
:10E030003FEC58F073EF78F0060EB45D07E121AACB
:10E0400073EF78F01BEC08F073EF78F0070EB45D17
:10E0500001E0B7D12650800B18E00201385115E1DC
:10E060006CECEFF002011E0E386F269E2850020B5A
:10E070000CE02A50010B09E1510E28ECE6F0300EBD
:10E0800028ECE6F0010E5CECF1F026AC03D0FEECDF
:10E09000E9F0269C26AA03D044EC0AF0269A010156
:10E0A0003951800B1BE00201485118E11BA404D038
:10E0B000040ECCECF1F01B941BA604D0070ECCECA4
:10E0C000F1F01B961BA804D0060ECCECF1F01B98C7
:10E0D0001BAA04D0050ECCECF1F01B9A2250080BC1
:10E0E00002E073EF78F02B50400B02E073EF78F012
:10E0F00002010B5139E1D70EB1ECE6F01F9A1FB0C7
:10E100001F8AE66801C2E6FF66ECEBF00201016FD0
:10E110001F901FBA1F801F50100B04E10101E65130
:10E12000080B22E028A006D001C2E6FF470EDBEC78
:10E13000ECF019D001C200F00101E6A703D0DDC365
:10E1400000F0E697030E005EFAECF0F004E2E4EC77
:10E15000E8F001E2006A00C006F23ABF02D000C057
:10E1600007F2E66A73DDE55202010B0548E1CF0EC6
:10E17000B1ECE6F01F9A1FB21F8AE66802C2E6FF02
:10E1800066ECEBF00201026F1F921FBA1F821F5054
:10E19000100B04E10101E651100B31E028A006D07C
:10E1A00002C2E6FF480EDBECECF028D002C200F021
:10E1B0000101E6A903D0DEC300F0E699030E005E7C
:10E1C000FAECF0F004E2E4ECE8F001E2006A00C0EE
:10E1D0000AF23AAF06D00201800E0A6F00C007F2C1
:10E1E0000AD0FAECF0F007E24A50E308000E4B5474
:10E1F00002E202010A69010EE66E28DDE552020E16
:10E2000002010B5D45E1E70EB1ECE6F01F9A1FB489
:10E210001F8AE66803C2E6FF66ECEBF00201036FBB
:10E220001F941FBA1F841F50100B04E10101E65117
:10E23000200B2EE028A007D003C2E6FF490EDBEC3E
:10E24000ECF0E55225D003C200F00101E6AB03D0AB
:10E25000DFC300F0E69B030E005E65DD00C008F240
:10E2600000501CECE9F0006EB7ECEBF00AE208C2DB
:10E2700009F20050E66EA70E4BECECF00201188993
:10E2800005D007C0C8F2076ABAECF2F0020118879D
:10E29000030E02010B5D01E08AD0EF0EB1ECE6F057
:10E2A0001F9A1FB61F8AB7ECEBF009E29E0EE66ECE
:10E2B00005C2E6FF66ECEBF00201056F07D0E668E9
:10E2C00004C2E6FF66ECEBF00201046F1F961FBA72
:10E2D0001F861F50100B04E10101E651400B67E05F
:10E2E00028A00CD0B7ECEBF003E205C2E6FF02D0A9
:10E2F00004C2E6FF4A0EDBECECF038D0B7ECEBF0F2
:10E3000037E2E0ECECF005C200F00101E6AD03D02D
:10E31000E0C300F0E69D030E005C0701056F0551A8
:10E32000A1ECE6F004E2E4ECE8F001E2056B05396B
:10E33000E8461F0B056F05511D0802E21D0E056F13
:10E34000050E0C5C03E0E1ECEFF003E18DEC0CF06A
:10E350002ED02150200B2BE00201415128E1010178
:10E3600059BD25D0130EE66E75EC2EF0E5521FD088
:10E3700004C200F0E6AD03D0E0C300F0E69D030E5A
:10E38000005ED1DCFAECF0F004E2E4ECE8F001E24B
:10E39000006A00C009F200501CECE9F0006E07C0F2
:10E3A000C8F2010E076EBAECF2F002011889030EF2
:10E3B00002010B5D01E12D920B2B030E0B1773EF86
:10E3C00078F0080EB45D02E0B4EF76F02850010B4F
:10E3D00002E0B4EF76F0B2BD3FD1B2A9E2D021AEF7
:10E3E0000FD0AA5101E0F6D02CA805D0D4C1E6FF89
:10E3F000B1EC53F003D0E66A07ECC7F0E552EAD07F
:10E4000025A03ED029AD7FD011EC09F00C500FE1D2
:10E41000500EE66E1E0EE66E2C0EE66E010ED5EC6C
:10E42000E5F001012C51E8240301D86F1CD009EC60
:10E43000E8F009E0030EE66E310EE66E010EE66EC0
:10E4400033EC9EF00DD0050E0C5C0DE1330ED1ECDB
:10E45000F4F0B30EE66E020EE66E29EC9EF0E55285
:10E46000E552E552E55221EC6AF06AECF2F0E6EC96
:10E470001CF002010A0E3C6F05013B853B8F43D027
:10E4800033A018D029AD13D009ECE8F003E0010166
:10E49000997105D078ECEBF002E001017A7DA6ECF1
:10E4A0000DF0BCEC25F04CEC26F03FEC6AF00101DD
:10E4B000299D5FD031A416D029AD25D011EC09F0EB
:10E4C0000C5006E1060EE66EF10EE66E060E05D065
:10E4D0001E0EE66EF30EE66E060ED0ECE5F042EC94
:10E4E0006CF011D030AA11D029AD0DD011EC09F08B
:10E4F000150EE66E07504B6A420F4A6E050E90EC01
:10E50000F0F072EC69F0010134D02D50400B03E1C2
:10E510002D50800B30E029AD5DD011EC09F00101E8
:10E52000B3511AE1630EE66E470EE66E010EA9ECDA
:10E53000E7F047C11FF202014E6B71ECE9F00009F0
:10E5400017E02D50800B14E001019151100B10E1E8
:10E550000201100E4E6F0CD0290EE66EB3054B6A09
:10E560004B0F4A6E060E90ECF0F06FECEFF0E552B8
:10E570000101AA6B2FD029A20DD029AD2BD011EC0F
:10E5800009F0E6686A0EE66E030ED0ECE5F095EC55
:10E59000C6F020D022B61ED06FC200F03DEC2EF0A7
:10E5A00019D0B2A305D026A215D02692238212D06C
:10E5B000B2A110D026A206D026922EC1E6FF1FECF3
:10E5C00043F0E5520201315105E11B50400B02E1DD
:10E5D00046EC4BF01CEC16F0006EFF083DE0420EDE
:10E5E000005C03E0450E005C15E129C70FF02AC767
:10E5F00010F0450E005C04E107012B510F6E106A0C
:10E6000000683DEC2EF00101150E116F030E006F36
:10E6100017EC2EF05D0E005C16E10101150E116F76
:10E62000100E126F020E006F2CC7E6FF08EC2EF0E2
:10E63000E5522DC7E6FF08EC2EF0E5522EC7E6FFA7
:10E6400008EC2EF0E5527E0E005C06E171EC94F0D1
:10E65000E80E006E3DEC2EF00101B2BF6BD3B2AB01
:10E660009CD12DA603D0B3EC54F04CD32DA403D0F1
:10E6700081EC54F047D331A424D02AAD17D0010E39
:10E680000E6E2ABF0E680C5005E148ECEEF033EC3C
:10E690009EF008D0010EE66EF20EE66E060EE66EF5
:10E6A00023EC9EF065ECF4F06AECF2F02450200BC1
:10E6B00005E101012A51400B01E17FD042EC6CF0F1
:10E6C0007CD033A01DD02AAD0DD0010E0E6E2ABF16
:10E6D0000E68B6C106F1030E2DECF5F006C1B6F1D9
:10E6E000B2EC6EF02450200B04E101012A51400BE2
:10E6F00064E0BCEC6EF03FEC6AF0020119815DD081
:10E7000025A00BD02AAD40D10201B57546EC4BF0E7
:10E7100021EC6AF001012A9D37D130AA19D02AAD27
:10E720000DD0010E0E6E2ABF0E68150EE66E075054
:10E730004B6A400F4A6E050E90ECF0F02450200B0F
:10E7400004E101012A51400B38E072EC69F035D048
:10E7500024AE19D02AAD0ED0010E0E6E2ABF0E685F
:10E7600068EC68F01F0ECDECF4F0010141ECEEF026
:10E7700006C1EFFF2450200B03E12A51400B1DE09E
:10E78000AEEC68F01AD031AC1CD02AAD0DD0010E21
:10E790000E6E2ABF0E68C40EE66E0A0EE66EB10E4D
:10E7A000E66E070ED5ECE5F02450200B04E10101E4
:10E7B0002A51400B02E0EEEC6AF001012A9D249AF6
:10E7C000E3D02D50400B03E12D50800B33E024AA01
:10E7D00004D0249A6FECEFF05ED02AAD93D22A9D3C
:10E7E000010E0E6E2ABF0E68006A26B4002A050EBE
:10E7F000CDECEFF0B30EE66E010ED5ECE5F00601C0
:10E80000030E426F0101B3510EE0B3294A6E010EAF
:10E810004A5204E0E846FE0B4A06FCE10601426F5C
:10E820001E0E436F02D035EC68F06FECEFF0E5524E
:10E830000101AAD029A214D024AA02D0249A0DD072
:10E840002AAD60D22A9D010E0E6E2ABF0E68E668C0
:10E85000690EE66E030ED0ECE5F095ECC6F052D2F0
:10E8600021AE1BD0AA5101E04DD2D4C101F023A8A2
:10E8700002D0C3EC83F0006A2C50100B05E1D9ECF8
:10E88000EFF002E2010E006E0050E66E0150E66EFF
:10E89000E1EC53F0E552E55235D21CA277D07DEC85
:10E8A00094F0140E76ECE9F0AFEC04F05A0ED88038
:10E8B0000054006E0050036E78EC97F00101200EBA
:10E8C0001D6F0201F251035C03E201012A0E1D6F6C
:10E8D00001012AAD58D02A9D9CEC0AF0E2EC0AF026
:10E8E000190E026E0101E4AF02D01A0E026E2ABFA9
:10E8F00009D06E0E02014A5F000E4B5B02504BECDA
:10E90000F2F008D06E0E02014A27000E4B2302508F
:10E910001DECF2F04A514B1106E0280ED8804A5502
:10E92000230E4B5519E201012ABF0AD00201280E1D
:10E930004A6F230E4B6FF0C20FF0F1C210F00CD0F3
:10E940006E0E02014A6F4B6B02501BECE8F0F05D5B
:10E950000F6E4B50F159106E0301D2510F5CD35121
:10E96000105804E2D6510F26D75110220F50D45D13
:10E970001050D55904E2D6510F5ED751105AAEEC63
:10E98000ECF00CEC0BF00101AA6BBCD122B6BAD1B1
:10E9900070C200F048EC2EF0B5D1B2B3B3D1B2A73B
:10E9A00016D07DEC94F00A0E006EBFEC2DF0010144
:10E9B000040E016F03C700F01AAC02D0AFEC04F0F4
:10E9C00078EC97F01AAC9ED10101200E70D13E5127
:10E9D000200B01E17ED12E50400B01E07AD1060ED2
:10E9E000006E2DA502D00A0E006E0050D880795519
:10E9F00001E2796B2AAD1FD02A9D010E0E6E2ABF4F
:10EA00000E680050E66E790EE66E010ED0ECE5F071
:10EA1000050E0101795D0BE12B50200B03E02B501B
:10EA2000010B05E02ABF02D0792B01D07907020142
:10EA3000FD6B0101AA6BAA5101E064D12150200BAA
:10EA400001E160D10201E05101E05CD10A0E010157
:10EA5000795D3FE17DEC94F0C4EC18F001012B0EE0
:10EA6000196F000110AE0BD001012D0E196FFF0EB2
:10EA7000D8800F561056010E0F26000E1022E70EFA
:10EA800041ECEFF004E2E70E0F6E030E106E0F5034
:10EA9000101003E10101200E196F80ECE8F0640E04
:10EAA00036ECF3F04A50006E0101012B78EC97F040
:10EAB000A5EC04F0300F01011A6F300E1A5D02E16F
:10EAC000200E1A6F1C8F640E1D6F420E1E6F560EA5
:10EAD00055D0090E795D1EE17DEC94F0B8EC18F08C
:10EAE0002DEC2EF00101410E196F460E1A6F560ED5
:10EAF0001B6F300E1C5D01E005D1200E1C6F300E27
:10EB00001D5D01E0FFD055ECEFF001E0FBD0200EE1
:10EB10001E6FF8D0050E795D03E0060E795D30E1D9
:10EB20007DEC94F00101500E196F410E1A6F050E25
:10EB3000795D03E1DDC700F006D0460E196F500E77
:10EB40001A6FE2EC14F000AE04D0006C01012D0E3F
:10EB50001B6F0101030E016F78EC97F0300E01017D
:10EB60001C5D0BE11BC11CF1200E1B6F300E1D5DE7
:10EB700004E11CC11DF1200E1C6F430E1F6FC2D09B
:10EB8000070E795D04E0080E795D01E077D07DEC39
:10EB900094F00101500E196F4C0E1B6F1BC11AF13E
:10EBA000310E1C6F07C0C8F2070E795D02E1076ADB
:10EBB00003D01C2B010E076E95EC3CF0C8C207F089
:10EBC00001017AA73BD07DEC94F0E60EE66EF30EE1
:10EBD000E66E010EE66EDEECE7F0080E0101795DEF
:10EBE00001E11C2B07C0C8F2076A080E795D02E13B
:10EBF000010E076E530E4FECEBF0005003E10201E3
:10EC0000FD5119E0005006E00201FD51005C02E0F8
:10EC100000C0FDF201012A0E1D6F0201FD390F0B2C
:10EC2000E5ECECF001011E6F0F0E0201FD15E5ECA5
:10EC3000ECF001011F6FC8C207F064D00050150D41
:10EC40002DECE6F080ECE8F0060EDCECF2F0FDE1F5
:10EC50004A50006E0050DF6E0201345153E15CEC0B
:10EC6000EAF00101200E1D6FDF50480803E3040E97
:10EC7000DF5C02E22A0E1D6F1F8F44D0020E795D09
:10EC800005E108EC53F0010E096E3CD0030E795DEE
:10EC900010E17DEC94F01EC200F078EC97F0300E9D
:10ECA0000101195D02E1200E196F1B8F560E1D6FB9
:10ECB00029D0040E795D03E1BFEC12F023D0795125
:10ECC00003E18CECC5F01ED079051CE1BCECC5F06D
:10ECD00019D002012A510AE02850400B13E1140E0A
:10ECE000095C10E2810E48ECE6F00CD00101B2A103
:10ECF00009D024AA03D0249ACCEC43F02EAC02D045
:10ED000046EC4BF01CEC16F0006EFF0813E07E0E94
:10ED1000005C0CE1006848EC2EF0DE0EE66EF30EAF
:10ED2000E66E010EE66EDEECE7F004D00050006EF9
:10ED300048EC2EF00101AA5101E0D5D1140EAA6FC2
:10ED400002016B5101E06B07020E7E5D01E0CBD149
:10ED5000CD0E0B5C07E0B30E0B5C04E0A10E0B5C68
:10ED600001E0C1D12682BFD1090EB45D03E125ECDB
:10ED700051F0B9D10A0EB45D08E12850010B05E14C
:10ED80005BEC96F03EEC96F0AED10B0EB45D01E07C
:10ED9000AAD12850010B01E0A6D1B55110E1C1EC78
:10EDA00014F09050800B01E198D19050400B01E19C
:10EDB00094D1909C1E0EE66EF9EC15F08DD1B50540
:10EDC00011E1800E08140BE13B51040B01E085D1E9
:10EDD0002E51070804E22FECE7F001E07ED10CECA5
:10EDE00005F07BD1020EB55D4AE11DEC14F0070180
:10EDF000DC0ED880DB55000EDC5501E36ED12FEC24
:10EE0000E7F001E16AD1DBC70FF0DCC710F0016A5F
:10EE1000030E015C09E21DEC14F00701DB510F2623
:10EE2000DC511022012AF4D7020E0F0B05E0D89016
:10EE300010320F32E806FBE1DC0E24ECE7F001E3D0
:10EE40004CD1D70EE66EF30EE66E010E56ECEEF0E8
:10EE5000010E006EF00E24ECE7F002E2050E006EEB
:10EE6000D9ECEFF004E200504B5F63ECE9F0780E70
:10EE700001014B5D01E331D184EC0FF02ED1030E83
:10EE8000B55D03E16DEC0FF028D1040EB55D57E1DF
:10EE900021AC2AD003016C0ED8806355000E645556
:10EEA00017E22FECE7F014E0D00EE66EF30EE66EFC
:10EEB000010E56ECEEF00201640E2D6F5AECEEF0EE
:10EEC00003E0E0ECF2F0FDE172ECECF0E5EC0BF0CD
:10EED0003250010B09E002018951070805E2145084
:10EEE000080B02E0640E436F2150400B01E0F5D0A7
:10EEF00002013B5101E0F1D001015951200B01E029
:10EF0000ECD0F00E8C1625AE287E28AE02D0030E73
:10EF10008C1267EC0CF000090DE067EC0CF00009B6
:10EF200009E067EC0CF0000905E0258E150EDBEC1E
:10EF3000E5F002D025BE259EF00E8C16CED0050E33
:10EF4000B55D34E1060150932550020B12E12050CB
:10EF5000020B04E0CAEC31F0000909E01350080B81
:10EF600003E11350040B05E0D7ECEEF002E00601DC
:10EF700050832550020B01E0B0D0AFECEBF001E084
:10EF8000ACD00201405101E0A8D078ECECF001E1F6
:10EF90004B5001E1A2D02D50800B01E09ED02D50AE
:10EFA000400B01E09AD00601108197D0060EB55DA6
:10EFB00045E15951040B40E02050080B3DE0DF0EC5
:10EFC000B1ECE6F02BBC24D08BECF1F002E6D4ECF3
:10EFD000EEF001E382D01E0E3EECE6F0DF0EB1EC67
:10EFE000E6F00050016E050E3EECE6F0DF0EB1ECEF
:10EFF000E6F0030EE66E0150CDECEFF09DECE7F08D
:10F000006CE02B8C45EC0CF002013C0E466F65D099
:10F01000FAECF0F00BE24A50B908000E4B5406E24D
:10F020002B9C1E0EE66E36EC29F056D0020146519E
:10F0300054E145EC0CF051D02B9C4FD0070EB55D40
:10F040004CE1EEECE8F049E02150200B46E0F1EC19
:10F05000F4F0C09EF00E8C160F6A106A01013EA9F2
:10F0600003D01E0E0F6E106A80ECE8F0FA0ED88006
:10F070004A56000E4B56C3504A5CC4504B582DE2C2
:10F080000201ED2BED51030828E2ED6B01015AADB1
:10F0900007D05A9D0FEC9CF077EC1EF0160E19D09D
:10F0A0000750DF6E076A02010691064306C2E6FFBB
:10F0B000A60EC3ECE5F001013EA908D002010791BC
:10F0C000074307C2E6FFBF0EC3ECE5F0DF50076E53
:10F0D000170EE66E75EC2EF0E5520101B52BB55119
:10F0E000070801E2B56B0101B42BB4510B0801E232
:10F0F000B46BE552B3EFE5F0016A700E015C0EE20D
:10F100003B0E4A6EEF0E4B6E010E4C6E01504D6E73
:10F110004EECF5F018ECEAF0012AEFD71200026A83
:10F12000300E025C08E2B00E0224016E0A0E18ECEA
:10F13000EAF0022AF5D712000FECF0F07A0E6DEC2F
:10F14000E9F03BEC96F0010E0A6EDF6A100EDF5C10
:10F1500035E2026A100E025C2FE201ECF1F003E0EE
:10F16000050E025C06E1DF50E824860F43ECE6F072
:10F17000006E020403E0060E025C07E1DF50E824A3
:10F18000860F010F43ECE6F0006E020EDF5C06E333
:10F19000030EDF5C03E00A0EDF5C0AE10A0E025C8C
:10F1A00002E1110E006E0B0E025C02E1240E006EF5
:10F1B00005EC4DF0022ACED7DF2AC8D7AC0E016E7F
:10F1C000580E18ECEAF0020E0A6EDF6A090EDF5CD8
:10F1D00012E2026A100E025C0CE201ECF1F003E0B4
:10F1E000050E025C02E11C0E006E05EC4DF0022AD9
:10F1F000F1D7DF2AEBD70A6A7FDFDF6A200EDF5CF8
:10F2000009E2100E006E800EDF24016E05EC4DF059
:10F21000DF2AF4D7DF6A0B0EDF5C03E280DFDF2A30
:10F22000FAD7DF6A090EDF5C31E2DF28006E0038B2
:10F23000F00B006E090E0012DFCFE6FFF5EC0BF0CD
:10F24000E5525CECF3F0EE52090E38ECF4F0B3EC5E
:10F25000ECF02C0E38ECF4F0030ECAECF0F0010EDA
:10F2600038ECF4F0040E7FECF1F0050E7FECF1F0D9
:10F27000070E7FECF1F0080E7FECF1F0060E7FEC4C
:10F28000F1F0090E5AECE9F0DF2ACCD719D823D8CF
:10F29000DF6A060EDF5C07E2DF50A5ECE6F0010E48
:10F2A000EF6EDF2AF6D790ECF4F0FD0E016EDB0E68
:10F2B00018ECEAF00101010EB26FE552B3EFE5F090
:10F2C000020E0A6E5A0EE66E000EE66E030EE66E33
:10F2D000A20E29EFF5F0730E6DECE9F03BEC96F021
:10F2E000140EEFECEFF0000EE66E0A0E9CECE6F06A
:10F2F0000A0EEFECEFF0CA0EE66E0A0E9CECE6F09A
:10F300000C0EE66EE66A010EE66E140EE66E0A0E4E
:10F310009CECE6F00A0EEFECEFF0200EE66E0A0E23
:10F320009CECE6F00A01D46BDA6BDA81D56B380E0F
:10F33000D66F040ED86F3C0ED96F190ED76F016AC5
:10F34000020E015C0CE20150050D02ECF4F0000E1F
:10F35000E9260A0EEA22360EEF6E012AF1D70C6A70
:10F36000050E0C5C1AE20701010EE26FFF0EE25D72
:10F3700012E0C0EC15F07DECEDF04FECF2F00C502B
:10F3800028ECF2F00701E251B6ECF4F048ECE8F0BA
:10F390000701E207EBD70C2AE3D70701E26B0C6AFF
:10F3A00005EC5FF00EEC5FF0030E0A6EFE0E016ED0
:10F3B000810E18ECEAF00A6A1200240E01014103E2
:10F3C000F350E66EE66AE1ECFBF0E552E55201012E
:10F3D0004351E8240A0FE66EE66A10ECFCF0E552B1
:10F3E000E5520C0EBD6E006A010141510AE0020EA9
:10F3F00042254103F3504A6E4B6AFF0E32ECF2F0A5
:10F40000006E0050BE6E1200AEECE5F04FECE6F080
:10F410000DECFDF0E552000902E0C69EF7D7B3EF10
:10F42000E5F0C79EC698C78C1200C78EC688C78CE9
:10F43000120084EC5EF02DA003D0210E7BECE6F0F0
:10F4400007010B8784EC5EF084EC5EF084EC5EF0E8
:10F4500007010B972DB003D0270E7BECE6F084EC70
:10F460005EF007010B8584EC5EF007010B952DA083
:10F4700002D00101E88984EC5EF00701128584EC7A
:10F480005EF0070112952DB003D0330E7BECE6F051
:10F4900084EC5EF007010F8F84EC5EF007010F9F94
:10F4A0002DB00DD00F8B84EC5EF007010F9B2DA0CB
:10F4B00003D00101E88B03D0240E7BECE6F084EC52
:10F4C0005EF007011F8984EC5EF007011F99228816
:10F4D0002DB003D06C0E7BECE6F084EC5EF0010105
:10F4E0002DA11FD00701108784EC5EF00701109753
:10F4F0002C842DA004D001017AAB11D00DD00101D4
:10F500007AAB0AD00701108F84EC5EF00701109FE0
:10F510000101E7812DB003D0630E7BECE6F084ECB3
:10F520005EF001012DA70ED007010D8784EC5EF07F
:10F5300007010D9720802DB003D02A0E7BECE6F05A
:10F5400084EC5EF001013D510EE00701168184EC70
:10F550005EF0070116912C862DB003D0660E7BEC71
:10F56000E6F084EC5EF001013C510EE00701138FE0
:10F5700084EC5EF00701139F2B8A2DB003D0690E37
:10F580007BECE6F084EC5EF001013AA73BD02588E5
:10F590000701078584EC5EF0070107952DB003D0C5
:10F5A0002D0E7BECE6F00701068384EC5EF007018C
:10F5B000078384EC5EF0070107930101EE932DB001
:10F5C000EE8384EC5EF0010162A50ED0070109878D
:10F5D00084EC5EF00701099731822DB003D0300E24
:10F5E0007BECE6F084EC5EF00701208984EC5EF0B1
:10F5F0000701209931802DB003D06F0E7BECE6F02F
:10F6000084EC5EF084EF5EF0D9CFE6FFE1CFD9FF66
:10F61000030EE126020EDB6A83EC12F00F0EC16EC0
:10F62000000000000000000000008D8C219A34864C
:10F630000201800E8B6FD5EC15F00601BA6B800EBF
:10F64000BB6F41EC0EF00A6AFB0E016E44EC4DF00C
:10F6500000C0F1F707010E6B07010F6B0701126B7A
:10F660000701206B20C71FF70701470E186F18C747
:10F6700017F70201A169A2690701010E066F0701D0
:10F68000076B84EC5EF084EC5EF00301310EE36FF7
:10F690000701090E326F32C731F732C730F732C770
:10F6A0002FF70701070E516F0301A00ED06F0F0E49
:10F6B000D16FE50EE66EECECFCF0E552E6683FEC4F
:10F6C000FCF0E552E668A9ECFCF0E552E66887EC50
:10F6D000FCF0E552050EE66E2BECFDF0E552010163
:10F6E000050E416F0101030E426F01010B0E436FC6
:10F6F00064DE850EE66ECBECFCF0E5520201320EC4
:10F70000256F000EA56EA26E9F6EA282D08EE66A55
:10F71000040EE66E210EE66E78ECFBF0E552E55243
:10F72000E552010EDB6A100EF36E010EDBCFF4FF23
:10F73000F350F45C28E20D0E4A6EF00E4B6E010E93
:10F740004C6E010EDBCF4DF04E6A4F6A4A504D248D
:10F75000F36E4B504E20F46E4C504F20F86EF4CFA9
:10F76000F7FFF3CFF6FF0800F550E66E010EDB5011
:10F77000EA6AC90FE96E060EEA22E552E750EF6E1B
:10F78000010EDB2AD0D70101296B01012991885094
:10F79000010B01E02981010129938850020B01E04E
:10F7A000298301012A918850200B01E02A8101015F
:10F7B0002A938850100B01E02A830101EE87F28E14
:10F7C0000601526952C650F625EC51F03CEC99F016
:10F7D0000101C30EAF6FED0EB06F010EB16F0601E8
:10F7E000526B52C650F625EC51F00101010EB26F7A
:10F7F00071EC94F07DEC94F0D3EC8AF00601178163
:10F800000601416941C640F60601426B148A138025
:10F8100012881282148614880A01380ED66F0A01E3
:10F82000010ED76FC0EC1EF03EEC96F0010EE66EB6
:10F83000DEEC51F0E552176E380E175C0AE101015B
:10F840003B89010EE66EDEEC51F0E552000901E065
:10F85000F8D7C80EE66E46ECFDF0E5520701D76B0F
:10F86000358E100EE66EE66AE668000EE66E090E4C
:10F87000E66ED6EC4DF04A6E050EE15E4A50359EBE
:10F8800041EC0EF00A6AFC0E016E44EC4DF0001CD7
:10F89000DF6EFC0E016EDF50006E05EC4DF0FC0ECD
:10F8A000016E44EC4DF0DF50005C06E0180EE66E91
:10F8B000F9EC15F0E5525AD0830E0A6EFC0E016E7B
:10F8C00044EC4DF0001CDF6EFC0E016EDF50006E4C
:10F8D00005EC4DF0FC0E016E44EC4DF00A6ADF5071
:10F8E000005C06E01B0EE66EF9EC15F0E5523ED02A
:10F8F000FD0E016E44EC4DF0DB0E005C03E13A0EB0
:10F90000175C07E119DC010EF36E020EF3CFDBFF8B
:10F9100024D0020E016E44EC4DF000C02DF1370EE4
:10F92000016E44EC4DF000C062F1110E016E44EC2A
:10F930004DF000C03CF1120E016E44EC4DF000C0E1
:10F940003DF10F0E016E44EC4DF000C03AF14F0E48
:10F95000016E44EC4DF000C07AF1B00E016E44EC43
:10F960004DF00050800802E28FEC78F0010E076E37
:10F97000010EE66E67EC3BF0E5528CEC36F0E6C229
:10F98000E6FF010EE66E1FEC38F0E552E552076A1D
:10F99000010EE66E67EC3BF0E5528CEC36F0E5C20A
:10F9A000E6FF010EE66E1FEC38F0E552E55201016C
:10F9B0003AB717D0E66AD0EC18F0E552040EE66EBE
:10F9C000D0EC18F0E552010EE66E46ECFDF0E55283
:10F9D000E66AD0EC18F0E552280EE66E46ECFDF033
:10F9E000E55232880701580E8F6F020E906F0701A3
:10F9F000BC69A6EC0DF0FCEC23F001013AA709D09C
:10FA0000010E076EA6EC0DF0FCEC23F0076AA6ECE5
:10FA10000DF084EC5EF0F29EC4EC4EF00201006F3B
:10FA2000000916E0C80EE66E46ECFDF0E552C80E81
:10FA3000E66E46ECFDF0E552C4EC4EF00201006FBC
:10FA4000000906E07E0EE66EF9EC15F0E55235820F
:10FA50005EEC99F00701F10517E00301010ED96F83
:10FA60000301DB6BE6DC0301DB5105E0C80EE66E4B
:10FA700046ECFDF0E5520301DB5106E00301D92B12
:10FA8000040E0301D95DECE3D9C3DAF30301D96BAA
:10FA9000F28E2A9E2BBA2A8E0101E295FD0E926EFD
:10FAA0000A0EE66E36EC29F0E55292688F0E006E73
:10FAB00060EC2DF0005010080EE20A0EE66E36ECF7
:10FAC00029F0E5528F0E006E60EC2DF0005010080A
:10FAD00002E20101E2850601D9918850800B01E024
:10FAE000D9810601D9938850400B01E0D98379EC84
:10FAF00051F020860001126A136A146A156A2D8279
:10FB0000800E086E186A229A700EE66EE66A2B0E58
:10FB1000E66E010EE66E6EEC4DF0E552E552E552F2
:10FB2000E552020E0A6E5A0EE66EA20EE66E000E48
:10FB3000E66E030EE66E6EEC4DF0E552E552E552D0
:10FB4000E552030E0A6E2A0EE66EE66A000EE66EB7
:10FB50000A0EE66E6EEC4DF0E552E552E552E552C6
:10FB6000AA0EE66E300EE66E2A0EE66E0A0EE66EFF
:10FB70006EEC4DF0E552E552E552E552FE0E016E97
:10FB800044EC4DF00A6A810E005C02E06BEC79F007
:10FB9000060EE66EF00EE66EE90EE66E070EE66EF7
:10FBA0006EEC4DF0E552E552E552E552040EE66E7C
:10FBB000A00EE66EF00EE66E060EE66E6EEC4DF0F2
:10FBC000E552E552E552E5520601F051040802E221
:10FBD0000601F06B0601F251010802E20601F26B28
:10FBE000200EE66E800EE66E910EE66E070EE66E55
:10FBF0006EEC4DF0E552E552E552E552060EE66E2A
:10FC0000EA0EE66E350EE66E050EE66E6EEC4DF013
:10FC1000E552E552E552E552830E0A6EF90E016E89
:10FC200044EC4DF000C087F202018751DA0803E28C
:10FC30000201DA0E876FF80E016E44EC4DF0349A33
:10FC40006E0E005C01E1348ADF0E016E44EC4DF073
:10FC50000101E291720E005C02E10101E2817E0E7F
:10FC60000A6E0C0EE66EE66AEE0EE66E020EE66EAA
:10FC70006EEC4DF0E552E552E552E5520A6A020E8D
:10FC8000DB5013E099EC09F0BB0ED8800F54200E26
:10FC9000105402E201017A890F0ED8800F54270E0A
:10FCA000105403E20101040E466F01017A9701012D
:10FCB000E885530EE66EADEC42F0E552001C810B78
:10FCC00005E0BA0EC95C02E101017A870101E895FD
:10FCD0000301DC69D2EC0DF0010190AB02D001010F
:10FCE0003F9FFF0E0201F35D03E10201640EF36F1B
:10FCF00001013AB702D001013E9901017AA703D070
:10FD00000101050E5E6F0501355150080EE2050137
:10FD1000280E386F38C535F50501050E396F39C520
:10FD200036F505013A6B3AC537F501018E510A08DF
:10FD300002E201018E6B180EE66EE3EC15F0E5525F
:10FD4000000908E10301DA5101080DE2040E030184
:10FD5000DA5D09E20101050E416F0101030E426FF8
:10FD600001010B0E436FDDEC79F044EC0AF0E66A1A
:10FD7000BBEC0EF0E5520101E28301012C51E824B5
:10FD80000301D86F01017AA703D003010A0EE36FC4
:10FD9000FBEC28F00401300EF76F01015AAB03D0E1
:10FDA0000401310EF76F04013B0EFE6F0501006B7D
:10FDB00000C502F500C501F50501800E056F0701BC
:10FDC0000C0E346F0701DD0E356F0701320EB16F77
:10FDD0000101D36B0C6A0701E26B010EE66E88EC41
:10FDE00091F0E5520701EF81076AA6EC0DF0E5C23C
:10FDF000E6FF010EE66E1FEC38F0E552E55252ECDC
:10FE000024F001013AA715D0010E076EA6EC0DF003
:10FE1000E6C2E6FF010EE66E1FEC38F0E552E55251
:10FE200052EC24F0076AA6EC0DF001016585E1ECC7
:10FE300023F03BEC25F01A940101E49F01012DAD64
:10FE400018D009EC27F00F5010100EE00F0E0F5CC9
:10FE5000270E105809E21A84680E0F1801E110509D
:10FE600002E10101E48F05D0600EE66EF9EC15F0B9
:10FE7000E5521AB402D0010199950301B00ED26F78
:10FE80000A0ED36F0301AD0ED46F120ED56F0301AE
:10FE9000FE0ED66F070ED76F0101E4AF0FD003013E
:10FEA000540ED26F070ED36F0301910ED46F0F0E55
:10FEB000D56F03013E0ED66F080ED76F4DEC05F0DF
:10FEC0002680E66842EC47F0E55283EC28F0010119
:10FED000B281D7EC2CF082D975EC38F00201320EE9
:10FEE000346F0101040EB76F0101A30EB86FB7C1E3
:10FEF0000BF002016E2B0201320E326FE66A23EC28
:10FF000091F0E55285ECC4F0DFECC4F08BECB6F078
:10FF10000301DA51010819E2040E0301DA5D15E26A
:10FF200000685FEC2EF0C80EE66EF30EE66E010E72
:10FF3000E66E24EC98F0E552E552E552030E03011B
:10FF4000DA5D03E10101330E1F6F030EE15C02E293
:10FF5000E16AE552E16EE552E7CFD9FF12009A0E51
:10FF60000B5C03E30B509D0801E2000C010CE20E58
:10FF70000B5C03E30B50E70801E2000C010C0101EC
:10FF80003E7B3EBB04803BEC0AF001012A9D286BBE
:10FF900012000FECF0F065ECF2F00101460E196F63
:10FFA0004C0E1A6F310E0A01D52501011B6F97EC1B
:10FFB00004F072ECF1F000507BECE9F004E14B50FE
:10FFC00002E173ECEFF0A0EC04F0006E3A50DF6E4B
:10FFD0005CECEAF001011F8F300E1D5D07E11EC1D0
:10FFE0001DF11FC11EF1300EDF241F6FE552B3EF6C
:10FFF000E5F00A01D6513DEFF5F0AEECE5F0016A0F
:020000040001F9
:10000000012A0A01D52BD551040801E2D56B6DEC0C
:10001000EDF00DE0050E015C0AE278ECEFF004E093
:10002000E846FE0BE706FCE10701E115E9E04FECCD
:1000300096F084EC5EF04AECEBF0FE0EDB5002E052
:10004000C0EC15F0E66A88EC91F0E552075002E04A
:10005000D5CAB2F252ECE7F01BE0D3EC09F000098C
:1000600017E102017E5114E107500DECF1F0016E31
:100070000150A1ECE6F00CE24A503808000E4B5457
:1000800007E2720EA3ECE9F0FA0E096EFE0EDB6ACF
:10009000FE0EDB0403E17DDF640E096EB3EFE5F0D5
:1000A0000C50006E005003E0030E005C1BE100509A
:1000B00005E10101CF7DCFAD0ED007D009ECE8F00E
:1000C00006E00101CF75CFA506D0048004D0010160
:1000D000CE75CEB504803BEC0AF0B9EC4BF0E6EC03
:1000E0001CF016D0000403E0020E005C11E1C0EC2D
:1000F00015F0000402E1020E01D0010E006E020EA6
:10010000005C01E104803BEC0AF000500C6E27D843
:10011000F9EFECF001013E51080B03E068ECE6F06A
:1001200002E0000E01D0010E1592E8B0158268ECD5
:10013000E6F004E101013F51800B0CE168ECE6F0D0
:1001400007E011ECE7F004E101013E51800B02E110
:10015000000E01D0010E1590E8B0158012000C5071
:10016000006E0050800802E2050E006E060E005C74
:1001700001E3006A000402E10101CE91020E005C7D
:1001800002E10101CE8100500C6E258A21BE0AD009
:1001900048EC15F052ECE7F002E095EC05F0E6ECE7
:1001A0001CF002D0B9EC4BF0BBEF2CF00FECF0F0F0
:1001B000030EDF6E010191BDDF6A4C514A6E4B6A3E
:1001C000B00E3E6E040E3F6E59ECE6F03E50D88005
:1001D000DF540201656FE552B3EFE5F00FECF0F08C
:1001E00027B012D0320EDF6E010191AD02D0640E45
:1001F000DF6E080E4C5D02E2080E4C6FDF50D880B7
:100200004C5502E2DFCF4CF1D1DFE552B3EFE5F020
:1002100065C2ADF123AE3AD0006A010140510C082D
:1002200003E3050E405D02E2090E406F050E405DDE
:100230004E6E4F6A02016551CBECE6F0140EB4EC41
:10024000E6F03EC04AF04A50006ED6ECF1F00101F3
:10025000AD514C6E4D6AFF0ED8804C56000E4D5677
:100260004B504D18E8AE02D04D3404D04C504A5C8F
:100270004D504B580BE20050D880AD5507E224A0FA
:1002800003D00050AD2702D00050AD5FA9ECEFF0D5
:1002900008E102013D510601F01106E02850400B33
:1002A00003E11E9257EC50F01200050EA3EFE9F0A7
:1002B000FCDF268E1200180EDBECE5F0268E120015
:1002C000AEECE5F0050EE12620A20FD0BEC1DFFFA7
:1002D000010EBFC1DBFF020EC0C1DBFF030EC1C1B7
:1002E000DBFF040EC2C1DBFF0ED0B9C1DFFF010E80
:1002F000BAC1DBFF020EBBC1DBFF030EBCC1DBFFDB
:10030000040EBDC1DBFF2FECE7F01BE00101E4BDF3
:1003100007D0DF50180815E21C0EDF5C12E245D052
:10032000190EDF5C42E01A0EDF5C04E1010EDB50C7
:100330005F083BE31B0EDF5C04E1290EE4ECE5F013
:1003400034E32C50100B14E1070EDF5C0EE1010EBC
:10035000DB50360803E22FECE7F027E1010EDB501B
:10036000400803E22FECE7F020E0080EDF5C1DE020
:100370002C50100B06E12F50800B03E0AAECE9F0A3
:1003800002E2F36A17D0790EE66E020EE66EC6EC54
:10039000EEF096ECE8F009E1C6ECEEF0740EE66ED5
:1003A000020EE66E96ECE8F004E085DF010EF36ED7
:1003B00001D0F36AF46A050EE15C02E2E16AE552FB
:1003C000E16EB3EFE5F065C301F023A802D075C379
:1003D00001F00E0E015C01E2010C100E015C01E265
:1003E000020C120E015C01E2030C140E015C01E22E
:1003F000040C160E015C01E2050C1B0E015C01E20F
:10040000060C220E015C01E2070C080C35B603D085
:100410007EECF0F017D0A70EB3ECF2F0016A006AA0
:100420000050D880015402E20150006E1AECFEF038
:1004300015ECFEF00009FCE1C450016E0050D880BC
:100440000154EEE32CA802D0005010D00050020856
:1004500002E2020E005E460E005C0BE2F50E4A6EF2
:10046000EE0E4B6E010E21ECF1F0F5500F6E106A9E
:1004700012000050020D2DEFE6F0F00E8C160490E5
:1004800035B80480B5ECE8F006E12350100B03E02A
:10049000010E3EECE6F0BADF0FC061F310C062F36C
:1004A00035B81200F00E8C16030E8C1214A637D03D
:1004B000D4C101F023B867D9050E01244A6E0A0E93
:1004C0007BECE7F03F50016E015005E12350400BFB
:1004D00002E0010E016E68ECE6F003E03550400BDF
:1004E00005E001C0D5F702010A0E08D00701D55179
:1004F000015C05E301C0D5F702010C0E3A6F63DF22
:100500000701D66F2C50100B04E137EC0FF00009F7
:1005100002E00701D66B1FECEBF045ECE9F01FECB5
:10052000E8F00480005009E03550400B06E1030E6E
:10053000005C04E110ECEAF001E10490070E016EAA
:100540003250010B03E10450010B04E0CD0EF7EC37
:10055000E7F0016E0F0E01140201896F32B002D074
:10056000070E891701380F0B016E04A0016A14A44D
:1005700008D0020EE66E89C2E6FF0150E66E45EC39
:10058000E9F02CA80AD001014D510F6E106AE10E5E
:10059000D8800F56000E105617D0D9ECEFF00CE2B1
:1005A00060510F6E106A770ED8800F56010E1056EC
:1005B00009ECEFF0FDE108D055510F6E106A430EC3
:1005C000D8800F56010E1056006A0301FF0ED88026
:1005D0006155000E625501E2002A005061C34CF0E3
:1005E00062C34DF005E0D8904D324C32E804FBE197
:1005F00061C33EF062C33FF06EECF2F062ECF3F0E8
:1006000075ECF1F00FC043F010C044F097ECF0F03F
:100610000050E85003E009ECEFF0FDE10FC0D4F129
:10062000FA0E24ECE7F003E20101FA0ED46F310E6A
:100630000101D45D03E0330ED45D02E1320ED46FCC
:10064000630ED45D03E0650ED45D02E1640ED46FE9
:100650001FECE8F0040E005C23E1100E016E015067
:100660004A6E4B6AE9C23EF0EAC23FF059ECE6F04E
:100670003EC0EBF20101D4511BECE8F00201E92786
:100680004B50EA23EB514A6E4B6AE9514A5CEA51FE
:100690004B5806E2EB511BECE8F0E95F4B50EA5B8C
:1006A000000406E0020E005C03E0030E005C08E1BB
:1006B0000201EC510101D880D45502E2D4C1ECF220
:1006C000B5ECE8F006E12350100B03E0010E3EEC20
:1006D000E6F09CDE0FC063F310C064F3F00E8C16DE
:1006E00003016151635D6251645906E3010E6325A4
:1006F000616F000E6421626F61516325676F625103
:100700006421686F675167254A6E685168214B6E96
:1007100067C34CF068C34DF0030EB5ECEFF0E8048E
:10072000FCE14A504C240301676F4B504D20686F29
:100730006351615D4A6E625164554B6E6FECF0F02F
:1007400067C33EF068C33FF0B8ECFDF03EC067F30E
:100750003FC068F367C365F367C34AF068C34BF0F3
:100760004C6A4D6A4D34000E4D1809E6D880FF0ED4
:100770004A54000E4B54000E4C54000E4D5402E2ED
:100780000301656912004BC101F02C50100B0BE105
:10079000D9ECEFF008E26C0E015C016E0A0E2E5DE2
:1007A00002E1040E015E12008EECF1F007E035501C
:1007B000400B04E1050E005C01E0000C010C04821A
:1007C000F3DF000901E00492358604A235963598DE
:1007D00054DE35B812001FECE8F0049A0498049631
:1007E000030E005C01E10486000403E0020E005CDD
:1007F00001E104882350400B01E10CD12350100B80
:1008000001E008D13450080B01E104D102012D515F
:1008100001E000D11A50010B01E1FCD004820494E4
:10082000C3DF000901E00492040E005C01E10484CE
:10083000AADF0150FC0BE842E842026E32A01CD055
:100840000201895107080AE20150E840E840E84007
:100850001F0B015C525D09E2522B07D0445105E1A8
:10086000525103E05207040E446F5251D880015494
:1008700005E25251015E02D00201526B0490045015
:10088000040B03E00250EB5D08E30450040B01E0AD
:1008900072D001500101D45D6EE20101320E076F8A
:1008A0000A0E2E5D02E1040E07270201BB51105D06
:1008B00002E3000E01D0010E049CE8B0048C480E47
:1008C0000F5D710E105901E396D003016C0E635D4C
:1008D000000E645901E38FD02FECE7F00CE02150BB
:1008E000800B05E06C0E010107254B5D04E0045010
:1008F000400B01E180D004B20BD00101D451015C66
:10090000020D2DECE6F00F5002010F27105005D01C
:1009100004A405D002010F2B000E10236BD002019E
:100920002E5169E10A0E2E6F0150EC5D22E2EC516E
:1009300020E004A802D0020E2E6F0450080B14E031
:10094000FDECECF007E0020EB65D04E00201895117
:1009500001080AE2320E02010F27000E10232F5168
:1009600007E02E912E4304D00A0E0F27000E10230D
:100970000480EC6B40D00450040B05E002500201EF
:10098000D880EB5508E30450040B35E10150010118
:10099000D880D45530E2020E036E04A402D0010EBA
:1009A00007D004A206D0320E036E04A802D0960E21
:1009B000036E03500F6E106A0450020B06E00450E1
:1009C000080B0EE002012F510BE001500101D45D34
:1009D0004A6E4B6A6FECF0F082ECF4F069ECF3F0E5
:1009E00002010F510F5C1051105805E20F500F5FBC
:1009F0001050105B048004A00DD0020111510F199A
:100A000002E11251101906E0E5EC0BF00FC211F2F1
:100A100010C212F20201305102E00F0E306F1200CC
:100A20001850100B0CE03A0E165C3CE0170E165CEA
:100A300039E02A0E165C03E1B1ECEFF033E0185018
:100A4000010B06E0190E165C2DE02D0E165C2AE057
:100A5000350E165C27E0250E165C24E00E0E165CA3
:100A600021E0080E165C1EE0390E165C1BE0380E05
:100A7000165C18E0A2ECB6F0000914E1090E165C51
:100A800007E11850100B04E0DAEC1DF000090AE150
:100A90002150800B06E102017E5103E03350200B10
:100AA00001E0000C010C020EA4ECECF0909C908E86
:100AB000010EE66ECEECFDF0E552FFEC1DF011EC00
:100AC000E7F003E0720EC6ECE5F0F8EC18F0060172
:100AD0005091120071C24BF172C20FF273C210F248
:100AE000E5EC0BF083EF28F00101AD5103E12C821E
:100AF000A9C108F02150010B12E068ECE6F00FE10B
:100B00001850800B03E001ECEDF006E02150040BDF
:100B100006E18150010B03E095D945EC8DF0120000
:100B20000101050EAC6F2150010B05E01A50020BBC
:100B300002E0AC6B120034BE13D05EC100F00A0EAE
:100B40002E5D05E17A51080B02E10A0E0026020132
:100B50000E51D880005404E20E51005C0101AC6FCC
:100B6000120073ECF2F00101E49952ECE7F002E0BC
:100B70000101E4892550020B04E11D50010B01E045
:100B8000238C23BC06D0E66AE66AC80EDFECE5F0EB
:100B900010D0B1ECEFF00BE13450080B08E05AEC48
:100BA000EEF003E0E0ECF2F0FDE172ECECF0E5ECED
:100BB0000BF002010A0E2E6FEC6B21AE1D84C80EE5
:100BC0002F6FF1EC18F0780E006E00505EECE9F03B
:100BD00092EC1DF00201326B68ECE6F003E0355058
:100BE000400B07E080EC0BF0000903E00D0EFFEC7A
:100BF000E7F02150800B06E111ECE7F003E0730E03
:100C0000C6ECE5F0909E349EBFECEBF001E0348E34
:100C10006FECF4F03EE12C50080B30E02350100B49
:100C20002DE101013D052AE016C2DFFF64ECC7F0AB
:100C3000DF500201165D22E0010E69C3DBFF020EE8
:100C40006AC3DBFF030E6BC3DBFF010EE66E0EEC27
:100C5000C8F0E552010EDB500301695D08E1020EA8
:100C6000DB506A5D04E1030EDB506B5D07E0D1EC05
:100C7000C6F084EC5EF01D82960E096E3450800B37
:100C800008E0AFECEBF005E16FECF4F002E128ECEA
:100C90000BF02150800B19E12150010B16E168EC9B
:100CA000E6F009E03550400B06E102013D510DE050
:100CB000050100510AE10101E49BAFECEBF003E018
:100CC0000101E48B02D0FEECE9F01EAC02D0ECECAA
:100CD0000BF0218C328234AE03D0909E908C6FD07A
:100CE000D5CAB1F21FECE8F0360E026E380E036E74
:100CF000005003E03550400B03E051C1D5FA12D04B
:100D00009FEC0BF0000904E087C1D5FA03680AD014
:100D1000050E005C05E10A01D56B0368026802D08C
:100D200058C1D5FA0A01D55161ECEEF0016E0250BE
:100D3000015C04E30350D880015403E2750E7BECA0
:100D4000E6F09BEC5DF00101E4B91AD0B9C194F270
:100D500070ECF3F03FC095F2FCEC38F0B9C192F2C0
:100D600070ECF3F03FC093F220A20AD0BEC192F221
:100D70004CECE6F0BFC13FF0FCECFDF03FC093F25D
:100D8000909E908C0101E4B91AD020A203D00701F3
:100D9000576B586B02019451925D0EE19551935D32
:100DA0000AE0B5ECE8F008E102019529935D03E063
:100DB0009505935D01E12A84308ED8EC3EF09CECE1
:100DC0000FF007011B991B9701013EA904D00701F1
:100DD0001C6B1CC71BF757ECECF00201FA0E336FCB
:100DE000248A2682329223AC02D00601508146EC3E
:100DF0004BF00201295109E00101E451080B05E122
:100E0000140E28ECE6F00101E487040EE15C02E236
:100E1000E16AE552E16EB3EFE5F00FECF0F00501A9
:100E200011071251EA6A150FE96E050EEA22EFCF9B
:100E3000DFFF122B12511F0801E2126BDF50E55247
:100E4000B3EFE5F053EC29F002012A6B2AC26AF2F3
:100E5000B6ECECF007E0200E01011F5D03E0200E70
:100E60000CECE7F00101AD6B006A19EF92F00FECAA
:100E7000F0F00850DF6E02011E0E316F05010051C7
:100E800002012A110BE01E50040B06E01E50080B55
:100E900003E08150080B02E1D5DF71D308503AE13D
:100EA000345101E06CD30101EE9521B002D059DE3E
:100EB0000ED068ECE6F006E002013D5108E00501C5
:100EC000005105E1AFECEBF002E1FEECE9F0B1EC32
:100ED000EFF014E10201B5A50FD0330EB35D09E1C7
:100EE0000101E3AF0BD003EC05F00201330E4D6FAF
:100EF00005D003EC05F002D008EC05F00101E4A9EF
:100F000002D0AC6B32D10CDE050E01018903F35027
:100F1000AC272BD1080430E10101AC5101E02BD307
:100F2000209C6FECF4F002E0208C0FD03450800B4A
:100F30000CE1AFECEBF009E128EC0BF00101E4ABC4
:100F400002D0FEECE9F00101E49B2E50200B03E1FE
:100F50002050020B04E0E5C2E6FF41ECEAF001019B
:100F6000280EAC6F23A802D0AC9FAC4721AE02D0B4
:100F7000050EAD6F082A0AD0020E085C09E10101D6
:100F8000AC5102E1DFEC83F032EC0BF0ADDDF3D2DB
:100F9000030E085C42E12CA226D05EC1ACF1B5EC98
:100FA000E8F005E17A51080B02E10A0EAC27E4B93A
:100FB000AC6BAD5104E0050E8903F350AC272C92C5
:100FC0002150010B04E01A50020B01E0AC6B68ECFD
:100FD000E6F006E002013D5103E13550400B03E02D
:100FE000006A19EC92F00101AC5106E068ECE6F001
:100FF0000FE03550400B0CE12050400B05E10201A1
:101000003D5102E12DEC0BF00101280EAC6F3BD1FC
:1010100027B8B1D2DFEC83F0AED2050E085C68E1F0
:101020000101AC5101E0A7D2082A279821B059D07C
:101030001C0E016EE4A902D0140E016E8951E82441
:101040000124006E02018D5107E000508D5D04E225
:10105000090E086E278845D03282909C219C34BEB0
:1010600010D0B1C2D5FA9BEC5DF00101E4B909D012
:10107000FCEC38F020A203D00701576B586BD8EC7A
:101080003EF007011D990101E8A102D007011D8969
:1010900007011D970101E8B102D007011D87070173
:1010A0001B990101E8A302D007011B8907011B97C7
:1010B0000101E8B302D007011B8701013EA905D059
:1010C000B2C2E6FF7DEC5DF0E55257ECECF068EC67
:1010D000E6F003E03550400B03E00101050EAC6F74
:1010E00032920101E4A902D0AC6B45D219DD43D2A2
:1010F000060E085C3CE10101AC5101E03CD221B09C
:1011000032D02750100B14E13E51080B0FE135513E
:101110000DE0EE51040B0AE168ECE6F003E0355017
:10112000400B04E001013F51800B02E1BCDC11D017
:1011300035C132F227A80DD052ECF5F089C13FF04D
:1011400092ECF1F0006E00500201325D02E200C04C
:1011500032F22E50200B03E12050020B04E0E5C2D6
:10116000E6FF41ECEAF002016B6B082A04D2070E9D
:10117000085C2EE10101AD5119E118AE15D001EC6A
:10118000EDF003E069ECB7F00FD0B0EC0BF0000924
:1011900004E10101EE51040B07E0100E165C03E1BF
:1011A0000101EE8101D0189EA9C108F002013D5154
:1011B00001E0E1D13A5106E03550400B03E11FEC6C
:1011C000EBF003D0E66AE66AE66AAAEC30F037D0C4
:1011D000080E085C4AE10101AD5106E01E50040B07
:1011E00003E01E50080B02E1A9C108F002013D51C5
:1011F00001E1C1D1DFEC83F032EC0BF002013E5192
:1012000001E0B9D18BEC0FF0000901E1B4D1050187
:10121000020E146F115115E000DE006E10ECEAF0C2
:1012200018E0016A0501115102E0F7DD016E00507E
:10123000E66E0150E66EE70EE66E57EC18F0E552EA
:101240000ED000510FE1006A10ECEAF002E1030E4B
:10125000006E0050E66EE60EE66E53EC18F0E552B6
:10126000E55289D102013D6B86D1090E085C2BE164
:101270000101AE417F0BAE25D880AE5506E20201DA
:101280008D6B8DC2AEF1050E75D181B674D1010E94
:10129000AE6F320EAC6FE4A902D0280EAC6F010E17
:1012A000086E68ECE6F006E002013D5103E13550BE
:1012B000400B05E0AFECEBF002E1FEECE9F00101E0
:1012C0000B0EA96F58D10A0E085C06E122BA9ED017
:1012D000189E0B0E086E9CD00B0E085C01E09BD094
:1012E0001850800B3CE12150010B06E02150040B0B
:1012F00003E18150010B33E168ECE6F003E0355087
:10130000400B0CE02150800B09E18150080B06E0F6
:101310001E50040B03E01E50080B21E168ECE6F0C0
:101320000CE03550400B09E12150040B06E18150DF
:10133000010B03E071ECEDF012E02150800B0CE0AA
:101340008150080B0CE01E50040B09E01E50080BE6
:1013500006E08150010B03E06FECF4F04DE018AEB5
:1013600018D001ECEDF005E069ECB7F0000911E1EF
:1013700006D1B0EC0BF0000904E10101EE51040BC1
:1013800008E0100E165C03E10101EE8102D0189E08
:10139000F6D068ECE6F014E03550400B11E111ECAA
:1013A000E7F00EE11AAA04D0A2EC0AF0D9EC22F080
:1013B00001018B5105E08BC1E6FF36EC29F0E552C7
:1013C000AEC18DF20101AE5102E0010EAE6F27A851
:1013D00002D0DFEC83F00701D36B030E086E01012E
:1013E000800EA96F2150800B03E11850800B08E09C
:1013F00021940C0EA96F04D023A802D0C8ECC8F029
:101400000101AC5105E12750100B02E1DFEC83F044
:1014100032EC0BF0B0D00C0E085C01E0ACD022BA7C
:10142000AAD0F6ECB9F021AEA4D01E50040BFDE01A
:101430001E50080BFAE08150080BF7E02B840101E5
:10144000B29B248AB29926829B510CE020A203D041
:101450009BC1D3F102D09BC10CF0FCEC38F0198C8D
:10146000AFEC80F023A803D06AEC85F06ED0320E8A
:10147000026EB5ECE8F002E1040E0226140E030140
:10148000655D5EE22C50100B04E0640E01014B5DC3
:101490000BE02C50100B54E1320E01014B5D04E0C7
:1014A0006C0E02244B5D4CE123EC15F010C200F0F1
:1014B00000504C6E4D6A0050C3ECE6F04BC100F09A
:1014C0002FECE7F004E06C0E01014B5D006ED6ECF2
:1014D000F1F06FECF0F06CECE6F0000E24ECE7F0CD
:1014E0002CE27D0EDDECEFF028E20F5018ECEAF074
:1014F0002FECE7F025E00201710EBB6F030EFDEC4F
:10150000F0F0BBC23FF092ECF1F0006E005002012F
:10151000D880105504E3030E1003F3CFBBF2100E76
:1015200001012E03F350056E680E0A6E0CECEEF00E
:101530000550CEECF0F00A6A03D0780E7BECE6F0B2
:1015400019A803D06AEC85F01998219E52ECE7F0B7
:1015500003E0B9EC4BF005D0010EE66E66EC4BF003
:10156000E552239850ECEAF0010139BF02D06CEC4F
:10157000EFF0800E086EDF50085C01E01D8CE55234
:10158000B3EFE5F03050100B0CE10701825109E197
:1015900001013E51200B06E076ECEAF003E0E05159
:1015A00001E1000C010C070EE66EE66A200EE66E05
:1015B000440EE66E060E7DEFECF045C644F646C6D8
:1015C00045F647C646F648C647F649C648F64AC6EF
:1015D00049F6120049C64AF648C649F647C648F6D3
:1015E00046C647F645C646F644C645F60601200EF1
:1015F000446F1200AEECE5F00101EA51EB1103E09B
:101600000D0E85ECE8F0EC51ED1103E00A0E85ECCF
:10161000E8F032AA02D0AFECF0F00101E451020B85
:101620000CE0280E0901BD5D08E2BD51BD2BEA6A40
:10163000950FE96E090EAFECF3F0B3EFE5F0CBECEC
:10164000F3F01B50010B0AE0800E1DECE6F004E203
:10165000FE0EDB50200802E11B905CD0AEDFFE0ED8
:10166000DBCF4AF6DB50800804E0850E1DECE6F087
:1016700003E30601200E21D0FE0EDB50300803E10B
:101680000601630E1AD02A50200B1CE02950080BCB
:1016900019E1DF6A150EDF5C15E249ECF3F00FE1AA
:1016A000DE52010EDD6EDF2A9DECE8F006014A6F86
:1016B00084DFDF2A9DECE8F006014A6F03D0030EB9
:1016C000DF26E8D776ECEAF012E0010EDB5004E00A
:1016D00049C6E6FF8FDFE5524AC600F0630E005CA4
:1016E00002E1300E006E0050E66E84DFE5524ADF04
:1016F000000910E08EECE8F044C619F145C61AF175
:1017000046C61BF147C61CF148C61DF149C61EF16D
:101710004AC61FF1020EE15C02E2E16AE552E16EA7
:10172000B3EFE5F00FECF0F00850DF6E2492100EEE
:10173000085C13E11C0E086E02016651010B03E107
:101740001E50040B02E1110E92D06651040B29E1E8
:101750001E50080B01E0ACD024D0110E085C0AE149
:101760002480238E0201080E666F2482086A01011C
:10177000120E9DD0120E085C07E124902482030E05
:10178000086E0101130E93D0130E085C0CE11C0EC1
:10179000086E02016651040B04E11E50080B01E0C3
:1017A00087D0140E64D0140E085C11E12480238EBF
:1017B000180E086E1E50040B01E07AD01E50080B64
:1017C00001E076D02482086A0101150E70D0150E52
:1017D000085C0BE101012DAF03D00201020E666F20
:1017E000239EEAECECF0160E62D0160E085C04E1C3
:1017F000EAECECF0170E5BD0180E085C08E1020171
:10180000020E666F2482086A0101190E50D0190E6B
:10181000085C05E1239EEAECECF01A0E48D01A0EA3
:10182000085C04E1EAECECF01B0E41D0170E085CFA
:1018300008E101012DBF03D00201020E666F1B0EED
:1018400016D01B0E085C05E12490238E2482030E23
:101850002BD01C0E085C2CE12490800E086E020137
:101860006651010B03E11E50040B03E1110E086EDB
:101870001FD035AC03D009ECF5F01AD01850800B0E
:1018800017E1A9ECEFF004E0090E0201685D0AE33C
:101890000601F05104E0080E0201685D03E3020155
:1018A0003D5106E02482080E086E0101100EA96F5A
:1018B00024A202D008EC81F0DF50085C01E01D8C0E
:1018C000E552B3EFE5F01AECF0F001013EB902D0B9
:1018D0001D9601D01D761D50080B01E0010E076E0C
:1018E0005951400B18E0D3EC09F0050814E002014F
:1018F000325111E133510FE134510DE1800E0814E2
:101900000AE02D50080B07E11E50400B04E1255062
:10191000010B01E102D822EFF0F0AAECF3F0D4C7FA
:10192000DFFF020EDB6A35A003D0010E1FECE7F0EB
:10193000010E7BC1DBFF1DA615D0020EDB6A1DA8C0
:1019400003D0010E1FECE7F001018DBD0BD0010E9D
:101950007CC1DBFF8D0EF7ECE7F0006E0EEC34F08F
:101960000050DF6EB7ECEBF003E2010E05C7DBFFC2
:10197000010EDB50DF5C0EE3020EDB5003E04E0E87
:10198000C6ECE5F0020EDB6A0201FA0E336F28A8FE
:101990000CD009D0020EDB5002E11DEC09F0010E63
:1019A0001FECE7F002010A0E336F1DA606D01D984A
:1019B000020EDB5007E01D8805D03590020EDB508B
:1019C00001E03580030EE15C02E2E16AE552E16E7E
:1019D000B3EFE5F002016B6BE66AE66AE66A45EC96
:1019E000E9F002013A6B0701D56BD5C7D4F121B0FC
:1019F00003D02180B1EC85F012000FECF0F0020171
:101A0000050E3D6F280E3E6FE5DF10ECEAF007E1B2
:101A1000DF6A99A102D0060EDF6E23ECF2F0050119
:101A2000040E146FE552B3EFE5F0358C210E69EF2B
:101A3000F1F00101E251020B13E03F51800B10E184
:101A40002150010B0DE12150100B0AE12550020B32
:101A500007E1E2933088190EDBECE5F0AA0E096E7F
:101A6000120001013F51800B04E12150010B01E103
:101A7000000C010C01015951800B05E0020E005CC5
:101A800003E0000401E0000C010C0FECF0F063EC4B
:101A900011F0000909E0030EDF6E010199A102D0E7
:101AA000070EDF6E23ECF2F021902194198C0701D0
:101AB000D36B0201325102E0010E326F56ECEAF0B4
:101AC000E552B3EFE5F081B003D01B0EDBEFE5F09C
:101AD00081B603D01A0EDBECE5F012000850CDEC15
:101AE000ECF031E14B502FE11A920101E4A503D053
:101AF000E49522EC1EF00101E451080B08E02150AE
:101B0000400B05E1120E28ECE6F00101E49735AC3C
:101B100002D009ECF5F021B00CD063EC11F0000913
:101B200003E0006A19EC92F0229602017E5101E175
:101B3000208622AE06D0010EE66EE8EC0AF0E552F1
:101B4000229E082A1200085040ECEBF001E0C8D1B8
:101B50004B5001E0C5D121A0239C1CEC16F0FF08DE
:101B600001E0F4D02E50400B01E0F0D02150200BCA
:101B700001E1ECD01950800B01E0E8D02850010BB6
:101B800001E0E4D00101EE51010B01E0DFD00201E0
:101B90008D6B8DC2AEF11A921FECE8F0359C1D9052
:101BA0008150080B18E1005006E02050020B13E1B1
:101BB00061DF000910E00101010EAE6F1A82086AB0
:101BC0000B0EA96F005003E14CDF000901E01D80FE
:101BD000005033E134D01E50040B03E01E50080BBC
:101BE00030E1005013E02050020B03E143DF000915
:101BF0000DE10601F25125E063EC11F0000906E168
:101C00002050020B1EE111ECE7F01BE01EB402D0E5
:101C1000110E05D01EB604D00201666B140E086EBC
:101C2000005003E11EDF000901E01D80005007E0C5
:101C3000030E0C5C02E1E1DE89D0F7DE87D0F9DE2D
:101C400085D0050100511CE0005003E011ECE7F0E5
:101C500010E0005003E105DF000901E01D800050A5
:101C600001E1E7DE11ECE7F001E0C7DE1E0E086ED1
:101C70006DD0268E810EA3ECE9F04BEC29F066D0F6
:101C800021AE04D0086A01010A0E47D0005048E096
:101C90008150010B06E02150040B03E171ECEDF0E3
:101CA0003FE002012A5114E071ECEDF007E123EC72
:101CB00009F000090DE18150010B0AE102014A6BB4
:101CC0004B6B2A6B2AC26AF2A2EC0AF055EC81F047
:101CD0006FECF4F007E08150010BFDE071ECEDF0EA
:101CE000FAE130D0A9ECEFF00FE01A50400B0CE015
:101CF000800EE66E030EE66E990EDFECE5F0B0ECBA
:101D00000AF09E0EEDECE7F002013A6B3AC2D5F70D
:101D10003AC2D4F1086A01010B0EA96F1D8016D0DA
:101D2000005014E12150010B11E18150010B03E03F
:101D30002150040B0BE00101E2936FECF4F004E09E
:101D400081A0FED7219412001D8044DE2150200B7B
:101D500004E1C1EC0BF0000907E10201475104E185
:101D60000101EE51010B28E00501006B2190219447
:101D7000810E086E0101EE51010B03E002017E515C
:101D800007E1A1DEC1EC0BF0000902E009C047F257
:101D90001BEC08F00101EEA10FD0B0EC0BF0000934
:101DA00007E10101EE910201476B010E096E04D0BB
:101DB00021AC02D056ECEAF0085040ECEBF001E127
:101DC0004B502FE06AEC98F002013A6B30AA02D037
:101DD000C3EC69F031A402D07CEC6CF031AC02D0E1
:101DE00012EC6BF025A002D030EC6AF033A002D0E8
:101DF00074EC6AF024AE02D0CCEC68F020A802D0DB
:101E0000A2EC12F02D50800B03E12D50400B02E0AC
:101E100096EC0FF0269A1BAC02D038EC0AF01D8C21
:101E200012002150010B14E002013D5111E1185044
:101E3000800B06E001ECEDF009E0250E165C06E0F3
:101E40002150040B05E18150010B02E045EF8DF0BC
:101E500002013A5104E01FECEBF045ECE9F018AE5A
:101E60006BD069ECB7F0EEECE8F017E03050200BE7
:101E700014E13150040B11E12450800B0EE131507C
:101E8000400B0BE12550010B08E13350010B05E13C
:101E90003350020B02E175EC38F0339220AA4CD09B
:101EA000209A01013EAB48D08EECE8F0020142518D
:101EB00010E1CCEC43F00D0E165C11E11850010B53
:101EC0000EE00C500101D35D0AE10201C80E426F21
:101ED0001200426B1C0E76ECE9F0960E096E1200B1
:101EE00078ECECF029E14B5027E12250200B24E163
:101EF0000101E651800B20E103EC08F0000910E13C
:101F0000F6ECF1F014EC33F00D0EC6ECE5F00C50ED
:101F100002E03C0E01D01E0E3EECE6F068ECEEF066
:101F200054EC0EF0248A810E086E03EC08F00009D0
:101F300003E075EC38F0268212000D04040F07014F
:101F4000006F04A002D0040E002712000101B29B12
